:020000040000FA
:107800005469616E59696E673130300000000000C4
:1078100054593230302E303830303030625F747925
:10782000424154333247313339474B3634464200B4
:1078300043414E5F5354440000000000000000002C
:1078400043414E5F43485F300000000000000000ED
:1078500043414E5F3530304B6270730000000000D2
:10786000E8070000E0070000DF070000000000005C
:020000040000FA
:1080000058330020DD800000E5800000E78000009C
:108010000000000000000000000000000000000060
:10802000000000000000000000000000EF800000E1
:108030000000000000000000F3800000EDC401001B
:10804000D51301001914010049140100791401002D
:10805000A9140100D9140100091501003915010006
:108060006915010099150100CD150100E115010008
:10807000F115010025160100351601004516010015
:1080800079160100BD160100051701004D1701000A
:1080900095170100DD170100ED17010021180100FF
:1080A0005518010085180100B9180100ED180100EC
:1080B000FD1801000D190100411901007519010099
:1080C000EF3FE8FF0448854600F02CFA00480047DF
:1080D00049090200C046C046583300201648804770
:1080E00016480047FEE7FEE7FEE7FEE7FEE7FEE78D
:1080F000FEE7FEE7FEE7FEE7FEE7FEE7FEE7FEE758
:10810000FEE7FEE7FEE7FEE7FEE7FEE7FEE7FEE747
:10811000FEE7FEE7FEE7FEE7FEE7FEE7FEE7FEE737
:10812000FEE7FEE7FEE7FEE7FEE7FEE7FEE7FEE727
:10813000FEE7FEE7FEE70000EDCA0100C580000093
:1081400030B50B46014600202022012409E00D46EF
:10815000D5409D4205D31D469540491B2546954077
:1081600040191546521E002DF1DC30BD70B50024BB
:108170002546002801DA01244042002901DA0125C0
:108180004942FFF7DDFFAC4200D04042002C00D056
:10819000494270BDF0B51FB40646002082B00546C6
:1081A0004024019100901BE0019922460F46304681
:1081B00000F066F9049A059B801A994110D3104685
:1081C0001946224600F04CF9361A8F410197224693
:1081D00001200021009F00F043F938184D41009024
:1081E0002046641E0028DFDC019B009829463246A9
:1081F00007B0F0BDF0B51FB486B00020009001902C
:1082000002900698069980B204900798090C02041F
:108210000014114307900027089D099806913E46D7
:108220003C4603900398A9B20204000C0390049802
:108230002D0C154348430021224600F011F9C719BF
:10824000714110340E46402CECDB3846029A00F0A7
:1082500007F9009A019B80180090594102980191FA
:10826000103002904028CCDB00980BB0F0BD0346E4
:108270000B439B0703D009E008C9121F08C0042A5A
:10828000FAD203E00B780370401C491C521EF9D24D
:108290007047D2B201E00270401C491EFBD2704709
:1082A0000022F6E710B513460A4604461946FFF7C2
:1082B000F0FF204610BD30B504460020034600E024
:1082C0005B1C934203D2E05CCD5C401BF8D030BD18
:1082D0000321001D401E037812021A43491EF9D5DE
:1082E00010467047034603220870000A491C521EBC
:1082F000FAD518467047024670B54A40D30FDB07DF
:1083000040002DD04A002AD0010E140E00021202A5
:108310000919400A520A8418E50104465443000A28
:10832000120A2E045043A4194219200CC543AA185E
:10833000120C0125AD03521C521912047F3924047A
:1083400000D0521C104301D44000491EC2B20C069A
:10835000C0092018401C4008802A02D003E00020F9
:1083600070BD40084000002900DA0020184370BDAD
:1083700070B502464A40D50F40004A00ED0740085C
:108380005208002814D0002A12D0C40DD30D410287
:108390000120C0055202490A520AE41A09181218AB
:1083A0007D34914201D3641C00E04900002C01DAC5
:1083B000002070BD0023914201D3891A0343400875
:1083C00049000028F7D100290AD0914202D10121A9
:1083D000C90705E0914201D2012101E00121C94311
:1083E000E005C018401900F05CF870BD10B500221F
:1083F0009623114600F05DF810BDC20FD207400071
:1084000040080BD0C10D0723DB01C9184002090544
:10841000400A1143C208400711437047002001463B
:108420007047000010B5002904DB0124E407404236
:108430008C412146002B04DB1C460123DB07524202
:10844000A341994200D1904210BD00000122D20701
:10845000002800DB101A002900DB511A88427047FF
:1084600010B5202A04DB0146203A9140002010BDBF
:10847000914020239C1A0346E3401943904010BDCD
:1084800010B5202A04DB0846203AD040002110BD58
:108490000B46D340D0402024A21A914008431946ED
:1084A00010BD002904DA401C490001D140084000F9
:1084B000704770B40024050C05D11024000402D1CB
:1084C000002921D01124050E01D100020834050F26
:1084D00001D10001241D850F01D18000A41C0028BA
:1084E00001DB4000641C002908D020252E1B0D460E
:1084F000F540A14000D001212943084301061B1B80
:10850000000ADB1D02D5002070BC7047DB0518187F
:1085100080180029F8DA401C4900F5D170BC4008E9
:1085200040007047064C0125064E05E0E36807CC85
:108530002B430C3C98471034B442F7D3FFF7C6FDE9
:10854000841D0200A41D020070B58C180578401C23
:108550006B075B0F01D10378401C2A1106D102780A
:10856000401C03E006780E70401C491C5B1EF9D1CC
:108570002B0705D40023521E0DD40B70491CFAE7BB
:108580000378401CCB1A921C03E01D780D70491C27
:108590005B1C521EF9D5A142D8D3002070BD70B526
:1085A00007F086F80524204618F088F900252846AB
:1085B00007F072F8204618F081F90126304607F0DE
:1085C00047F8204618F07AF9284607F041F8204687
:1085D00018F074F9304607F05FF8204618F06EF98D
:1085E00070BDB0B507F064F80524204618F066F9B0
:1085F0000125284607F050F8204618F05FF9284674
:1086000007F026F8204618F059F9002007F020F866
:10861000204618F053F9B0BDF0B581B007F034F83A
:10862000052018F04BF908270026012007F010F864
:108630000524204618F042F9204618F03FF907F0CB
:1086400019F80546204618F039F9002007F000F81F
:10865000204618F033F976002E437F1E3806E4D109
:10866000F0B201B0F0BD70B50446002006F0F0FF96
:1086700007F01EF8052018F021F90826E0B2C0091D
:1086800007F00AF80525284618F018F9012006F029
:10869000DFFF284618F012F9002006F0D9FF28461F
:1086A00018F00CF9284618F009F96400761E300617
:1086B000E4D1052018F002F9012070BDF0B583B0B7
:1086C000019314460E4607460120384302900325C5
:1086D00004E000F08EF86D1E280631D000F067F837
:1086E0003846FFF7C0FF00F0A7F80028F1D1304668
:1086F000FFF7B9FF00F0A0F80028EAD100F057F822
:108700000298FFF7B0FF00F097F80028E1D1019838
:1087100002280BD3451E0026FFF77EFF2070FFF7CF
:108720003EFF641C761CF0B28542F5DCFFF774FF57
:108730002070FFF756FF00F05CF8202003B0F0BD7A
:10874000102003B0F0BDF0B583B01C46009201913B
:108750000290032504E000F04CF86D1E280623D09B
:1087600000F025F80298FFF77EFF00F065F800287A
:10877000F1D10198FFF777FF00F05EF80028EAD109
:10878000002C0CD00026009F3878FFF76CFF00F01B
:1087900053F80028DFD1761C7F1CA642F4D300F0EA
:1087A00028F8082003B0F0BD102003B0F0BDB0B52C
:1087B00006F07EFF0524204618F080F801252846A3
:1087C00006F046FF204618F079F8284606F064FFC8
:1087D000204618F073F80025284606F05DFF204675
:1087E00018F06CF8284606F033FF642018F066F89D
:1087F000B0BDB0B506F05CFF0524204618F05EF869
:108800000025284606F024FF204618F057F8284691
:1088100006F042FF204618F051F80125284606F0E0
:1088200017FF204618F04AF8284606F035FF642066
:1088300018F044F8B0BD0000B0B506F025FF0524DF
:10884000204618F03BF8012006F002FF204618F001
:1088500035F80B4D06F00EFF044606F0F3FE002C33
:1088600002D06D1E2804F5D10525284618F026F8FB
:10887000002006F0EDFE284618F020F82046B0BD96
:1088800033210000034801780B2901D8491C0170ED
:108890007047C046472F002070B584B0002503956F
:1088A00002950195009506F0CDFE0F20C6430E4CB3
:1088B0001036F1B2A0206A461023FFF744FF20468D
:1088C00017F0FCFF204617F0F9FF912EF0D3A020FF
:1088D000B0216A461023FFF736FF204617F0EEFF5F
:1088E0000248058004B070BD581B00003A2F0020DC
:1088F00070B5022902D2EB24E0B270BD891EEB25CF
:108900000022134605E0401C5B1CDDB2A94225464F
:108910000EDB04786C40154604E034466E1C072DCF
:108920003546F0D26608E407F7D09A246640F4E7AB
:10893000E0B270BDF0B591B00C91417810AA117001
:1089400083781B025918C37804792402E3181B04A6
:1089500059180B0ED3700C0C94700D0A55700B91B6
:1089600008956918099409190A93C9180278D2431D
:108970008918427983791B029A18C379047A2402F0
:10898000E3181B049A188918130A0693C918130CC4
:108990000593C9180792120E04928918827AC37A35
:1089A0001B029A18037B0F90447B2402E3181B04DC
:1089B00098180918020A02928918020C0192891863
:1089C0000D910390000E0E9000200346014606E034
:1089D00032409A40D2B211435B1C082B0ED00126C4
:1089E00035469D400746024602E07F1C042FEFD02B
:1089F00010ACE45D2542F8D0521CF6E70E9C0D98B1
:108A00000019C3B20F98827B934205D0427A9142FB
:108A100002D1002011B0F0BD1021FFF769FF0C99C1
:108A2000CC72019A8A72029A4A72039A0A72049A62
:108A3000CA71059A8A71069A4A71079A0A710A9A46
:108A4000CA70099A8A70089A4A700B9A0A7011B013
:108A5000F0BDF0B58DB055220270002747720B783B
:108A60004370CA79059202728A790492C2714A7976
:108A7000039282710A7902924271CA7A0892427311
:108A80008A7A019202734E7AC6720C7A84720CAAA8
:108A900013704D782D02EB188D78C97809024919A9
:108AA0000904CB18190E01711D0CC57009931B0A1E
:108AB0000B90837038460A91D17007959570069394
:108AC000537031020919089A1202019BD21812043C
:108AD0005118089103990902029A8918059A1202FD
:108AE000049BD2181204511805913D463A4605E000
:108AF0002640AE4032436D1C082D0ED00124214685
:108B0000A9400346064602E05B1C042BF0D00CAFE4
:108B1000FF5C3942F8D0761CF6E70B9B5A72099835
:108B200006994018079940180A994018059A801824
:108B3000110A4018110C4018110E4018089A80189C
:108B4000110A4018110C4018110E4018563898732D
:108B500010211846FFF7CCFE0DB0F0BDF0B58FB078
:108B60000446FF20E070A07060700F20C0430290A8
:108B70000F302070704817F0A1FE70490868632814
:108B800001D8642008606E4F002038806D4E01903F
:108B9000308008E00B99814222D338881030388029
:108BA00080B2A1286DD206F04DFD3978A02003AA2D
:108BB0001023FFF783FD30802028EED103AD0BA9F1
:108BC0002846FFF7B7FEE97B8842E6D1287855288A
:108BD000E3D15D48017800290298DBD10846D9E746
:108BE0003888A0284DD8C0B20021019105E006F0D8
:108BF00029FD3988C8B2A12943D2C1B2A02003AA55
:108C00001023FFF75BFD3080398810313980202830
:108C100037D103AD07A92846FFF78CFEE97B8842D0
:108C2000E5D128785528E2D14748007800280299F4
:108C300000D1014607988842D9D240490A68962156
:108C400051430B9A824208D90818904219D30BA9B4
:108C50000E222046FFF70BFBC9E78918814210D38B
:108C600007A90E222046FFF702FB0BA80A99818173
:108C700007980B9008980C9009980D9038880190EF
:108C8000B5E72078617809020818A178E278120225
:108C9000511809040818401C24D100200190388084
:108CA000A020B02103AA1023FFF708FD3080202860
:108CB00018D103AD0BA92846FFF73CFEE97B88429B
:108CC00010D1287855280DD11F480078002800D1F0
:108CD00002900B980299884204D20BA90E222046DA
:108CE000FFF7C5FA2078617809020818A178E278C0
:108CF0001202511809040818401C0CD10020E0721F
:108D0000A07260722072E071A07160712071E070D9
:108D1000A070607020700198388020786178090216
:108D20000818A178E27812025118090408180749B6
:108D3000086030880FB0F0BD70110100342F0020A2
:108D40003A2F0020302F0020332F0020402F00200A
:108D5000F0B581B000910646214800250570002A33
:108D60002ED01446C036631B71190F200840102204
:108D7000101A834200D303461A480278102A01D001
:108D8000042A1AD1C809FE2707405F2F13D80127EC
:108D9000B8436038C0B29E3282420CD3009A521956
:108DA000C9B2DFB23B46FFF789FC0F490880ED19D5
:108DB000A542D8D304E0082000E004200A49088036
:108DC000094801880020042902D0082900D0012088
:108DD00003490870411E8841400001B0F0BDC04603
:108DE000462F0020322F0020442F00200A4A012362
:108DF00013700A4A10700A4A11600A4A0021116071
:108E0000042801D105218901102801D11D208101EB
:108E1000054801807047C046332F0020322F0020C4
:108E2000342F0020402F0020382F0020F0B587B0CD
:108E3000994D00262E80994B1B688B4224D1994C6A
:108E40002188202925D1029000920196964C002776
:108E50002760964D964E2878062809D806F0F2FB32
:108E60002068401C2060B042F5D38D480421018069
:108E70002F70904C20880107029B31D08848202118
:108E80000180854D019E0BE001204002844908804D
:108E900006E003A8FFF762FE208081488021018060
:108EA0007F4800883F2807DD874988420BDC40283F
:108EB00012D0802810D010E004280DD008280AD045
:108EC000202809D009E001214A02904204D0C902B9
:108ED000884201D001E002262E80288807B0F0BD2C
:108EE000A128019E00D32780009A012A6A4D1ED135
:108EF000187B012856D1DF719F715F711F711F733D
:108F0000587B012804D1DF729F725F721F725F73FA
:108F100003AF38461946FFF79CFDF87320880028F8
:108F200046D01038C1B2A02003AA102344E0002A82
:108F3000B6D1614801780029B2D00270187859780A
:108F4000090208189978DA781202511809040818E9
:108F50005A490978002901D00F21C943884233D2E8
:108F6000274603AC20461946FFF773FDE0733978B6
:108F7000A02010232246FFF7E6FB029A484908800A
:108F800008288DD13888103038801078517809023F
:108F900008189178D2781202511809040818484923
:108FA00008607DE7597B012911D10128A3D0A7E7EB
:108FB000A02003AA10230146FFF7C5FB384908800B
:108FC0003D48009901706BE70120C0025EE73D4813
:108FD0000078012812D103AC20461946FFF739FD6D
:108FE000E073A020B02110232246FFF7ACFB2C49F0
:108FF00008800828E4D133480770E1E718785978E9
:10900000090208189978DA78120251180904081828
:109010002B490968214A12685118884203D2204816
:1090200040210180CCE725490978002901D00F2192
:10903000C94388422DD203AF384619461C46FFF774
:1090400008FDF8731B480178A02010233A46FFF76B
:109050007AFB134908800828B2D1164908881030D5
:1090600008802078617809020818A178E278120255
:109070005118090408181249086008490A6815219E
:109080005143FFF75DF800299AD101200D4908707E
:1090900096E70120C00291E74C2F0020342F0020DA
:1090A0004A2F0020302F0020502F0020472F002073
:1090B000818D5B003A2F00203C2F0020332F0020B1
:1090C000402F0020482F0020FF010000F0B585B0A0
:1090D0000646434C0027278004921018414A128804
:1090E000904241D201910397404F00200290386096
:1090F0003F4C404D2078052809D806F0A3FA38687F
:10910000401C3860A842F5D33748042101800298FA
:1091100020703948018839480278102A01D0042A81
:1091200032D188190346C033049C651A0F240440C9
:109130001020001B854200DB0546DC09603C01264F
:109140003002E7B27F09052F12D3B443E6B29E3254
:10915000B242234C039F0DD301984218D9B2EBB20F
:109160003046FFF7F0FA05E01F482021018011E0AA
:109170001B4C039F1C49088008280BD1E8B21E4AEB
:1091800011880818108005E0012080021649088027
:10919000134C039F144800881F2809DD202813D092
:1091A00001210A0290420FD0890288420CD00CE0C3
:1091B000042809D0082808D10F480088049988425B
:1091C00001D3022700E001272780208802210143E4
:1091D000022902D1084900220A8005B0F0BDC0462C
:1091E0004C2F0020382F00204A2F0020502F002025
:1091F000472F0020818D5B00542F0020322F00204C
:10920000F0B585B0044600200190042C6FD20CF01C
:1092100057F8002801D10CF0D3F80020009000BFCF
:109220000098401C00900CF04BF803900398002825
:1092300003D0484900988842F2D30398002856D1B9
:10924000042145480CF01EF8444845490880210196
:10925000444A515C4900404A505A41490A88012118
:10926000090300F055F902900120049020013D49C6
:1092700040184078002801D100264BE020013949F0
:1092800040184078012802D13548068842E0200184
:1092900034494018407802282AD120014018057925
:1092A0002901304A515C49002B4A505A2C490A88FE
:1092B0000121090300F02CF9064628012A49431828
:1092C0002801284940180289280140180021C76850
:1092D0003046B84706462801224BC018C2882801EC
:1092E000C0188178304600F087F8064612E02DE07D
:1092F00020011C4940184078032804D02001401860
:109300004078132804D1200116494018868801E0CE
:10931000002004900498002818D020011249431816
:109320002001104940180289200140183146C768C1
:109330000298B847019020010A4BC018C28820014A
:10934000C0188178019800F057F80190019805B095
:10935000F0BD000050C300000E0100208813000083
:10936000080100202014020060140200F8B5054630
:109370000E4614460020009001211C4801751C482F
:10938000007888431A490870084680780821084305
:109390001749887000208871084600780121084329
:1093A0001349087008460572002717E01048007836
:1093B000802108430E49087000BF0E48007D002838
:1093C000FBD000200B4908750948C0892080A41CE7
:1093D0000748C1890098081800907F1CB742E5D360
:1093E00031460098FEF7ACFE80B2F8BD4061004007
:1093F000005004404060004010B50346012908D1E8
:10940000094CA41A9C4202D99C18A0B20BE0064851
:1094100009E0022906D1934202DD9C1AA0B202E0C3
:10942000002000E0184610BDFFFF000010B5044604
:109430000121202002F00AF80020324908700121A1
:1094400031480175002031490875152016F01EFFBE
:109450002C488078E17808432A498870084680784B
:1094600021780843274988702078802806D108464B
:109470000079E17949000843224908712148807840
:10948000E17A08431F498870A078002803D1084674
:10949000007908710FE0A078012806D119480079F9
:1094A000602108431749087105E0164800798021BA
:1094B00008431449087113488079217908431149F8
:1094C000887108468079617908430E498871207A4D
:1094D000C872607A88720846007838218843094942
:1094E0000870084600786178C9000843054908708B
:1094F000A07A0873084600780121084301490870E2
:1095000010BD000000500440406100404060004039
:10951000F8B504460E461746002E01D100250FE08F
:10952000A64201DC3D460BE00094009C20467843B7
:10953000009031460098FEF703FE0090009885B237
:109540002846F8BD0146042904D28A00024BD218ED
:10955000508800E00020704724290020014604299B
:1095600003D28A00024B985C00E0002070470000A4
:1095700024290020FFB587B004460898844203DA06
:109580000A988068002802D12448019042E0089897
:10959000001B82B20292002625460A9880680021AC
:1095A0002F463A463346049605910690FEF722FE72
:1095B00005460E46002328463146029AFEF7EAFD8C
:1095C00005460E46304600210A46494050400143B8
:1095D00002D0124801901DE003950A98C068039DCF
:1095E000A84202D30020019014E00A98C1680398B1
:1095F000401A039009990398FEF7A2FD039003987F
:10960000000C0004002802D00448019002E00398F6
:1096100080B2019001980BB0F0BD0000FFFF000088
:1096200010B5084800788021884306490870012158
:1096300005480175002005490875152016F026FE1D
:1096400010BD0000005004404061004040600040F8
:10965000F8B505460E4614461F4621462846FEF735
:1096600085FD80B2F8BD0000FFB587B006460A98B8
:109670004068002801D1029035E00A9801684068EE
:1096800008180390002534460021274603980695C4
:109690000491059038462946049B059AFEF7AAFDD9
:1096A00004460D460A984068024600230190204671
:1096B0002946FEF76FFD04460D4600232046294645
:1096C000099AFEF767FD04460D46284607492140E2
:1096D000002359405840014303D00448C04302903E
:1096E00001E0A0B2029002980BB0F0BD0000FFFFB5
:1096F00010B5FE4800688079030016F0ADFD07053F
:109700009ED8F5F4F3F2F100F848006840790300C0
:1097100016F0A2FD0805138A2A8A468A638A12F087
:109720001DFE0020F1490968C873F04800684079BF
:10973000401CEE49096848717DE0ED494969EB4AF2
:109740001268D27A885C12F081FEE848006840799D
:10975000401CE64909684871E44800684079401CAB
:10976000E2490968487166E00AF08EF8002810D1D5
:1097700012F06CFEDD4800684079401CDB49096846
:109780004871DA4800684079401CD8490968487136
:1097900005E012F00DFE0020D449096848714AE046
:1097A0000AF072F8002811D1112012F04FFECF48B4
:1097B00000684079401CCD4909684871CB48006871
:1097C0004079401CC9490968487105E012F0F0FD74
:1097D0000020C649096848712DE00AF055F80028B4
:1097E0001BD1C2480068C07A401CC0490968C872D1
:1097F000BE480068C07ABE49097888420DDB002067
:10980000BA490968C872B94909684862B748006826
:109810008079401CB5490968887112F0C9FD0020A3
:10982000B2490968487106E012F0C2FD0020AF4954
:109830000968487100BF00BF32E3AC480068407C53
:10984000002817D0AA48C068002803D0A848C168DB
:10985000192088470020A54909684862A348006884
:109860008079401CA1490968887100209F490968D6
:1098700048711BE09D480068406A282807D29B4831
:109880000068406A401C9949096848620EE000205F
:10989000964909684862954800688079401C934958
:1098A000096888710020914909684871F8E28F4879
:1098B00000684079030016F0CFFC080518A42FA417
:1098C0004CA480A412F04AFD002088490968C8739E
:1098D000864800684079401C84490968487197E0CF
:1098E000D4E2C7E230E25DE194E0814949697F4A10
:1098F0001268D27A885C12F0A9FD7C480068407931
:10990000401C7A4909684871784800684079401CD1
:109910007649096848717BE009F0B6FF002811D14B
:10992000012012F093FD714800684079401C6F4996
:10993000096848716D4800684079401C6B490968A6
:10994000487105E012F034FD00206849096848714B
:109950005EE009F099FF002828D164490968C97AB6
:1099600024225143634A12688918604A1268D27BE4
:10997000885C12F06BFD5D480068C07B401C5B4951
:109980000968C87359480068C07B242814D3574815
:1099900000684079401C554909684871534800687F
:1099A0004079401C51490968487105E012F000FDFA
:1099B00000204E49096848712AE009F065FF002837
:1099C00018D14A480068C07A401C48490968C872E2
:1099D00046480068C07A4649097888420ADB002078
:1099E00042490968C872414800688079401C3F4973
:1099F0000968887112F0DCFC00203C490968487154
:109A000006E012F0D5FC002038490968487100BF13
:109A100000BF45E2354800684079030016F01CFCA1
:109A20000A0614B92BB948B978B995B912F096FC61
:109A300000202E490968C8732C4800684079401CF2
:109A40002A4909684871ABE029494969274A1268DF
:109A5000D27A885C12F0FAFC244800684079401CF5
:109A6000224909684871214800684079401C1F4913
:109A70000968487194E009F007FF002811D14A20D5
:109A800012F0E4FC194800684079401C1749096845
:109A90004871164800684079401C144909684871AB
:109AA00005E012F085FC002010490968487177E054
:109AB00009F0EAFE002824D1FF2012F0C7FC0B4871
:109AC0000068C07B401C09490968C87307480068E2
:109AD000C07B24281BD3054800684079401C0349FB
:109AE0000968487101480068407905E0D407002002
:109AF000182F0020D0070020401CEA49096848714F
:109B000005E012F055FC0020E6490968487147E07D
:109B100009F0BAFE002811D1FF2012F097FCE148AD
:109B200000684079401CDF4909684871DD480068D9
:109B30004079401CDB490968487105E012F038FCA7
:109B40000020D849096848712AE009F09DFE0028E4
:109B500018D1D4480068C07A401CD2490968C8723C
:109B6000D0480068C07AD049097888420ADB0020D2
:109B7000CC490968C872CB4800688079401CC94943
:109B80000968887112F014FC0020C6490968487100
:109B900006E012F00DFC0020C2490968487100BFC0
:109BA00000BF7DE1BF4800684079030016F054FB18
:109BB0000C0715C32CC349C366C382C39FC312F0ED
:109BC000CDFB0020B7490968C873B64800684079E2
:109BD000401CB44909684871B4E0B3494969B14AC5
:109BE0001268D27A885C12F031FCAE480068407985
:109BF000401CAC4909684871AA4800684079401C7B
:109C0000A849096848719DE009F03EFE002811D17D
:109C1000772012F01BFCA34800684079401CA14942
:109C2000096848719F4800684079401C9D4909684F
:109C3000487105E012F0BCFB00209A4909684871A0
:109C400080E009F021FE002811D10C2012F0FEFB6B
:109C5000944800684079401C9249096848719148CD
:109C600000684079401C8F490968487105E012F08E
:109C70009FFB00208B490968487163E009F004FEEE
:109C8000002810D112F0E2FB864800684079401CA1
:109C9000844909684871834800684079401C8149BB
:109CA0000968487105E012F083FB00207D490968CE
:109CB000487147E009F0E8FD002811D1132012F0A7
:109CC000C5FB784800684079401C764909684871AE
:109CD000744800684079401C72490968487105E081
:109CE00012F066FB00206F49096848712AE009F00C
:109CF000CBFD002818D16B480068C07A401C694928
:109D00000968C87267480068C07A6749097888425C
:109D10000ADB002063490968C872624800688079DC
:109D2000401C60490968887112F042FB00205D49BF
:109D30000968487106E012F03BFB002059490968A8
:109D4000487100BF00BFABE056480068407903008F
:109D500016F082FA080513872A874787638712F06F
:109D6000FDFA00204F490968C8734E4800684079E1
:109D7000401C4C49096848717AE04B494969494A95
:109D80001268D27A885C12F061FB4648006840791C
:109D9000401C444909684871424800684079401CA9
:109DA00040490968487163E009F06EFD002811D14F
:109DB000492012F04BFB3B4800684079401C394970
:109DC00009684871374800684079401C354909687E
:109DD000487105E012F0ECFA002032490968487138
:109DE00046E009F051FD002810D112F02FFB2D485C
:109DF00000684079401C2B4909684871294800686F
:109E00004079401C27490968487105E012F0D0FAF2
:109E100000202449096848712AE009F035FD00282E
:109E200018D120480068C07A401C1E490968C872D1
:109E30001C480068C07A1C49097888420ADB002067
:109E400018490968C872174800688079401C15498C
:109E50000968887112F0ACFA00201249096848714B
:109E600006E012F0A5FA00200E490968487100BF0B
:109E700000BF15E000200B4909688871094909688D
:109E80004871062007490968C87009E012F090FA85
:109E9000002004490968487102490968887100BFB7
:109EA00000BF10BDD4070020182F002010B56A484D
:109EB00000684079030016F0CFF9090610C627C6DE
:109EC00044C6608EC60012F049FA634800684079C3
:109ED000401C614909684871BCE0604949695E4AB3
:109EE0001268D27A885C12F0B1FA5B480068407957
:109EF000401C594909684871574800684079401C1E
:109F0000554909684871A5E009F0BEFC002811D147
:109F10007F2012F09BFA504800684079401C4E495F
:109F2000096848714C4800684079401C4A490968F2
:109F3000487105E012F03CFA002047490968487171
:109F400088E009F0A1FC002810D112F07FFA424805
:109F500000684079401C4049096848713E480068E3
:109F60004079401C3C490968487105E012F020FA2C
:109F700000203949096848716CE009F085FC002827
:109F800022D135480068C07A401C33490968C8723C
:109F900031480068C07A3149097888420FDB0020D7
:109FA0002D490968C8722C4800684079401C2A492C
:109FB00009684871002028490968486208E00020C3
:109FC00025490968487103E0002023490968487160
:109FD00012F0EEF93EE020480068407C002816D0E0
:109FE0001E48C068002803D01C48C1681920884753
:109FF00000201949096848621749096848711649DB
:10A0000009688871052014490968C8701AE0124867
:10A010000068406A282807D20F480068406A401C40
:10A020000D49096848620DE000200B490968486243
:10A030000949096848710849096888710520064975
:10A040000968C87006E012F0B3F9002002490968F7
:10A05000487100BF00BF10BDD4070020182F00209A
:10A0600010B50024F7480068807A01287ED1F548B1
:10A070000068C07900287AD0F2480068807900280A
:10A0800004D0012874D0022873D191E1ED48006812
:10A09000007B24286ED2EB480068C07901287AD171
:10A0A000002475E0E7480068C07A24214843E64967
:10A0B00009684018E3490968097B415CE148006888
:10A0C000C07A24225043E14A12688018DD4A12689F
:10A0D000127B805C814229D0DA480068C07A242152
:10A0E0004843DA4909684018D6490968097B415C48
:10A0F000D4480068C07A24225043D34A126880189A
:10A10000D04A1268127B8154CE480068407B2428D4
:10A1100005D3CC480068007BCA4909684873C94820
:10A120000068007BC7490968887308E0C548006873
:10A13000407B242803D20120C24909688871C148A4
:10A140000068007B401CBF4909680873BD4800686F
:10A15000007B242808D3BB480068407B242803D216
:10A160000120B84909688871B64805E0D3E1CDE11E
:10A1700069E0BAE138E00EE00068007B242804D2F0
:10A18000B04800688079012800D103E0601CC4B2A7
:10A19000242C87D356E0002413E0AA480068C07A34
:10A1A00024214843A94909684018015DA548006871
:10A1B000C07A24225043A44A126880180155601CBA
:10A1C000C4B2242CE9D300209E4909684873232097
:10A1D0009C490968887301209A490968887124207C
:10A1E0009849096808732DE00020964909680873AA
:10A1F00094480068C07A401C92490968C872914826
:10A200000068C07A92490978884217DB8D48006857
:10A21000007C012804D102208A490968887106E07F
:10A22000002088490968887186490968C87100203A
:10A2300084490968C8728349096808740020814903
:10A240000968487161E17F4800684079030016F0B1
:10A2500003F8080513A62AA651A68EA6012079495F
:10A260000968087412F07AF8764800684079401C52
:10A2700074490968487199E075494969714A1268D9
:10A28000D27A885C12F0E2F86E4800684079401C8F
:10A290006C49096848716B4800684079401C6949FD
:10A2A0000968487182E009F0EFFA00281BD165497E
:10A2B0000968497B491CC8B212F0C8F861480068B7
:10A2C000407B60490968C8735E4800684079401C5B
:10A2D0005C49096848715B4800684079401C5949ED
:10A2E0000968487105E012F063F8002055490968D3
:10A2F00048715BE009F0C8FA00282BD15149096880
:10A30000C97A24225143504A126889184D4A12686A
:10A31000D27B885C12F09AF84A480068C07B401CE7
:10A3200048490968C87347480068C07B45490968BF
:10A33000897B88421ADD434800684079401C4149C6
:10A34000096848713F4800684079401C3D490968E8
:10A3500048710BE012F02CF83A480068407B39490C
:10A360000968C87300203749096848711EE009F080
:10A370008BFA00280CD133490968887124203149AF
:10A380000968C8732F49096848732E49096888739A
:10A3900012F00EF800202B490968487106E012F00F
:10A3A00007F8002027490968487100BF00BFACE0EA
:10A3B000244800684079030015F04EFF08050F8E11
:10A3C000268E4C8E688E11F0C9FF1E4800684079B9
:10A3D000401C1C490968487185E01D494969194AB2
:10A3E0001268D27A885C12F031F816480068407919
:10A3F000401C144909684871124800684079401CA3
:10A400001049096848716EE009F03EFA002811D140
:10A41000492012F01BF80B4800684079401C09499C
:10A4200009684871074800684079401C0549096877
:10A43000487105E011F0BCFF00200249096848712D
:10A4400051E00000D4070020D0070020CC070020F6
:10A45000182F002009F018FA002810D111F0F6FF8B
:10A460009C4800684079401C9A490968487199489D
:10A4700000684079401C97490968487105E011F06F
:10A4800097FF00209349096848712CE009F0FCF916
:10A4900000281AD18F480068C07A401C8D4909688D
:10A4A000C8728C480068C07A8B49097888420CDBF6
:10A4B000002088490968C8728649096888718549F9
:10A4C0000968487183490968C87111F071FF00205B
:10A4D00080490968487106E011F06AFF00207D4953
:10A4E0000968487100BF00BF0FE011F061FF002054
:10A4F0007849096848717749096888717549096818
:10A50000087374490968C87200BFE2E0002071490D
:10A5100009688872DDE06F480068807A0228F4D10B
:10A520006C480068007A002879D06A480068407951
:10A53000030015F091FE0B0711BB25BB41545EBB18
:10A540007590BB0011F00AFF624800684079401C1A
:10A55000604909684871B7E05F494969087811F0B6
:10A5600075FF5C4800684079401C5A490968487189
:10A57000584800684079401C564909684871A3E072
:10A5800009F082F9002810D111F060FF51480068ED
:10A590004079401C4F49096848714E48006840792D
:10A5A000401C4C490968487105E011F001FF00208A
:10A5B00048490968487187E009F066F9002807D121
:10A5C000444800684079401C42490968487103E0EA
:10A5D000002040490968487111F0EAFE74E011F06A
:10A5E000BDFE3C4800684079401C3A490968487102
:10A5F0006AE0394949690978491CC8B211F026FF57
:10A60000344800684079401C324909684871314833
:10A6100000684079401C2F490968487154E054E0B3
:10A6200009F032F900280FD111F06AFE29490968B2
:10A630008870012011F0DEFE264800684079401C39
:10A6400024490968487105E011F0B2FE0020214953
:10A650000968487138E01F480068807811280CD1DB
:10A6600000201C4909680872AA201A4909688870E4
:10A67000002018490968487011E0164800684078C1
:10A68000401C144909684870124800684078032843
:10A6900005D309F099F900200E490968487011F0B6
:10A6A00087FE00200B49096848710DE011F080FE1B
:10A6B0000020084909684871064909684870AA20BD
:10A6C00004490968887000BF03E000200149096857
:10A6D000887210BDD4070020182F0020F0B5054661
:10A6E0000C4616461F462088482806DA3A46294670
:10A6F000304604F0E5FF012800D0F0BD2088C000FE
:10A700002E502088401C208000BFF6E710B502467E
:10A710009000074BC018405C002802D00320C043C3
:10A7200010BD01209300024C1B1958540020F7E77C
:10A73000982A002070B5002508E06D1C1B48854252
:10A7400002D20AF069FE01E0002503E00AF0B8FD3C
:10A750000028F2D100BF022100200AF0BFFD032132
:10A7600000200AF0BBFD052100200AF0B7FD0721FB
:10A7700000200AF0B3FD002408E00020A1000C4AEC
:10A780005054A10089184880601CC4B2042CF4D332
:10A7900001200849087000204870052088700020BA
:10A7A000C87005480549088070BD000050C300000E
:10A7B000242900200A01002088130000080100203D
:10A7C000F8B58D480078030015F046FD060405161F
:10A7D0003D5EFDFC0EE10AF0F3FD00208649C870E5
:10A7E000487008468078002802D10320087002E0F3
:10A7F000022081490870FDE07F488078002804D05D
:10A800007D488078401E7C4988700AF059FD0028F8
:10A810000BD10AF0D5FD00207749C8700846807832
:10A8200000280FD1032008700CE07348C078401C4A
:10A830007149C8700846C078052803D30520087000
:10A840000AF0EAFDD6E00AF03BFD00280ED1042113
:10A850006A480AF017FD00206749C87048706848C8
:10A86000684908800420644908700CE06248C07898
:10A87000401C6149C8700846C078052803D30520EC
:10A8800008700AF0C9FDB5E05B49497809015E4AE4
:10A89000515C4900594A505A5A490A880121090312
:10A8A000FEF736FE009001255348407800015649D6
:10A8B00040184078002801D100243CE04E48407800
:10A8C0000001514940184078012802D14D480488C0
:10A8D00031E04948407800014B494018407802284F
:10A8E00012D1454949780901474A89180879FEF784
:10A8F00029FE0446404949780901434A89180879E4
:10A90000FEF72CFE054616E03B48407800013E4924
:10A9100040184078032806D0374840780001401896
:10A920004078132806D13448407800013649401851
:10A93000848800E00025002D2FD02F4840780001AA
:10A94000324943182C48407800012F4940180289A9
:10A9500029484078000140182146C7680098B84748
:10A960000646254840780001274BC018C288224877
:10A9700040780001C01881783046FEF73DFD06465C
:10A980001D484078800022494018468001201A491D
:10A99000497889001E4A50540AE000201649497837
:10A9A00089001B4A89184880134949788900505406
:10A9B00011484078401C10494870084640780428E7
:10A9C00009D301E013E007E00AF0FAFC00200A498D
:10A9D0004870032008700DE00AF072FC002803D1D3
:10A9E00001200549087001E00AF016FD02E0FFF7BA
:10A9F000A1FE00BF00BFF8BD0A0100200E0100202B
:10AA000088130000080100202014020060140200D6
:10AA10002429002010B50AF01DFC002405E00020C8
:10AA2000A100074A5054601CC4B2042CF7D3002084
:10AA3000044908700520887003480449088010BD47
:10AA4000242900200A0100208813000008010020AA
:10AA500070B50446002000F0AFF8002000F0DAF8EE
:10AA6000002000F09BF8002000F0C4F8002000F067
:10AA700087F8002000F0AEF800BF012000F08EF84B
:10AA8000012000F0B7F8002521E0002000F086F852
:10AA9000002000F0AFF880202040002806D00120E0
:10AAA00000F08AF8012000F0B5F805E0002000F081
:10AAB00083F8002000F0AEF800BF012000F06EF82F
:10AAC000012000F097F86006040E681CC5B2082D3E
:10AAD000DBDB012000F054F8012000F07BF870BDB2
:10AAE00070B504460D46012000F066F8012000F024
:10AAF00091F8002000F052F8002000F07BF80020D0
:10AB000000F03EF8002000F065F800BF012000F0E2
:10AB100045F8012000F06EF8002628E0002000F043
:10AB20003DF8002000F066F880202040002803D087
:10AB3000012000F041F802E0002000F03DF8802004
:10AB40002840002803D0012000F064F802E0002033
:10AB500000F060F800BF012000F020F8012000F0B4
:10AB600049F86006040E6806050E701CC6B2082E71
:10AB7000D4DB012000F004F8012000F02BF870BDB8
:10AB800010B50446002C04D0812103200AF0D6FC25
:10AB900003E0802103200AF0D1FC10BD10B504466B
:10ABA000002C04D0812104200AF0C8FC03E080219D
:10ABB00004200AF0C3FC10BD10B50446002C04D0DC
:10ABC000812102200AF0BAFC03E0802102200AF071
:10ABD000B5FC10BD10B50446002C04D081210448FA
:10ABE0000AF0ACFC03E0802101480AF0A7FC10BD8C
:10ABF0000107000010B50446002C05D08121072074
:10AC000000020AF09BFC04E08021072000020AF009
:10AC100095FC10BD10B50446002C04D081210448D9
:10AC20000AF08CFC03E0802101480AF087FC10BD8B
:10AC30000207000010B5F920FFF70AFF8820FFF790
:10AC400007FF9020FFF704FF9820FFF701FF08217E
:10AC50000846FFF745FFE820FFF7FAFE12210846F5
:10AC6000FFF73EFFA020FFF7F3FE70210846FFF735
:10AC700037FFA820FFF7ECFE70210846FFF730FFF2
:10AC8000B020FFF7E5FE70210846FFF729FFB82046
:10AC9000FFF7DEFE00210846FFF722FFC020FFF786
:10ACA000D7FE00210846FFF71BFFC820FFF7D0FEA4
:10ACB00000210846FFF714FFD020FFF7C9FE2F211F
:10ACC0000846FFF70DFFD820FFF7C2FE2F210846E8
:10ACD000FFF706FFE020FFF7BBFE2F210846FFF736
:10ACE000FFFE4020FFF7B4FE00210846FFF7F8FE04
:10ACF0000A20FFF7ADFE002405E000210846FFF71B
:10AD0000EFFE601CC4B25A2CF7DB00240AE00020DE
:10AD10000B4908550B4908550B4908550B4908556F
:10AD2000601CC4B25A2CF2DB8120FFF791FE002098
:10AD3000074908708870C8700871487010BD00001D
:10AD40004C260020A6260020002700205A2700209D
:10AD5000D700002010B58020FFF77AFE10BD00005C
:10AD60000020044908700120034908700020487041
:10AD700070470000DC000020D700002010B54848D4
:10AD8000007800287AD046488078030015F064FAED
:10AD90000604434A535A687E414800794149085C99
:10ADA0003F490979404A515C884209D13C480079C1
:10ADB0003E49085C3A4909793D4A515C88421BD0BA
:10ADC000374800793749085C35490979364A505483
:10ADD000334800793549085C31490979344A50547F
:10ADE0002F48C078002803D004202D49887011E036
:10ADF00001202B4988700DE000202949C8700846C1
:10AE00000079401C0871084600795A2802DB0020AE
:10AE10000871087041E04020FFF71AFE0220204927
:10AE200088703AE01E4A11791079FFF759FE032025
:10AE30001B49887031E00A20FFF70AFE04201849F8
:10AE400088702AE0164A1279194B995C144A1279D3
:10AE5000154B985CFFF744FE0520114988701CE0F3
:10AE60000F480079401C0E490871084600795A289D
:10AE700005DB002008710870C87003E00EE00120B7
:10AE80000749C87000200649887006E00020044980
:10AE900008708870C870087100BF00BF10BD000046
:10AEA000D70000204C260020A626002000270020E6
:10AEB0005A27002010B511F087FE012837D107204E
:10AEC00009F0A6FA002810D01C480078052805DAF9
:10AED0001A480078401C1949087016E005201749E7
:10AEE00008700020164908700FE015480078052802
:10AEF00005DA13480078401C1149087005E0052068
:10AF00000F49087000200D4908700C48007805288A
:10AF100006D1FF22A5320021012013F057FB0BE0E0
:10AF20004B22D2000021012013F050FB04E000224C
:10AF30001146012013F04AFB10BD00001D00002047
:10AF40001C00002000200349087248708870486087
:10AF5000704700005C0A002058221152704710B55B
:10AF600004460121022000F071FA0021022000F0C5
:10AF70006DFA10BD014600205322525C10231A4086
:10AF8000002A08D05322525C0C231A409210032A44
:10AF900018D1032016E05422525A0123DB031A4031
:10AFA000002A0ED05322525C0C231A409210032A1E
:10AFB00005D05322525C9207920F032A01D102203E
:10AFC00000E0012070470246002058239B5A0B40A6
:10AFD000002B01D0012000E0002070470146002234
:10AFE0006020405AFF231B0218400005020F100189
:10AFF000014BC018704700000055044010B5002AEE
:10B000000AD056231B5A0C0223435624235256239C
:10B010001B5A8B43235209E056231B5A0C02A343AD
:10B020005624235256231B5A0B43235210BD0000B3
:10B03000F8B504460D46012700263448844203D162
:10B040000121022000F002FA2878401EA07020881A
:10B05000FF210131084320802088400840002080E3
:10B06000A878401EC1B25A20015568790007000C2B
:10B07000E97909020843A97908435C210853288922
:10B0800081B240200153A868C000C10C4220015386
:10B09000A88981B244200153E868C000C10C462051
:10B0A0000153288A81B2482001532869C000C10C8D
:10B0B0004A200153A88A81B24C2001536869C0001C
:10B0C000C10C4E2001535020005B2979090208432E
:10B0D000502108535020005B2979884350210853A0
:10B0E00000E0761C5020005B4007400F2979884221
:10B0F00002D007488642F4D15020005B4007400F41
:10B100002979884200D000273846F8BD0054044011
:10B11000FFFF000030B5034600201C898C4209DD8A
:10B12000082A05D218244C431D682C19A05C02E0A3
:10B13000002000E0002030BD10B5024613898B428C
:10B1400005DD18234B431468E318987C00E00020C9
:10B1500010BD0146FF22C889C007C00F00280AD0D1
:10B160000120C88100E0521EC889C007C00F002816
:10B1700001D0002AF7D1C889C007C00F00280FD11D
:10B180000220C8810420C881487A400840004872E3
:10B19000487A38239843487200204872012070474B
:10B1A0000020FCE70246507A012318435072507A7F
:10B1B0000B78DB0018435072087A012808D1888880
:10B1C00050814868000C0123DB031843908108E09C
:10B1D000087A002805D15081486880001A4B184031
:10B1E0009081487A012804D1507A40231843507244
:10B1F00006E0487A002803D1507A402398435072E1
:10B200000878002811D1C87A1072087B1070487B2A
:10B210005070887B9070CB7BD370087C10714B7C16
:10B220005371887C9071CB7CD371887A002803D0CD
:10B230000120C002D08101E00820D081FF20013030
:10B24000D081012070470000FC1F0000002904D0BD
:10B25000427A80231A43427203E0427A80239A435F
:10B260004272704730B5024600200F4B5024A45A5A
:10B270000D022C435025AC525024A45A8C43AC529E
:10B2800000E05B1E5024A45A6407640F8C4201D076
:10B29000002BF6D15024A45A6407640F002C01D06F
:10B2A000002000E0012030BDFFFF0000827A8023F3
:10B2B0001A40802A00D081727047000070B50446A1
:10B2C00000250023002D02D0012660200653042013
:10B2D000C88188890126F6033040002808D0012063
:10B2E00010728889C004C0084E893043506006E05F
:10B2F0000020107288890F4E304080105060087A0C
:10B30000D072002304E0CE5C10460C30C6545B1CA7
:10B31000D07A9842F7DCC88904263040002804D14E
:10B32000C889F6023040002801D0002070BDD07AD4
:10B33000FCE70000FC1F0000027C80231A40802AEA
:10B3400000D00174704710B50246FF23D089C007B2
:10B35000C00F00280AD00120D08100E05B1ED089F8
:10B36000C007C00F002801D0002BF7D1D089C0073B
:10B37000C00F002801D0002010BD507A01242043C6
:10B380005072507A3824A0435072C87A1072487AAA
:10B3900000280FD1087B1070487B5070887B90701C
:10B3A000CC7BD470087C10714C7C5471887C90717B
:10B3B000CC7CD471FF200130D0814000D081107A44
:10B3C000DAE70000F8B504460D460020002C00D155
:10B3D00000BF002A00D100BF012C01D1412630431B
:10B3E000012A01D112263043022C01D1C02630435C
:10B3F000022A01D130263043134E307076788027F0
:10B40000BE43114F7E70012C08D1FF2100BF0E4EAC
:10B41000B3781E460E4033468B42F8D10A4E7678FA
:10B420004027BE43084F7E70012A0BD100260096AC
:10B4300003E000BF009E761C0096FF276937009E40
:10B44000BE42F6D9F8BD000000040240002905D034
:10B45000054A12780243044B1A7004E0024A12783B
:10B460008243014B1A70704720040240002905D026
:10B47000054A927E0243044B9A7604E0024A927E89
:10B480008243014B9A76704700080240012006492A
:10B49000087000BF04480078802108400028F9D0D7
:10B4A0000120024908707047000C0240A4010020EE
:10B4B00070B5034614460020002B01D1C0B202E053
:10B4C00005468035E8B2012902D1051DE8B206E043
:10B4D000022903D105460835E8B200E0C0B2012CCC
:10B4E00002D1851CE8B200E0C0B2084DA870AD786A
:10B4F00001263543054EB570002201E000BF521C05
:10B500007D252D01AA42F9D970BD0000000C024032
:10B5100070B500242448007920210840002801D07B
:10B52000224D3FE000F046F8054621480078802192
:10B530000840002836D01E4880780840002801D0F6
:10B540001A4D02E000F036F80546194880780007E9
:10B55000840F022C01DBAD0804E0012C01D16D0841
:10B5600000E000BF124880788007C00F002801D09B
:10B570002D0101E00C2045430D4800784007840F61
:10B58000002C02D1601CC4B207E0032C03D1601C64
:10B590004006040E01E06006040E21462846FCF732
:10B5A000CFFD0546284670BD0004024000127A0017
:10B5B000000C024000B5C0229178F82211401C4ACC
:10B5C00012781143EA2923D00ADC0A46E03A130034
:10B5D00014F042FE0A181C20242A2A2A2A161A2AA3
:10B5E000ED291FD004DCEB2916D0EC291CD117E083
:10B5F000F02903D0F82917D10E4817E00E4815E0BE
:10B600000E4813E00E4811E00E480FE00E480DE022
:10B610000E480BE00E4809E00E4807E00E4805E032
:10B620000E4803E00E4801E00D4800BF00BF00BD1A
:10B63000201C02400090D003006CDC020048E801AE
:10B6400000366E010024F400001BB70000127A00DF
:10B65000808D5B0000093D00C0C62D0080841E0067
:10B6600040420F0010B50446204600F097FD002030
:10B6700010BD000010B5A8211348FCF711FE1248B8
:10B68000124908601248486007200881002088722B
:10B6900007220F490D4800F065FA00210B48FFF71B
:10B6A00005FEA0210B48FCF7FBFD0A480A4948604B
:10B6B0000A4B05220A49084800F0E0FB55210648DC
:10B6C000FFF73AFE10BD0000740800205408002067
:10B6D000581002001C0900206008002065B6000018
:10B6E000CC0F02000C4A127812060B4B5B781B043D
:10B6F0001A43094B9B781B021A43074BDB781A430A
:10B70000104642084240D20083085A401146034A7C
:10B710005140034A116070471B07002001020000DE
:10B7200020070020F8B504460F46A07A4006400ED8
:10B73000002874D10025ACE018206843216808185F
:10B74000407C01283CD10121182068432268101850
:10B75000017400260CE0182068432168081808309E
:10B76000815D18206843226810188155701CC6B28C
:10B77000082EF0D3002118206843226810180174A5
:10B780001820684322681018417418206843226802
:10B7900010184161182068432268101881742C2009
:10B7A000684361680818406A002809D018236B4371
:10B7B0002268D0182C236B436268D218516A8847DC
:10B7C00018206843216808184069FF21C94388424E
:10B7D0005DD818206843216808184069C1191820ED
:10B7E00068432268101841611820684321680818CE
:10B7F00041692C206843626810188069814246D3F1
:10B800001820684321680818807C55283FD05521AE
:10B8100018206843226810188174002624E03CE058
:10B820001820684321680818805D2C2169436268EC
:10B8300051181031895D0840182169432268511858
:10B8400088551820684321680818805D2C216943B9
:10B85000626851180831895D0843182169432268DC
:10B8600051188855701CC6B2082ED9D32C206843B5
:10B8700061680818806A002809D018236B43226881
:10B88000D0182C236B436268D218916A8847681CD1
:10B8900085B22089A84200DD4EE7F8BD10B5044608
:10B8A000002015F03DF8022841D1214800780028F9
:10B8B00002D101201E4908701D48007801281FD1BF
:10B8C0001B484078401C1A49487021465A20FCF712
:10B8D00037FC17494978884229D800201449487014
:10B8E00008468078401C8870084680780A2803D370
:10B8F0000020887002200870002015F041F816E042
:10B900000B480078022812D109484078401C0849A9
:10B91000487021467D20C000FCF712FC044949789C
:10B92000884204D800200249487015F029F810BD5B
:10B930007600002000B587B000216846017104211F
:10B9400041710C480290411003910B4904910591FB
:10B950000A480690FFF78EFE01A815F075F800F072
:10B9600043FB00F00FF80021054809F053FE07B033
:10B9700000BD0000FFFF1F00FFFFFF1FEDBB000029
:10B980000205000010B5FF20023072494860002017
:10B9900008720120087000204872012088726E48E9
:10B9A000FFF7D7FB6B496C48FFF7FCFB01216A48A6
:10B9B000FFF74CFC69486749486000200872012085
:10B9C0000870002048720120887263481030FFF729
:10B9D000C0FB604960481030FFF7E4FB01215E487E
:10B9E0001030FFF733FC5D48401E5A494860002084
:10B9F00008720120087000204872012088725648A1
:10BA00005030FFF7A6FB534953485030FFF7CAFBAD
:10BA1000012151485030FFF719FC5048C1384D49B9
:10BA20004860002008720120087000204872012040
:10BA3000887249484030FFF78CFB46494648403001
:10BA4000FFF7B0FB012144484030FFF7FFFBFF2028
:10BA50001230404948600020087201200870002020
:10BA60004872012088723C486030FFF772FB394908
:10BA700039486030FFF796FB012137486030FFF707
:10BA8000E5FBFF2021303349486000200872012087
:10BA9000087000204872012088722F48A030FFF7FC
:10BAA00058FB2C492C48A030FFF77CFB01212A4889
:10BAB000A030FFF7CBFB29488F382649486000208B
:10BAC0000872012008700020487201208872224804
:10BAD000E030FFF73EFB1F491F48E030FFF762FBF5
:10BAE00001211D48E030FFF7B1FB3F20400119491B
:10BAF0004860002008720120087000204872012070
:10BB0000887215482030FFF724FB12491248203074
:10BB1000FFF748FB012110482030FFF797FB104842
:10BB20000C4948600020087201200870002048720B
:10BB30000120887208483030FFF70BFB05490648A2
:10BB40003030FFF72FFB012103483030FFF77EFB39
:10BB500010BD00005C2A00201055044002040000C3
:10BB6000DF070000F0B50B46144643600481002156
:10BB700036E0002216E02C254D4346687519AD5C71
:10BB800018274F430668F619B5542C254D434668CF
:10BB90007519AD5C18274F430668F6190836B55479
:10BBA000551CEAB2082AE6D3002518274F43066839
:10BBB000F619357418274F430668F6197574182757
:10BBC0004F430668F619B57418274F430668F619EF
:10BBD000F57418274F430668F61975614D1CA9B214
:10BBE00005898D42C5DC00258572F0BD70B504461F
:10BBF000606800F04BFE0546E27A23460C33294686
:10BC0000094800F00BFE09496068884203D0491CCE
:10BC10006068884206D1E17AA28890B222460C324E
:10BC200003F08EF870BD000054080020DF0700000C
:10BC3000F8B5054600262C46002C11D000BF03E0C5
:10BC40000020A055701CC6B2082EF9D304F0ACFF3A
:10BC5000C000082108400746206888433843206018
:10BC6000F8BD0000F8B5054600262C46002C49D04A
:10BC700000BF03E00020A055701CC6B2082EF9D307
:10BC80002148007B002809D12088000A000220807A
:10BC90002088FF2109028843208012E005F0AAF8DD
:10BCA00007122088000A00023843208005F0A2F81D
:10BCB0000002FF21090208400746208888433843D4
:10BCC00020801148407B002809D16088000A0002CA
:10BCD00060806088FF2109028843608012E005F0DF
:10BCE0008DF907126088000A00023843608005F071
:10BCF00085F90002FF210902084007466088884351
:10BD000038436080F8BD00003C28002070B505462F
:10BD100000262C46002C2CD000BF03E00020A055AC
:10BD2000701CC6B2082EF9D305F084F901280AD197
:10BD300031202070012060705920A0700820E07030
:10BD40000020207115E005F075F902280AD1312094
:10BD50002070012060705920A0700820E070012040
:10BD6000207106E0002020706070A070E07002205A
:10BD7000207170BDFEB5054600260020019001F03F
:10BD800025FD0A210090FCF7DBF9074604F040FF8F
:10BD90000A210090FCF7EAF980B201902C46002CB1
:10BDA0003AD000BF03E00020A055701CC6B2082E98
:10BDB000F9D3FF21090260688843390C0902FF2288
:10BDC0001202114008436060110260688843390A1A
:10BDD0000904120211400843606060680002000A12
:10BDE0003906090E09060843606005F019F8FF28B6
:10BDF00006DDFF21090420688843401820600BE01D
:10BE000005F00EF80004FF210904084000902068A6
:10BE10008843009908432060FEBDFEB50546002614
:10BE200000200190002704F0C7FC64210090FCF77B
:10BE30009DF980B20190002001F0EAFC87B22C4607
:10BE4000002C1AD000BF03E00020A055701CC6B221
:10BE5000082EF9D3FF210904206888433912090408
:10BE6000FF22120411400843206020680002000AEB
:10BE70003906090E090608432060FEBDFFB581B0F2
:10BE800004460F46002500260020009027600398F6
:10BE900020810498E0600020207400BF9DE01C20F9
:10BEA0006843216808586A01616888501C2068430B
:10BEB0002168081880686A016168891848601C2038
:10BEC00068432168081840686A01616889188860B9
:10BED0001C20684321680818C0686A0161688918D5
:10BEE000C8601C20684321680818007C6A016168EA
:10BEF000891808741C20684321680818407C6A016E
:10BF00006168891848741C20684321680818807C7F
:10BF10006A016168891888831C20684321680818B1
:10BF2000C07C6A0161688918887400206A016168B0
:10BF30008918C8741C2068432168081840680028C4
:10BF400013D01C20684321680818C07C002805D144
:10BF5000401E6A0161688918C8831AE00020C04346
:10BF60006A0161688918C88313E01C20684321684E
:10BF70000818C07C002805D000206A016168891873
:10BF8000C88306E000206A0161688918C88301201F
:10BF90000090002607E000216A01606880181430D4
:10BFA0008155701CC6B2690160684018808BB04230
:10BFB000F1DC1C20684321680818406900280AD079
:10BFC0006B016268D218104614301C236B43226840
:10BFD000D21851698847681CC5B22089A84200DD83
:10BFE0005DE7009805B0F0BD00B58BB068480790DC
:10BFF000002108A801706846017608A84170002059
:10C0000064498872082108A8C170002004E0002259
:10C0100009A90A54411CC8B208A9C9788142F6DCB2
:10C020005D48FFF796F806A95B48FFF7BBF858484C
:10C03000401C0790002108A801706846017608A8F6
:10C040004170002053498872082108A8C17000205F
:10C0500004E0002209A90A54411CC8B208A9C97801
:10C060008142F6DC4C484030FFF773F806A94A4895
:10C070004030FFF797F8452000010790002108A8FD
:10C0800001706846017608A8417000204149887215
:10C09000082108A8C170002004E0002209A90A5460
:10C0A000411CC8B208A9C9788142F6DC3A48503030
:10C0B000FFF74FF806A938485030FFF773F8112002
:10C0C00040010790002108A801706846017608A881
:10C0D000417000202F498872082108A8C1700020F3
:10C0E00004E0002209A90A54411CC8B208A9C97871
:10C0F0008142F6DC28482030FFF72BF806A92648B5
:10C100002030FFF74FF80B20C0010790002108A84E
:10C1100001706846017608A8417000201D498872A8
:10C12000082108A8C170002004E0002209A90A54CF
:10C13000411CC8B208A9C9788142F6DC16486030B3
:10C14000FFF707F806A914486030FFF72BF8FD2029
:10C15000C000029000216846017301714173817330
:10C160000821C173002004E0002204A90A54411CE4
:10C17000C8B26946C97B8142F6DC07481030FEF739
:10C18000E8FF01A904481030FFF70CF80BB000BD20
:10C19000EE0600005C2A00208055044030B585B0D2
:10C1A0000446002520680190A1796846C172617932
:10C1B000417200210172017000BF05E02046083085
:10C1C000415D03A841556D1C6846C07AA842F5D868
:10C1D0000B22D2010199881A914226D007DC184817
:10C1E000081A1CD023210901401A24D111E0FF387C
:10C1F0006F38002802D001281DD104E0694611489B
:10C20000FFF7A1F818E069460E484030FFF79BF8A9
:10C2100012E069460B485030FFF795F80CE069468C
:10C2200008482030FFF78FF806E06946054860307F
:10C23000FFF789F800E000BF00BF05B030BD000087
:10C240002002000080550440F0B585B004460F463A
:10C2500000250026207C4006400E55287ED100BFD8
:10C2600076E1690160684018807C002877D1690117
:10C270006068401840686A01616889188968884266
:10C2800009D26901606840184068C0196A01616894
:10C29000891848605AE1690160684018C068AF4970
:10C2A000884208D8690160684018C068401C6A016B
:10C2B00061688918C860690160684018C07C0028FE
:10C2C00021D1002607E000216A016068801814303F
:10C2D0008155701CC6B2690160684018808BB042FD
:10C2E000F1DC1C20684321680818406900280AD046
:10C2F0006B016268D218104614301C236B4322680D
:10C30000D2185169884769016068405800906901F6
:10C3100060684018017C6846017100214171690123
:10C3200060684018017F6846817169016068401843
:10C33000417C6846C171002608E0690160684018C8
:10C340001430815D02A88155701CC6B26901606815
:10C350004018808BB042F0DCE06801E0FCE01DE0BA
:10C36000002806D06846E16888476A016168891834
:10C37000C874690160684018C07C002804D16A0153
:10C38000616889184860E1E06901606840184068A8
:10C39000C01B6A01616889184860D7E0690160685C
:10C3A000401880680028EED0690160684018C08B92
:10C3B0000028E8D0690160684018C08B6A01616894
:10C3C0008918C968884207D1690160684018C08B24
:10C3D0006249C94388427DD169016068401840685C
:10C3E0006A01616889188968884209D269016068B0
:10C3F00040184068C0196A01616889184860A5E062
:10C4000000206A0161688918486069016068401805
:10C41000C0685249884208D8690160684018C068FD
:10C42000401C6A0161688918C860002607E0002185
:10C430006A016068801814308155701CC6B26901A9
:10C4400060684018808BB042F1DC1C206843216892
:10C450000818406900280AD06B016268D21810469B
:10C4600014301C236B432268D21851698847690134
:10C47000606840580090690160684018017C684617
:10C48000017100214171690160684018017F6846AF
:10C490008171690160684018417C6846C17100265D
:10C4A00008E06901606840181430815D02A8815578
:10C4B000701CC6B2690160684018808BB042F0DC25
:10C4C000E068002808D06846E16888476A0161682A
:10C4D000891800E015E0C874690160684018C07CE4
:10C4E000002804D16A016168891848602EE069015A
:10C4F000606840184068C01B6A016168891848601C
:10C5000024E01C20684321680818406800280FD0E8
:10C510000020C0436A0161688918C8831C206843F1
:10C520002168081840686A0161688918886008E015
:10C5300000206A0161688918C8836A0161688918E6
:10C54000886000206A0161688918C860681CC5B2EB
:10C550002089A84200DD84E605B0F0BD0000FFFFA1
:10C560007CB500BF19212C480078FBF7E9FD044693
:10C570002A4860432A4A8118002201200DF09AF8C7
:10C5800020460A2250436430001981B20022012063
:10C590000FF0DCF801200A2262431219D1B20A22FC
:10C5A000624312190090D0B201231A4609F046FBEB
:10C5B000BA220721002006F0FFFF01200090019021
:10C5C0000B20604382B20B20604381B20023012024
:10C5D0000EF0EEFD6F20604381B201200FF05CFB96
:10C5E000104860430246032101200BF0E1FD0025C5
:10C5F00005E0012128460BF015FD681CC5B20F2D82
:10C60000F7DB21460B2251436431C8B20FF0A8FD7D
:10C610000FF090FD7CBD000073000020672B000030
:10C62000A0860100FCB10100002005490870054901
:10C630000870054908700549087005490870704779
:10C64000740000207500002073000020720000209C
:10C6500071000020F0B589B000BF00BF00BF00BF6F
:10C6600000BF00BF00BF00BF00BF00BF5D48007833
:10C670003C2805DA5B480078401C5A49087002E003
:10C680003C2058490870574800781D2805DC56485A
:10C690000078401C544908700BE05348007800288B
:10C6A00002D15149087004E04F480078401E4E49BD
:10C6B000087003214C480078FBF758FD4B4948436C
:10C6C0000390052148480078FBF73AFD0446032112
:10C6D00045480078FBF74AFD0B214843643080B29F
:10C6E0000690414909788A0088180621FBF73EFD2B
:10C6F000FF21F531484380B2079003213A48007882
:10C70000FBF734FD0B214843643080B208900321CD
:10C7100035480078FBF72AFD35494843354940182C
:10C720000490032130480078FBF720FD0B210646DA
:10C730004E4303212C480078FBF718FD0B210746D8
:10C740004F43032128480078FBF710FD6F21484331
:10C7500080B2059003210120039A0BF029FDE1B27C
:10C7600001200BF0EDFAE1B201231846069A09F018
:10C770003FFDFF21F5310798FBF7F8FCC0B20146F9
:10C78000029001200AF018FA0022012008990EF008
:10C79000DDFF0022012004990CF08CFF0120059997
:10C7A0000FF07AFA0120F9B20090F0B201231A4694
:10C7B000029009F043FABA220721002006F0FCFE9D
:10C7C000032109480078FBF7D1FC0B21484385B2CF
:10C7D0000120009000232A46294601900EF0E8FC33
:10C7E00009B0F0BD7500002074000020FCB101000C
:10C7F000672B0000A0860100002000BF06E000219A
:10C80000044A1154044A1154411CC8B25A28F6DB98
:10C81000704700004C26002000270020FFB581B0A3
:10C8200004460F463D462089A8422DDD1820684366
:10C8300021680818007C002826D1002609E0049809
:10C84000815D182068432268101808308155701CDB
:10C85000C6B2082EF3D301211820684322681018AD
:10C8600041742C20684361680818006A00280BD0C6
:10C8700018236B432268D218104608302C236B43D0
:10C880006268D218116A884705B0F0BD01460720DA
:10C89000124BCA1A994211D008DCCA1FFA3A002A70
:10C8A00014D0102A0CD01F2A14D10DE0322A0FD038
:10C8B000C02A07D0C12A0DD100200DE001200BE0D5
:10C8C000022009E0032007E0042005E0052003E042
:10C8D000062001E0072000BF00BF704741030000B1
:10C8E00010B504467D21C90061430846322103F09A
:10C8F00005FF10BDFF200B4908700020C0430A4906
:10C9000008800A490880FF20094908700949087011
:10C910000949087000200949086009490860094967
:10C9200008607047580000205A0000205C0000207A
:10C930005E0000205F000020600000204C0000200E
:10C94000500000205400002001480068704700009B
:10C950005000002001480068704700004C00002093
:10C9600010B5054909886522514308466421FBF743
:10C97000FDFB80B210BD00005A0000200148007885
:10C98000704700005F0000200148007870470000F9
:10C990005800002010B510F017F901282CD100F034
:10C9A00063F8012000F066F803F00CFF044600F085
:10C9B00043F804F00BF9044600F04AF804F05CFB7D
:10C9C000012805D100F03EF8012000F047F805E00D
:10C9D000002000F037F8002000F040F80020134954
:10C9E000086013480068134988421ED21048006846
:10C9F000801C0F49086018E000200D4908600B48B2
:10CA000000680C49884204D208480068801C074925
:10CA10000860002000F028F8012000F02BF800202A
:10CA200000F00AF8002000F013F810BD50000020BC
:10CA30004C000020FFFFFF7F014908807047000085
:10CA40005A00002001490870704700005F00002074
:10CA500001490880704700005C000020014908700F
:10CA60007047000060000020014908707047000016
:10CA70005800002001490870704700005E00002047
:10CA80000021014A117170470060004000220149F5
:10CA90004A75704700600040002201494A7670479D
:10CAA000006000400021014A1172704700600040A0
:10CAB0000021014A11737047006000400021014AC3
:10CAC00011747047006000400021014A11757047E1
:10CAD000006000400021014A11767047006000406C
:10CAE000002201494A73704700600040002201495A
:10CAF0004A7470470060004010B51C4C1C49206807
:10CB000088421ED106221B49201DFBF7D4FB0028BA
:10CB100017D11122184920460A30FBF7CCFB002818
:10CB20000FD10622154920461B30FBF7C4FB002815
:10CB300007D10622124920462130FBF7BCFB002812
:10CB40000DD000F089FE0A480E490860074814F02D
:10CB500048F80C4A2821054814F06EF804E0282211
:10CB600021460848FBF783FB10BD0000000250007F
:10CB70007AA7A55A31070020370700202B0700208D
:10CB800025070020682E0020002008490870084969
:10CB900008700120074908700020074908700748FD
:10CBA00007490860002007490870704713070020F4
:10CBB00012070020150700201A0700202506000094
:10CBC000480700202407002070B5044600BF9120CC
:10CBD000604305460A212846FBF7B2FA0546284677
:10CBE00070BD000070B5A8B0054600240026A02145
:10CBF0006846FBF755FB00F09FFC1E490A681421AC
:10CC00006943505000211B480268142068431018E3
:10CC10004160184802681420684310188160154864
:10CC20004068002824D000BF17E06006060E282EBA
:10CC300000D316E00F480168142060430858B10083
:10CC40006A4650500B480168142060430818416838
:10CC5000701C80001150601CC4B20648007AA042CB
:10CC6000E3DC00BF6200034869464368022098473E
:10CC700028B070BDE02E002030B5A9B000240025FA
:10CC8000A02101A8FBF70CFB00BF25E06006050E04
:10CC900000F052FC1F490A681421614350500021E2
:10CCA0001C4802681420604310184160194802684B
:10CCB0001420604310188160282D0BD2154801689C
:10CCC000142060430858A90001AA50500021681C94
:10CCD00080001150601CC4B20E48007AA042D5DC1E
:10CCE0000C484068002813D00A48007A40002828E1
:10CCF00006D30848282201A943680220984707E084
:10CD00000448007A4200034801A94368022098477A
:10CD100029B030BDE02E002010B50FF055FF0128DE
:10CD20007ED1FFF717FE5549884216D20F2054498D
:10CD30004871887108468078002801D10520487024
:10CD40004F488078052802D100204D4948700020C6
:10CD50004B4908724872087035E0FA20484948711A
:10CD600088714849088803F055FE464880780028B5
:10CD70000CD14349087008464079C870084680794C
:10CD8000087100208870487048721CE001203C49FE
:10CD900008700846407A022805D101204872002018
:10CDA000C87008710FE03648407A00280BD1022085
:10CDB0003349487208464078887008464079C87000
:10CDC0000846807908712E4880782D494978884234
:10CDD00013DD00202A49C87008460079401C0871FC
:10CDE000084600798979884222DB002024490871AD
:10CDF00008468078401E88701AE0214880782049D3
:10CE00004978884214DA00201D4908710846C07824
:10CE1000401CC8700846C0784979884208DB00E0A9
:10CE20001EE000201649C87008468078401C8870B3
:10CE300014488078002803D10120114908721BE0B2
:10CE400010480088732803DB02200D49087213E0A4
:10CE50000C48008870280FDC0020094908720BE09C
:10CE600000200749087008464079C8700846807954
:10CE7000087100200872487210BD0000B80B000055
:10CE8000BC0900207C000020002004498870487004
:10CE9000C87008710872487270470000BC09002011
:10CEA0000020064908808870054988704870FA207B
:10CEB000C870087100200872487270477C0000201A
:10CEC000BC09002070B503F0ADFC044603F0BCFCC7
:10CED00005460FF079FE01282ED105211A48FEF7EC
:10CEE0002BF9552804D1002018498870088027E0C4
:10CEF000012D04D1002015498870088020E0012010
:10CF0000124988701248844202DB201A84B200E081
:10CF100000240A212046FBF729F9052901DB601DC1
:10CF200084B20C48844200DD04460A212046FBF707
:10CF30001DF90649088003E0002004498870088034
:10CF4000FFF7EAFE70BD0000540800207C000020BE
:10CF5000AA0A0000C60700001CB50020009001903E
:10CF600000F0EAFA0B49086000200B4909680860E4
:10CF70000A48006800280CD00749096808680A2197
:10CF8000FBF7DEF80090012269460520034B1B6881
:10CF900098471CBDE4070020D8070020E0070020C8
:10CFA0000020084948800849088008490880084945
:10CFB0000870084988720849088048800120087173
:10CFC00070470000300000202000002022000020D8
:10CFD000240000203808002028000020F8B503F0C5
:10CFE00003FC074603F012FC0090FFF7CDFC01287C
:10CFF00060D10521C548FEF79FF8552802D000985A
:10D00000012807D10020C2490870C2490880C249DE
:10D01000887256E0BE480078002810D10120BC4933
:10D0200008703D462846E917890F091889030D0C39
:10D03000BA48854200DD0546B648058041E0B6485D
:10D04000807A4000B4490F520846867A0EE070009C
:10D05000B1490D5A701E4000085A7100AE4A505234
:10D06000701E400011460D52701EC6B2002E08DD23
:10D070007000A949095A701E4000A74A105A8142FF
:10D08000E5DBA548807A401CA34988720846807A6F
:10D09000052816DB002088720846C5882846E9174F
:10D0A000890F09188D109D48854200DD0546994875
:10D0B000058006E000209649087096490880964948
:10D0C00088729448058896480088A84257DA9448A0
:10D0D0000088281A84B292480079012827D1904804
:10D0E0004088A0420BDA8E4840880A308C4948803C
:10D0F00008464088A04204DD0846448001E0884894
:10D1000044808748448803212046FBF72FF884B2E7
:10D11000192C00DA192482480088001980490880F7
:10D1200008460088A84201DD08460580CDE07C481D
:10D130004088142805DD7A484088143878494880AA
:10D1400002E0002076494880754844880321204643
:10D15000FBF70CF884B2192C03DA0120704908712E
:10D16000B3E06F480088A04205DD6D480088001BD1
:10D170006B490880A9E0002069490880A5E068485B
:10D180000088A84259DD66480088401B84B2644884
:10D190000079012827D162484088142805DD6048BD
:10D1A000408814385E49488002E000205C4948808D
:10D1B0005B48448803212046FAF7D8FF84B2192C33
:10D1C00003DA0220564908717FE0554800880019AB
:10D1D00053490880084600885049884275DD084652
:10D1E0004F49088071E04E484088A0420BDA4C4815
:10D1F00040880A304A49488008464088A04204DDF9
:10D200000846448001E0464844804548448803215C
:10D210002046FAF7ABFF84B2192C00DA19244048F3
:10D2200000882919884202DA3D4805804DE03C48D3
:10D230000088001B3A49088047E0394844880321A8
:10D240002046FAF793FF84B2192C3EDD344840881B
:10D25000142805DD3248408814383149488002E0FE
:10D2600000202F4948802E48448803212046FAF7A1
:10D270007DFF84B22A480079012813D1192C03DAE2
:10D2800002202749087120E0254800880019244918
:10D290000880084600882149884216DD0846204952
:10D2A000088012E0192C03DA01201D4908710CE0F6
:10D2B0001B480088A04205DD19480088001B18495A
:10D2C000088002E00020164908801648008850288F
:10D2D00004DC134800881349088016E010480088D1
:10D2E00010490988884204DD0D4800880D490880EE
:10D2F0000BE00B4800880B490988081A84B2502CAF
:10D3000003DB0748008807490880F8BD540800205F
:10D31000240000202000002038080020E02E00001B
:10D32000280000202200002010B504466420444359
:10D33000A1212046FAF704FF0446204610BD000054
:10D340007CB5002400200190009000F03FFA0546D3
:10D350000A21FAF7F5FE044601226946042000F08E
:10D36000DDFE0098401C002814D17D20C00020184C
:10D3700011490860084600680190012201A90320B4
:10D3800000F018FF0120009001226946042000F0FF
:10D3900011FF0FE0009801280CD17D20000120181A
:10D3A00005490860084600680190012201A9032090
:10D3B00000F000FF7CBD00002C01002010B5012012
:10D3C0000F49087000200F49096808600D49096875
:10D3D00048600C490968886000F07EF9FFF7BCFDE1
:10D3E000FFF74AFC08480068002807D001220548DA
:10D3F000016808310020044B1B68984710BD0000ED
:10D40000B1070020AC070020A807002010B518487D
:10D4100000681849884229D117480068002804D0BC
:10D4200015480068804715490870154800680028AD
:10D4300004D01348006880471249087012480068F9
:10D44000002804D010480068804710490880104820
:10D450000068002805D00E48006880470D49088004
:10D4600002E00D480B49088000F078F810BD00007C
:10D47000BC0700207856341298070020B00700201F
:10D480009C070020B2070020A0070020B40700205E
:10D49000A4070020B60700201027000010B50023C5
:10D4A000174C2360174C2370174C2370174C2370B4
:10D4B000174C2380174C2380174C2370174C13688C
:10D4C0002360174C53682360164C93682360164CF6
:10D4D000D3682360154C1369236000280CD0144BCB
:10D4E0001860134C0B682468A3600023104C246858
:10D4F00023600F4C246863600E4B014C236010BD09
:10D50000BC070020B8070020B0070020B2070020A9
:10D51000B4070020B6070020B107002098070020BC
:10D520009C070020A0070020A4070020A8070020D7
:10D53000AC07002078563412054800680549884237
:10D5400003D105480068806870470020C043FBE7AE
:10D55000BC07002078563412AC07002070B50024B8
:10D56000002500263048007801285CD12F4800783B
:10D57000002858D12E480078012854D12D4805881C
:10D580002D490988694308462C49FAF7D9FD85B227
:10D59000E1200001854207D8192169430846092185
:10D5A000FAF7CEFD044600E0244C254800680068E8
:10D5B000001923490968086021480068006820496B
:10D5C00009684968884207D31D48006800681C49FB
:10D5D00009684968461A0AE019480068406800214D
:10D5E000C943081A1649096809684018461C1548B5
:10D5F000864218D3344601462046FAF7A1FD044678
:10D600000F48006841680F48604308180C490968D2
:10D61000486001200C4908700948006880680019BA
:10D6200007490968886070BDB0070020B107002075
:10D63000B2070020B4070020B60700201027000022
:10D64000AC070020A0860100B807002000220C4B88
:10D650001A600C4B0A681A600B4B4A681A600B4B35
:10D660008A681A600A4BCA681A600A4B0A691A600B
:10D67000002801D0084A1060084A014B1A60704720
:10D68000BC070020980700209C070020A00700206E
:10D69000A4070020A8070020AC0700207856341209
:10D6A00010B50A48006800280ED009480078012803
:10D6B0000AD1002006490870012206480168083195
:10D6C0000020024B1B68984710BD0000A8070020EF
:10D6D000B8070020AC0700201CB500200090019086
:10D6E0000024FFF729FF04460E480068046000206C
:10D6F0000C49096848600B49096888600A48006855
:10D7000000280DD0074800680068009005480068B0
:10D7100040680190022269460120034B1B6898472C
:10D720001CBD0000C0070020C4070020F8B5054656
:10D730000C4616460027002D17D00E480560FFF74F
:10D74000FBFE07462068B84203D90A480068076014
:10D7500003E00849206809680860064960680968AC
:10D7600048600449A0680968C8600348066000F082
:10D7700005F8F8BDC0070020C407002070B50024DC
:10D780000025FFF7D9FE04460F4800680068A04254
:10D7900000D903E00C4800680068251A0A480068B0
:10D7A000406840190849096888600748006880682F
:10D7B00005490968C968884205D903480068C068F6
:10D7C00001490968886070BDC007002001480068F1
:10D7D00080687047C0070020002801D0024A10600E
:10D7E000024A116070470000C0070020C4070020F3
:10D7F0000549002005E00A1D135C044A1354421C2D
:10D80000D0B22028F7DB704700065000942E00208D
:10D8100001461048026814204843101882680D48D9
:10D820000368142048431818C06882420BD909487D
:10D830000268142048431018C26806480368142080
:10D84000484318188260034802681420484310189F
:10D8500080687047E02E00200021002005E01A4A71
:10D86000135C1A4A1354421CD0B20628F7DB11216C
:10D87000002006E0164A135C144A921D1354421C01
:10D88000D0B28842F6DB002006E0124A135C0F4A51
:10D8900017321354421CD0B20628F6DB002006E0F3
:10D8A0000D4A135C094A1D321354421CD0B206289B
:10D8B000F6DB002005E00023044A23321354421C07
:10D8C000D0B20128F7DB7047310700206C2E002012
:10D8D000370700202B0700202507002038B5044615
:10D8E00000200090009401226946052000F062FCAF
:10D8F00038BD000008B500200090012269460620CE
:10D9000000F00CFC684600780C49087368464078C3
:10D9100048730846007B0A4948730848407B88736F
:10D920000648807BC8730548C07B087400200873D4
:10D930000448054908600549086008BD3C280020E6
:10D94000C80900207117000080000020840000201A
:10D9500008B50020009001226946062000F0DEFB99
:10D96000684600781149087368464078487300207B
:10D970000F490860486008724872887203F01AF90B
:10D980000B49C8720948007B48730848407B88737C
:10D990000648807BC8730548C07B08740020087364
:10D9A0000448054908600549086008BD3C28002076
:10D9B000C8090020711700008000002084000020AA
:10D9C00038B500240025002000900121FE48FDF715
:10D9D000B3FB55280AD002F07BFFFC49487302F0E4
:10D9E0008BFFFA4988730120087308E0F848007B30
:10D9F000F6494873F648407B887300200873F34863
:10DA0000407B002833D1F3480068F349884208D8A6
:10DA1000F0480068401CEF4908600020EB4948735B
:10DA200082E0EA48407C012802D10020E9490860F0
:10DA30000020E6494874E648007B022812D0E448FA
:10DA4000007B03280ED00121DF48FDF775FB552828
:10DA500003D00320DD49487366E0DD48007BDB49E5
:10DA6000487361E0DA48007BD84948735CE0D748E6
:10DA7000407B012832D1D548407C002801D1D549CE
:10DA800008600120D1494874D2480068D2498842D0
:10DA900008D8D0480068401CCE4908600120CB4916
:10DAA000487341E0CA48007B022812D0C848007B76
:10DAB00003280ED00121C448FDF73EFB552803D0B2
:10DAC0000320C24948732FE0C148007BBF49487317
:10DAD0002AE0BF48007BBD49487325E0BB48407B36
:10DAE00002280FD10020BB49086002F01BFF00286C
:10DAF0001AD002F017FF401C002815D00220B349AD
:10DB0000487311E0B148407B032806D10020B14999
:10DB100008600320AD49487306E00020AD49086065
:10DB2000AB48007BA9494873A848807B002833D1C3
:10DB3000AA480068A849884208D8A8480068401C3C
:10DB4000A64908600020A149887382E09F48807C34
:10DB5000012802D10020A149086000209B49887457
:10DB60009B48407B022812D09948407B03280ED066
:10DB700001219548FDF7E0FA552803D00320934989
:10DB8000887366E09248407B9049887361E09048D2
:10DB9000407B8E4988735CE08C48807B012832D1C1
:10DBA0008E4800688C49884208D88C480068401C20
:10DBB0008A4908600120854988734AE08348807C4F
:10DBC000002801D185490860012080498874804877
:10DBD000407B022812D07E48407B03280ED00121D2
:10DBE0007948FDF7A9FA552803D0032077498873AF
:10DBF0002FE07748407B754988732AE07448407B62
:10DC00007249887325E07148807B02280FD100207B
:10DC10007249086002F0A4FE00281AD002F0A0FEAB
:10DC2000401C002815D002206849887311E067481D
:10DC3000807B032806D100206849086003206349DF
:10DC4000887306E00020654908606148007B5F49F1
:10DC500088735E48407B5E49097B884205D15B48FA
:10DC6000807B5B49497B884246D05848407B584975
:10DC7000097B884202D001205449C8735348807BF5
:10DC80005349497B884202D00120504908744F48CB
:10DC9000407B022803D04D48407B032803D14B48EA
:10DCA000407B4B4908734948807B022803D0474892
:10DCB000807B032803D14548807B4549487343480E
:10DCC000407B02280BD04148407B032807D03F48C7
:10DCD000807B022803D03D48807B03280CD13C4840
:10DCE000017B684601703A48417B684641700122D9
:10DCF0006946062000F05EFA02F05CFF3349C87204
:10DD000002F0F0FD044602F003FE0546FEF73CFE7D
:10DD100001286DD101212C48FDF70EFA552807D1B5
:10DD200000202A4908724872086048608872CBE077
:10DD3000FF2C01D0FF2D72D1FF2C2ED1FF2D2CD026
:10DD400000202249087201204872254808602548B1
:10DD50006843486048686621FAF7F2F91B49486051
:10DD6000084640682049884202D908461749486059
:10DD70001648406832301D49884206D3134840682F
:10DD800032301849FA39884203D901200F49887284
:10DD90009AE000200D49887296E0FF2C44D0FF2DB8
:10DDA00042D1012009490872002048720C4848609D
:10DDB0000C486043086008686621FAF7C1F9034916
:10DDC00008600846006814E054080020C8090020D4
:10DDD0003C280020800000207017000084000020F4
:10DDE000DE030000BE0A0000AC260000A40600000E
:10DDF000A5E05749884202D9084656490860554867
:10DE0000006832305449884205D3524800683230A5
:10DE10005249884204D901204E49887254E00CE0EE
:10DE200000204C4988724FE049484A4908604860E0
:10DE3000002088720872487246E001204549087245
:10DE4000487247486043086008686621FAF778F925
:10DE500040490860084600683D49884202D90846A2
:10DE60003C4908603E4868433A4948604868662132
:10DE7000FAF766F9374948600846406834498842ED
:10DE800002D9084633494860324800683230324986
:10DE9000884212D32F4800683230304988420CD86B
:10DEA0002C48406832302C49884206D329484068C3
:10DEB00032302A49C831884203D901202549887265
:10DEC00002E00020234988722248407B002802D1CA
:10DED0002049C87315E01F48407B012802D11D4925
:10DEE000C8730EE01B48407B022802D11949C87351
:10DEF00007E01848407B032803D11649C87314482B
:10DF000008601448807B002802D1124908741DE083
:10DF10001048807B012802D10E49087416E00D4894
:10DF2000807B022802D10B4908740FE00948807BEE
:10DF300003280BD1074908740548486006E0002013
:10DF400004490872487208604860887238BD000051
:10DF5000AC260000C8090020A4060000FC08000050
:10DF6000BE0A0000FFB583B006460D4617460024E2
:10DF70000020029000BF1420784380190190002EE9
:10DF800057D00198002854D02B4806602A4906989B
:10DF900048600846077200BF45E0FFF7CDFA0290DF
:10DFA000200129580298814204D820012858401C99
:10DFB000002806D1204902980A6814216143505074
:10DFC00006E0200129581C480268142060431150C3
:10DFD000200140194068401C002807D10021164844
:10DFE0000268142060431018416008E020014019C5
:10DFF00041681148026814206043101841602001F4
:10E00000401981680C480268142060431018C160F0
:10E0100020014019017B0848026814206043101851
:10E020000161601CC4B20448007AA042B5DC00F073
:10E0300005F807B0F0BD0000E02E002070B5002408
:10E0400000250026FFF778FA054600BF4EE02A4873
:10E050000168142060430858A84239D8264801684E
:10E060001420604308582E1A234801681420604386
:10E07000081840688119204802681420604310186D
:10E0800081601D48016814206043081881681A489F
:10E090000268142060431018C068814224D91648D1
:10E0A00001681420604308180069002803D0204646
:10E0B000FEF798FD18E01048016814206043081826
:10E0C000C1680D48026814206043101881600BE09D
:10E0D00009480168142060430818406806490A6826
:10E0E0001421614351188860601CC4B20248007A50
:10E0F000A042ACDC70BD0000E02E002010B500BFD7
:10E1000014244C432318002805D0002B03D0024CC4
:10E1100020606260217210BDE02E0020F8B5054637
:10E120000E4614462B0012F097F80705131A212803
:10E130002F363D001D48FAF711FD1D4908701B4898
:10E14000FAF7C6F807466421F9F7FAFF30602AE0CB
:10E15000A004020C31461620FAF7FAFD23E0A004D1
:10E16000020C31464820FAF7F3FD1CE0A004020C33
:10E1700031468020FAF7ECFD15E0A004020C314690
:10E18000A020FAF7E5FD0EE0A004020C3146B02015
:10E19000FAF7DEFD07E06004020C3146C020FAF712
:10E1A000D7FD00E000BF00BF0020F8BD2E280020F2
:10E1B000E100002070B505460E4614462B0012F013
:10E1C0004BF807051D242B32393F460030680028E4
:10E1D00002D1FAF761FB10E064223168514308462E
:10E1E0001C49FAF77FF800201B49087001226421BE
:10E1F0001848FAF71BFE1849087029E0A004020C21
:10E2000031461620FAF762FF22E0A004020C3146E4
:10E210004820FAF75BFF1BE0A004020C3146802087
:10E22000FAF754FF14E0A004020C3146A020FAF7DC
:10E230004DFF0DE0A2B23146B020FAF747FF07E0EC
:10E240006004020C3146C020FAF740FF00E000BF36
:10E2500000BF70BD20280020E000002000B5AFB056
:10E2600050211BA8FAF71CF800201A90142115A8B9
:10E27000FAF716F800201290139014901190402194
:10E2800001A8FAF70DF8002000905149086001221A
:10E290001BA9FFF743FF1B98401C002801D11A90CF
:10E2A00001E01B981A904B4815904B4816904B482C
:10E2B0001790002018904A48199015AA1AA94948A1
:10E2C000FFF7ECF802221CA90120FFF727FF1C989A
:10E2D000401C002801D1129001E01C9812901C985B
:10E2E000401C002801D1139001E01D9813903E4876
:10E2F000149012A93D48199AFFF718FA08221EA98E
:10E300000220FFF70BFF1E98401C002801D101904E
:10E3100001E01E9801901F9802903548039001205B
:10E3200069460874801E059032490791012101A8B1
:10E330000177881E09902F490B91012109A80173CB
:10E34000881E0D902B490F9101210DA80173042205
:10E3500001A92948199BFFF705FE01221BA90320EB
:10E36000FFF7DCFE25491B9808601B98401C00281D
:10E3700006D1FF20F530086001220320FFF71AFFC5
:10E3800001221BA90520FFF7C9FE1B98401C00288D
:10E3900007D101201A498860012208310520FFF7C2
:10E3A00009FF01221BA90620FFF7B8FE1B98401C9D
:10E3B000002808D100216846017041700122694699
:10E3C0000620FFF7F7FE0F48014908602FB000BD97
:10E3D000E400002089C900007DC9000061C9000077
:10E3E000B5E10000B427002076841E00C02700207D
:10E3F0000F2700009F860100D02700202C0100205D
:10E400003C280020A33AA55A00B585B014216846DF
:10E41000F9F746FF00200F4908600F4800900F48A9
:10E4200001900F480290002003900E480490694626
:10E430000D48FFF70BF90D480499FFF7CDF90421BA
:10E440000B48049AFFF75AFE0A480249086005B0D3
:10E4500000BD0000E400002089C900007DC9000063
:10E4600061C90000B5E10000B4270020C0270020EA
:10E47000D0270020A33AA55A00200C4908800C4957
:10E4800008800C49088001200B49087000200B49C6
:10E4900008730B4908804880012008710020074953
:10E4A0004880088007490860704700003800002055
:10E4B0003A000020400000204200002044080020D4
:10E4C000440000203C000020F8B502F0C7F90646E1
:10E4D00002F0CEF90746FEF757FA012865D105216B
:10E4E000AB48FCF729FE552807D10020A949087040
:10E4F000A9490880A94988805FE0012F07D1002041
:10E50000A4490870A4490880A449888055E0A1481E
:10E510000078002808D101209E49087035460A205D
:10E5200068439D49088048E09C48007B42009B4826
:10E53000801D8652801F047B11E061009748801D7A
:10E54000455A601E41009548801D415A6200815223
:10E55000601E41009148801D4552601EC4B2002CCF
:10E560000ADD61008D48801D415A601E42008B48C3
:10E57000801D805A8142E0DB8848007B401C87492F
:10E5800008730846007B032807DB00200873084651
:10E5900005890A206843804908807F4800887F49B0
:10E5A000888001207B49087007E0002079490870C5
:10E5B00079490880794908738880774800887849C4
:10E5C000086074480078002815D0084600686C215F
:10E5D000484373490860642171480068F9F7B0FD49
:10E5E0006F490860084600686E49884206D90846A7
:10E5F0006B49086002E000206949086068480068CB
:10E6000069490988884203D2654800680F2804D206
:10E6100063480088644908800AE0634800886049CC
:10E620000968401A0F2803D35D4800885E490880B6
:10E630005A480088401C59490880084600880A2822
:10E640002CDB0020088059480088574909888842F7
:10E6500003DA01205649087108E0544800885249FD
:10E660000988884202DD022051490871504800792A
:10E67000012840D14C4800884C49098888420DDB6C
:10E680004948018849480088FF309130814206DDC1
:10E6900046480088FF3073304449088077E042489C
:10E6A0000188424800889630814205DD3F48008855
:10E6B00078303E4908806AE03B4801883B48008842
:10E6C0003230814205DD394800881E3037490880E4
:10E6D0005DE035480188354800880A30814205DD13
:10E6E000324800880A303149088050E02E480088BE
:10E6F0002E4908804BE02E480079022847D12A484D
:10E7000000882A490988884239DA27480088FF307A
:10E71000913026490988884206DA24480088FF3863
:10E720007338224908802AE01F48008896301F4924
:10E730000988884205DA1D48008878381B49088016
:10E740001DE019480088323018490988884205DAE6
:10E75000164800881E381549088010E012480088C5
:10E760000A3012490988884205DA104800880A38B8
:10E770000E49088003E00C4800880C4908800B48CB
:10E7800000880849884202DB084608490880F8BD2D
:10E7900054080020420000203800002044080020D7
:10E7A0003C000020C6070000400000203A00002086
:10E7B00044000020002008490880084908800849D2
:10E7C00008804880012008710020064948800880A0
:10E7D00005490860704700003A0000204000002012
:10E7E00044000020440800203C0000200020044990
:10E7F0000870044908700021034801767047000042
:10E8000088000020890000203C0A002070B5002507
:10E810000024FEF7B9F8012863D103213448FCF73E
:10E820008BFC552808D10020324908703249087005
:10E8300000213248017659E02F480078002807D19E
:10E8400002F0ACF82B49087001202B4908704DE00C
:10E8500001202949087002F0A1F82849097E8900A1
:10E86000264A603A50502548047E10E0A000234913
:10E8700060390D5C601E80000858A1001F4A603A94
:10E880005050601E800011460D50601EC4B2002C16
:10E890000ADDA000194960390958601E8000174A36
:10E8A000603A10588142E1D31448007E401CC1B246
:10E8B00012480176007E1E2818DB00210F480176E1
:10E8C00001466039896B0246603AD26B891802466C
:10E8D000603A126C88180321F9F732FC0549087078
:10E8E00004E00020034908700349087070BD00006F
:10E8F0005408002088000020890000203C0A0020E5
:10E90000F0B5A9B004460E46002500270020289047
:10E91000A0216846F9F7C4FCFEF70EFE26490A68F6
:10E9200014216143505024480168142060430818A2
:10E93000C068B0420CD22048016814206043081817
:10E94000C1681D480268142060431018416005E04A
:10E95000194801681420604308184660164840684A
:10E96000002826D0002517E06806070E282F00D3C0
:10E9700016E011480168142068430858B9006A4637
:10E9800050500D4801681420684308184168781CED
:10E9900080001150681CC5B20748007AA842E3DC29
:10E9A00000BF6A0004486946436802209847012076
:10E9B0002890289829B0F0BDE02E002010B500F076
:10E9C000F5FD00F0D7F810F061FB00F00DFB00F052
:10E9D00001F810BD70B541480078912800D070BD95
:10E9E00000F0BEF8012876D13D4800883D490880F6
:10E9F00008468078F021884320303A4988700846DC
:10EA00008078000900013549097A0907090F084390
:10EA1000344988703148807A401E304988720846EF
:10EA20000089401C088108460089C988884216DA96
:10EA300008202C49887200240EE028484188284884
:10EA4000001D415C2748C01C015524484088401CDB
:10EA500022494880601CC4B2072CEEDB2DE01F4821
:10EA600000891E49C98888421CD11C4800791B496D
:10EA70008978401AC5B2681C1A49887200240EE0D1
:10EA8000164841881648001D415C1648C01C0155B7
:10EA900012484088401C11494880601CC4B2AC42F6
:10EAA000EEDB0AE000F00EFD00200C4908700C4976
:10EAB0000888092100F0B8F991E7012000F0C4FCB2
:10EAC000084A917A1088921C00F070F9054908886C
:10EAD000002100F0C1F800BF81E700001C2C0020DD
:10EAE000B82B0020482B00201B49097E002932D07A
:10EAF0001949897E0C225143174A515A174A1180ED
:10EB000000200CE01449897E0C225143124A8918D6
:10EB1000891C0A5C1149891C0A54411CC8B2082886
:10EB2000F0DB0D49897E0C2251430B4A8918897A02
:10EB30000A4A91720121D1720749097E491E064A8B
:10EB400011761146897E491C91761146897E0229EB
:10EB500001DB002191767047142B00203C2B002014
:10EB60000349487B012802D10021014A51737047B3
:10EB70002C2C002010B533484068002861D1314862
:10EB8000007B030011F068FB07590512212E3D4A56
:10EB900059002D480078002807D000202A49087025
:10EBA0002A490888012100F03FF947E0264800780B
:10EBB000002809D000202449087025494A8808887F
:10EBC0000123091D00F040F938E01F4800780028B3
:10EBD00007D000201C4908701C490888022100F059
:10EBE00023F92BE018480078002809D000201649A6
:10EBF000087017494A8808880923091D00F024F97C
:10EC00001CE011480078002807D000200E49087049
:10EC10000E490888092100F007F90FE00A4800783A
:10EC2000002809D000200849087009494A88088846
:10EC30000323091D00F008F900E000BF00BF00F049
:10EC400041FC10BD2C2C00201C2C0020B82B0020D7
:10EC5000542B00207047000070B504460D46344820
:10EC60000088A04263D1002D61D13248007822286B
:10EC70004ED004DC20283DD0212856D141E09028F8
:10EC800002D0912851D115E02A48C08801280AD124
:10EC900000202849087000F015FC27490888002149
:10ECA00000F0C2F805E0032000F0CEFBA0202149CF
:10ECB00008703BE01F4800891E49C98888420AD174
:10ECC00000201C49087000F0FDFB1B49088800214A
:10ECD00000F0AAF80DE01748807A002806D000F06E
:10ECE000F1FB1449087B00F091FB02E0032000F0E7
:10ECF000ABFB1BE0062000F0A7FB11200D490870BC
:10ED000014E0062000F0A0FB11200A4908700DE075
:10ED100000200849087000F0D5FB08494A88088897
:10ED20000923091D00F090F800E000BF00BF70BD8E
:10ED3000302B00201C2C0020B82B0020542B00204E
:10ED400070B50346184C247E022C00DB70BD164CB7
:10ED5000647E0C256C43144D2B5300200AE0155C97
:10ED6000114C647E0C2674430F4EA419A41C255428
:10ED7000441CE0B28842F2D30B4C647E0C267443F0
:10ED8000094EA419A1723446247E641C35462C76A3
:10ED90002C46647E641C6C762C46647E022C01DB5F
:10EDA00000246C7600BFD1E7142B0020F0B585B0AD
:10EDB00007460D4616461A480780002406E03178BB
:10EDC0001748801C0155761C601CC4B2AC42F6DBAF
:10EDD0002C4605E0AA211248801C0155601CC4B2D3
:10EDE000082CF7DB0E480088019008216846C172A4
:10EDF0000021417201720170002406E00848801C65
:10EE0000015D03A80155601CC4B2082CF6DB6946FD
:10EE10000448FCF798FA01200149887205B0F0BD5A
:10EE2000302B00209055044070B504460D4629460D
:10EE3000204610F04DF870BD70B504460D462946C9
:10EE4000204610F053F870BDF8B504460D4616463E
:10EE50001F463B4632462946204610F048F8F8BD8A
:10EE6000F8B507460E4615465C480078002804D0E1
:10EE700009213846FFF7D8FFF8BD002D01D0602DDD
:10EE800004DD09213846FFF7CFFFF5E75448078036
:10EE90004580002406E031785148001D0155761C5C
:10EEA000601CC4B2AC42F6DB00204C4948700846F6
:10EEB0008580FF2088727F20087308468088082894
:10EEC0002EDA0120C8800846808848800120088109
:10EED000434800884349088008468078F0218843E9
:10EEE0004049887008468078000900013B4909794B
:10EEF0000907090F08433B49887038480079401CCE
:10EF00008872002407E03648001D015D3548C01CAA
:10EF10000155601CC4B231488088A042F3DC4AE04D
:10EF20000721681CF9F722F9002907D00721284694
:10EF30000830F9F71BF92949C88005E00721681C4A
:10EF4000F9F714F92549C880062024494880012092
:10EF50000881234800882349088008468078F021EA
:10EF6000884310301F4988700846807800090001E6
:10EF70001A4989880905090F08431A498870084603
:10EF80004088FF2109028843144989880902FF2229
:10EF90001202114008431349488008208872002457
:10EFA00007E00F48001D015D0E48001D0155601C63
:10EFB000C4B2062CF5DB012000F046FA094A917A2A
:10EFC0001088921CFFF7F2FE902004490870054952
:10EFD00008880021FFF740FE00BF4DE71C2C0020F1
:10EFE000B82B0020482B002010B5FFF77DFD1448FA
:10EFF000C07A002822D0124880780009002806D064
:10F00000012807D002280AD0032810D10CE000F014
:10F01000A5F90FE000F09EF800F062FA0AE000F0B7
:10F0200011F800F05DFA05E000F000F902E0FFF7EA
:10F0300011FE00BF00BF00200149C87210BD0000D2
:10F040003C2B002010B540480078112800D010BD9E
:10F050003E4800883F214901884200D0F7E73B48FD
:10F0600080780007000F3849097A0907090F88429C
:10F070000CD000203449087000F024FA34494A8842
:10F0800008880423091DFFF7DFFEE0E72E4800890A
:10F09000401C2D4908810846807A401E8872084627
:10F0A0000089C98888421BDA2848807A082800D05D
:10F0B000CDE700240EE02548C01C015D22484288AF
:10F0C0002348001D815420484088401C1E49488028
:10F0D000601CC4B2072CEEDB062000F0B5F930E06E
:10F0E0001948808818494988401A1849897A8842FD
:10F0F00003DA1648807A082800D0A8E700240EE03A
:10F100001248C01C015D104842881148001D8154FE
:10F11000601CC4B20C484088401C0B4948800A4817
:10F120004088094989888842EADB0020064908703E
:10F1300000F0C8F906494A8808880023091DFFF72E
:10F1400083FE00BF83E700001C2C00203C2B002026
:10F15000542B002070B53248007880210840802868
:10F1600000D170BD2F4800883F214901884200D05E
:10F17000F7E72C48807A082800D0F2E72948807801
:10F1800005072D0F2D0227484088000A0543082D4A
:10F1900000DAE6E700202249487006204880084649
:10F1A000858001200881082088720020C872898823
:10F1B000481C0721F8F7DAFF002909D01849898887
:10F1C000084608300721F8F7D1FF1549C88007E045
:10F1D00013498988481C0721F8F7C8FF1049C880DF
:10F1E000104800881049088008464580002407E040
:10F1F0000C48001D015D0C48001D0155601CC4B287
:10F20000062CF5DB042000F01FF9102004490870DB
:10F21000054A51881088FFF70FFE00BFA1E70000E4
:10F220001C2C00203C2B0020542B002010B54848FB
:10F230000078A02808D046480078912804D0444897
:10F240000078A12800D010BD424800883F21490124
:10F2500088420AD0404908880921FFF7E5FD00F0FF
:10F2600031F900203A490870EDE73A48807A0828D9
:10F270000AD0394908880921FFF7D6FD00F022F9A4
:10F28000002033490870DEE7324880780007000F1D
:10F29000002804D001282DD002284BD136E02C487C
:10F2A0004078002800D050E02A48C078002803D1D8
:10F2B00001202749487003E02648C0782449887215
:10F2C0002348007891280BD022480079002803D1E8
:10F2D00001201F49087303E01E4800791C49087388
:10F2E00091201B49087000F0EDF81949087B00F0E7
:10F2F0008DF82AE016484078002800D025E0A120AB
:10F3000013490870032000F09FF81EE01048407871
:10F31000002800D019E00E480078A02809D10E4935
:10F3200008880821FFF780FD00F0CCF8002008498C
:10F3300008700AE0084908880521FFF775FD00F00C
:10F34000C1F800200249087000BF00BF00BF7AE783
:10F350001C2C00203C2B0020B82B002010B5284886
:10F36000007880210840802800D110BD2448007812
:10F37000002806D0234800883F214901884200D058
:10F38000F3E72048807A1F4989780907090F8842E6
:10F3900003DD1C48807A082800D0E6E71948807809
:10F3A0000007000F002805D0164880780007000FDE
:10F3B000072800DDD9E71348008813490880114861
:10F3C00080780007000F4880002407E00D48C01C2B
:10F3D000015D0D48001D0155601CC4B20A484088FB
:10F3E000A042F3DC00200649087000F06BF80649E3
:10F3F0004A8808880023091DFFF726FD00BFB4E7EF
:10F400001C2C00203C2B0020542B00207F2805DCE6
:10F410007D21C90041430A4A91600DE0F12808DBD3
:10F42000F92806DC0107090F64225143044A916060
:10F4300002E00449024A91600221014A5173704777
:10F440002C2C002018F0010000B5030010F004FF80
:10F450000729050B11171D2329000121144A1173D7
:10F460001449516022E00221114A1173114951607F
:10F470001CE003210E4A11730F49516016E004216C
:10F480000B4A11730D49516010E00521084A1173B0
:10F49000002151600AE00621054A117308495160B4
:10F4A00004E00021024A1173516000BF00BF00BD9B
:10F4B0002C2C0020A8610000F82401002823000063
:10F4C000F049020000200149087370472C2C0020ED
:10F4D000024909880918014A118070472C2C002024
:10F4E00010B52F480078102818D12E484088602881
:10F4F0000ADD2D48807800090001801C2A498870A7
:10F5000022202749087025E027488078000900015B
:10F51000254988702020224908701BE02048007887
:10F52000112816D11E48807A002800D010BD1C4832
:10F530004078002800D0F9E70820194988721A4855
:10F54000807800090001184988702020144908704B
:10F5500000E0EBE7FD20C0001349088008468078F2
:10F56000F02188433030104988700846C078002068
:10F57000C8700846007914200871032088720220A0
:10F58000FFF762FF084A917A1088921CFFF70EFC81
:10F59000054908880021FFF75FFB00BFC6E70000B0
:10F5A0001C2C0020542B0020482B0020244A1188BA
:10F5B00052888A4242D0224A52888A4204DA204A39
:10F5C00052888A1A90B207E01D4A52880023DB4312
:10F5D0009A1A521C521890B2194A5180127B002A72
:10F5E00010D0174A5268002A0CD0154A526882423D
:10F5F00005D9134A5268121A114B5A6002E00022D0
:10F600000F4B5A600E4A527B022A17D10C4A92685D
:10F61000002A0CD00A4A9268824205D9084A9268A8
:10F62000121A074B9A6002E00022054B9A60044AC6
:10F630009268002A02D10122014B5A7370470000E0
:10F640002C2C002010B506F0BFF810BD00BF70478D
:10F6500010B504468020204301460320400205F0F7
:10F660006DFF10BD10B510210320400205F066FFAC
:10F6700010BD000010B50224024805F0AFFF04469B
:10F68000204610BD0106000010B50021014805F01C
:10F6900055FF10BD0106000010B504468020204330
:10F6A0000146024805F04AFF10BD000001060000B7
:10F6B00010B51021014805F041FF10BD0106000002
:10F6C00030B503460C46002101250D48834201D088
:10F6D000002B01D1022030BD012A01D10120FAE71F
:10F6E000002108E0C8002058984202D10025284691
:10F6F000F1E7481C81B29142F4DB2846EBE70000B9
:10F70000FFFF0000002000BF14E00021C200134BE7
:10F710009950C200D2189180C200114B9950C2007A
:10F72000D2189180C2000F4B9950C200D21891801C
:10F73000411C88B24828E8DB0B490C4A11600C498F
:10F740005160002191600B4911610B49D16000218A
:10F750000A4A11800A4A1170704700008C1F00206D
:10F76000CC2100200C240020310C0100781F002047
:10F77000CD0C0100770D0100690D0100D2000020C1
:10F78000D6000020F0B585B00646674F3846039096
:10F79000029000250024002001900090634800683A
:10F7A000002803D061490868804707465F484068E1
:10F7B000002803D05D494868804703905B48806813
:10F7C000002803D05949886880470290574800694B
:10F7D000002803D055490869804700905348C06805
:10F7E000002803D05149C86880470546482D00DDF0
:10F7F00048250098002876D0002D74DD4C480088FC
:10F80000A8420BDA2B463A4649494A48FAF766FFBE
:10F810002B4647494748039AFAF760FF4448008857
:10F82000002833DD42480088A84202D10020404928
:10F830000880002415E0E0003F490858E1003D4AF7
:10F84000515888420BD0E00011460858E1003A4A6E
:10F850005050E00011460858E100384A5050601CF2
:10F8600084B2AC42E7DB0120354908702C460BE03E
:10F870000020E100314A5050E1002F4A5050E10091
:10F880002C4A5050601C84B2482CF1DB2B48006895
:10F890002549884246D0294880882A49884205DA85
:10F8A000264880888019254988803BE0002023492C
:10F8B0008880084600680190012D33DD002408E0AF
:10F8C000601CC0001D490858E1001C4A5050601CD3
:10F8D00084B2681EA042F3DC691EC900174A019871
:10F8E00050501FE0FFE7002015490870002414E085
:10F8F0000020E100114A5050E10089188880E100A1
:10F900000C4A5050E10089188880E1000A4A5050A2
:10F91000E10089188880601C84B2482CE8DB002054
:10F920000349088005B0F0BDFFFF0000781F0020EC
:10F93000D2000020CC2100200C2400208C1F0020AD
:10F94000D6000020881300002E480078401C2D4966
:10F9500008702D480078401C2B4908702B4800780F
:10F96000401C2A4908702A480068401C2849086041
:10F9700008460068FF219131884202D900202449BD
:10F98000086020480078C82802D900201D49087066
:10F990001D480078842802D900201B4908701B48A4
:10F9A0000078502802D900201849087019481849D1
:10F9B0000968405C18490870184812490978405C89
:10F9C00017490870174810490978405C16490870B3
:10F9D00016480E490978405C1549087015480949D0
:10F9E0000978405C14490870144806490978405C5D
:10F9F00013490870134803490978405C124908709C
:10FA000070470000570700205807002059070020C2
:10FA10005C070020BB170200500700204B190200B2
:10FA200051070020131A0200520700205F1B02003A
:10FA300054070020971A020053070020AF1B020052
:10FA400055070020771C02005607002010B58200E1
:10FA5000054BD218525C012A04D100228300024CCB
:10FA60001B195A5410BD0000982A002010B50446F6
:10FA7000204600F04FFA204600F002F810BD0000CA
:10FA800010B50446B248007800287DD1B1480088FE
:10FA9000B149884278DAB148007800284FD0B048A0
:10FAA0000078002803D0AB480088AE490880AE48F3
:10FAB0000078002818D1A7480188AA4800880F308C
:10FAC000814206D30120A8490870A2480088A549B0
:10FAD0000880A0480088A349098888421CDA9D480C
:10FAE0000088A049088017E09E480188994800884E
:10FAF0000F30814206D300209B490870954800884A
:10FB0000984908809348008896490988884203DD0F
:10FB1000904800889349088093480078002857D17E
:10FB200092480078042803D08D480078002807D038
:10FB300088480088822803DA05208C490870A1E0F3
:10FB40008A480078032803D085480078002809D027
:10FB500080480088FF211931884203DA0420834954
:10FB600008708FE081480078022803D07C48007834
:10FB700000280AD077480088FF21AF31884204DA94
:10FB800003207A4908707DE0E0E078480078012899
:10FB900003D073480078002808D06E480088744964
:10FBA000884203DA0220714908706BE06F480078E0
:10FBB000002803D06A480078002863D06548008890
:10FBC0003721090188425DDA01206849087059E04F
:10FBD00065480078012855D164480078012803D091
:10FBE0005F480078002809D05A4800883721090169
:10FBF000884203DB00205D49087043E05B480078E1
:10FC0000022803D056480078002808D051480088C0
:10FC10005749884203DB01205449087032E05348B9
:10FC20000078032803D04E480078002809D04948BE
:10FC30000088FF21AF31884203DB02204B49087066
:10FC400020E04A480078042803D04548007800287E
:10FC500009D040480088FF211931884203DB032086
:10FC6000424908700EE041480078052803D03C481E
:10FC70000078002806D037480088822802DB04205C
:10FC80003A490870FCF766FE3349643988425DD30F
:10FC90003848006800193749086031480078002862
:10FCA00008D000202E490870324908602F4800789B
:10FCB0003149087000F086FD00281FD12D480068EA
:10FCC0002E49884239D300202A4908602A48007802
:10FCD00026490978884205DA27480078401C2649D9
:10FCE00008702AE02448007820490978884224DDF9
:10FCF00021480078401E204908701EE01D48006819
:10FD00001F49884219D300201A4908601A48007810
:10FD100016490978884205DA17480078401C1649C8
:10FD200008700AE01448007810490978884204DD18
:10FD300011480078401E104908700F4800780B49A0
:10FD40000978884202D100200A49086010BD0000ED
:10FD50000B000020020000201C0C000012000020FC
:10FD600008000020040000200A00002006000020F7
:10FD7000760200001800002007000020C05D00008F
:10FD8000407E050000200B4908700B4908700120D7
:10FD90000A4908700A49087000200A4908700A498F
:10FDA00008700A4908800A4908800A4908800A49F7
:10FDB000087070470600002007000020080000209F
:10FDC000090000200A0000200B0000200C00002089
:10FDD0000E000020100000201200002000200B491F
:10FDE00008700B49087001200A4908700A49087018
:10FDF00000200A4908700A4908700A4908800A491F
:10FE000008800A4908800A490870704706000020E7
:10FE10000700002008000020090000200A00002040
:10FE20000B0000200C0000200E000020100000201D
:10FE300012000020F1B5002730480078002809D0D2
:10FE40000320F9F78BFB002804D00320F9F77AFB95
:10FE50002B4908802B4800880A2847D300202949CD
:10FE6000088029480078282829D20320F9F76AFB5E
:10FE70000746002407E060002449085AB84200DD24
:10FE800005E0601CC4B2204800788442F3DB00BF68
:10FE90001D48057808E0681E40001C49085A6900A2
:10FEA0001A4A5052681EC5B2A542F4DC60001749D8
:10FEB0000F5215480078401C1349087016E00026C0
:10FEC0000F2405E060001149085A8619601CC4B26D
:10FED000192CF7D30A213046F8F732F9084908807F
:10FEE0000020094908700120094908700548018867
:10FEF0000098081803490880F8BD00000900002098
:10FF0000020000201600002000000020E80700206A
:10FF1000120000203A4909881E2928DA0021394AAE
:10FF20001180394A118039490988394A914207DCE0
:10FF300038490978002914D034490988914210DDE4
:10FF40000121354A11700021344A1170344A117070
:10FF5000304A11700121334A11700021324A117068
:10FF60004CE02A4909880918284A118046E02449AA
:10FF70000988274A643291422BDB0021234A1180F1
:10FF8000214A11801F490988AF221201914207DCE2
:10FF900020490978002916D01A490988914212DDB2
:10FFA00002211D4A117000211C4A117005211C4AB2
:10FFB00011700021174A117001211A4A1170002195
:10FFC000194A11701AE00F49098809180D4A118061
:10FFD00014E000210D4A11800A4A11800A4909885B
:10FFE0000B4A914205DD00210B4A1170094A11703C
:10FFF00004E0054909880918034A11807047000088
:020000040001F9
:1000000002000020100000200C0000200E00002044
:10001000B80B0000090000200B00002006000020A3
:1000200007000020080000200A0000200148007896
:1000300070470000BC0900200148007A70470000AA
:10004000BC0900200148807870470000BC090020EE
:1000500001480088704700007C000020F8B50023AC
:10006000002500950024002200BF94E001259D405A
:10007000ACB20D8825400095009DA5426FD11A466F
:100080008D79012D0DD1464D03263602AD192D5C1B
:10009000012696403543424E03273F02F619355458
:1000A0000CE03F4D03263602AD192D5C012696402B
:1000B000B5433B4E03273F02F6193554CD78002D4A
:1000C0004ED1374D60352D5CCE78002E01D1012602
:1000D00000E000269640B543314E603635548D78A9
:1000E000002D2ED12E4D19267601AD192D5C8E785E
:1000F000002E01D1012600E000269640B543284E8F
:1001000019277F01F61935540D79002D0ED1244D94
:1001100050352D5C0E79002E01D1012600E000261D
:100120009640B5431E4E5036355423E01C4D503595
:100130002D5C0E7996403543EEB2194D50352E5454
:1001400018E0174D19267601AD192D5C8E78964072
:100150003543134E19277F01F61935540AE018E08C
:100160000F4D60352D5CCE7896403543EEB20C4D88
:1001700060352E544D79012D0AD1094D30352D5C55
:10018000012696403543EEB2054D30352E5400E041
:1001900000BF5D1CABB2082B00DA67E7F8BD0000BA
:1001A00000000440FFB5074615461E4600243846A9
:1001B000019900F01FF8002802D0012004B0F0BD22
:1001C00000240CE00A2060430949085CB04204D1D5
:1001D0002946204600F05EF807E0601C84B20A2041
:1001E00060430349085C0028ECD100BF0020E5E72C
:1001F000B00100200246002A03D1402901DD012080
:100200007047032A03D1022901DD0120F8E7042AFF
:1002100003D1202901DD0120F2E7052A03D120299D
:1002200001DD0120ECE70C2A03D1102901DD0120BA
:10023000E6E70D2A05D1012903DD402901DA012075
:10024000DEE70E2A03D1202901D10120D8E70020C2
:10025000D6E7000010B5064A03231B02D218125C31
:100260008A43034B032424021B191A5410BD0000B7
:100270000000044010B5064A03231B02D218125C8A
:100280000A43034B032424021B191A5410BD000017
:100290000000044070B502460020B1E00A23534339
:1002A0005A4C1B195B1C440004191B199B788B4288
:1002B0007DD10A235343554C1B195B1C4400041980
:1002C0001B195B78082B33D10A2353434F4C1B195E
:1002D0005B1C440004191B574D4C4E4D6419E35CE4
:1002E000012423430A245443484D6419641C4500E7
:1002F00045196457464D474EAD192B550A235343B4
:10030000424C1B195B1C440004191B57404C3546DA
:100310006419E35C022423430A2454433B4D6419CB
:10032000641C450045196457394DAD192B5564E0DF
:100330000A235343354C1B195B1C440004191B1939
:100340005B78092B34D10A235343304C1B195B1CB7
:10035000440004191B572E4C2E4D6419E35C4024B5
:1003600023430A245443294D6419641C450045194C
:100370006457274D274EAD192B550A235343234C61
:100380001B195B1C440004191B57214C354664198A
:10039000E35C8024A3430A2454431C4D6419641C69
:1003A0004500451964571A4DAD192B5525E025E038
:1003B0000A235343154C1B195B1C440004191B579B
:1003C000134C144D6419E35C0A2454430F4D641913
:1003D000641C45004519641965780124AC40234329
:1003E000DCB20A235343094D5B195B1C45004519D8
:1003F0005B57074D074EAD19EC5404E0431CD8B2CF
:10040000032800DA4AE700BF70BD0000B0010020F9
:100410000000044075080000F8B50024FCF7B4FAA9
:10042000012861D100F086FB0446BA220721002092
:1004300003F0C2F8012C21D100F0A0FC00280ED05E
:1004400000F0ACFB054600F09DFB0646012003468C
:10045000024629460090304605F0F0FB50E000F0DF
:100460009DFB054600F08EFB064601200023024658
:1004700029460090304605F0E1FB41E0022C21D1F5
:1004800000F07CFC00280ED000F088FB054600F050
:1004900079FB064601200346024629460090304675
:1004A00005F0CCFB2CE000F079FB054600F06AFB80
:1004B0000646002001231A4629460090304605F0E2
:1004C000BDFB1DE000F05AFC054600F067FB064648
:1004D00000F058FB0746012003462A4631460090AB
:1004E000384605F0ABFB0BE0002003460246014610
:1004F000009005F0A3FB00220721104603F05CF8F2
:10050000F8BD0000F0B585B00024734800780128DC
:1005100024D1FCF739FA012812D1FCF721F800BFE9
:100520000BE0182C02D1601CC4B204E0BA222146B0
:10053000002003F041F8601CC4B2242CF1DBC9E0B8
:10054000FCF75AF9002406E000222146104603F089
:1005500033F8601CC4B2242CF6DBBBE0FCF714FAC1
:10056000012879D1FCF7F6F95C49884271D300F093
:100570000FFB064600F02AFB07460A21F7F7E0FDCD
:1005800005463246294601200BF0E0F800F058FD00
:10059000064600F0E9FC0A210390F7F7D1FD054675
:1005A00000F0F6FA07463246294609F083F8FFF7CD
:1005B00033FF00F0ADFA05462946012007F0C0FBE5
:1005C00000F0FEFA0646FF21F531F7F7CFFDC5B280
:1005D0002946012006F0F0FAFFF728FD0546FFF74F
:1005E00037FD0646FFF72EFD07462B4632463946B5
:1005F000012005F0FDFD00F0EBF80546294601203D
:100600000BF04AFB00F0D0FC054600F0C9FB0646A3
:1006100000F0D0FA074600F0CDFC039000F0C6FBD6
:100620003B4600960195029001460120039A0AF08C
:10063000BFFD00F08DFC054600F084FC064600F08E
:100640008DFC07462A46314607F0B2FD42E003E042
:10065000FFE7FBF7FFFF3DE0FCF7CEF80022232188
:10066000104602F0A9FF00222221104602F0A4FF4A
:1006700000220721104602F09FFF002208211046A9
:1006800002F09AFF00220921104602F095FF002295
:100690000A21104602F090FF00221321104602F0BA
:1006A0008BFF00221121104602F086FF002212214A
:1006B000104602F081FF00220E21104602F07CFF5E
:1006C00000220F21104602F077FF00221021104671
:1006D00002F072FF05B0F0BD05010020B80B00006C
:1006E0000149086070470000840700200248006844
:1006F000401C01490860704780070020F3B581B0B5
:10070000064600200E49086000F01EF8044600F07E
:100710001BF805462F1B3046029903F0F9FE0090A6
:100720000AE000F011F805462F1B06480068002873
:1007300002D004480068804700988742F1D3FEBD8C
:1007400080070020840700200148006870470000EF
:10075000800700200B490978012901D101200FE011
:1007600008490978022901D1022009E005490978E0
:10077000032901D1042003E00121024A1170012064
:10078000704700001507002010B5094B1B8899B26F
:100790000A12C8B2D3433133064C2370C343233308
:1007A000637013465633A37003467133E37010BD74
:1007B000480700201B070020014800887047000000
:1007C0002000002001480088704700003800002009
:1007D0000148007870470000880000200148007838
:1007E000704700008900002010B50022052106484E
:1007F000FAF790FC0402012205210348FAF78AFC6B
:10080000201880B210BD00005408002010B5062248
:1008100005210348FAF77EFCC006C00F10BD00009A
:100820005408002010B5042205210648FAF772FC8E
:100830000402052211460348FAF76CFC201880B226
:1008400010BD00005408002010B506220521024802
:10085000FAF760FCC01110BD5408002010B5022248
:1008600005210248FAF756FC10BD0000540800208C
:1008700010B5062205210348FAF74CFC8006C00F8C
:1008800010BD00005408002010B5042202210348C6
:10089000FAF740FCC007C00F10BD0000540800204C
:1008A00010B5052202210348FAF734FCC007C00F37
:1008B00010BD00005408002010B500220421034898
:1008C000FAF728FC4006400F10BD00005408002035
:1008D00010B5042201210248FAF71CFC801110BD5A
:1008E0005408002010B5002201210248FAF712FC3A
:1008F00010BD00005408002010B505220121034856
:10090000FAF708FC8007800F10BD00005408002093
:1009100010B5012211460248FAF7FCFB10BD000099
:100920005408002010B5002206210C48FAF7F2FB0B
:100930000402012206210948FAF7ECFB2018040200
:10094000022206210548FAF7E5FB201804020322DB
:1009500006210248FAF7DEFB201810BD54080020DB
:1009600010B5042206210C48FAF7D4FB0402052234
:1009700006210948FAF7CEFB201804020622114688
:100980000548FAF7C7FB201804020722062102488F
:10099000FAF7C0FB201810BD5408002010B5022241
:1009A00003210248FAF7B6FB10BD000054080020EE
:1009B00010B5032200210248FAF7ACFB10BD00007D
:1009C0005408002010B5002211460248FAF7A2FB95
:1009D00010BD00005408002010B504220021024878
:1009E000FAF798FB10BD00005408002010B5012252
:1009F00000210248FAF78EFB10BD000054080020C9
:100A000010B5052200210248FAF784FB10BD000052
:100A100054080020322815DA3C498978012903DD81
:100A200001213A4A517070E038498978002905DD82
:100A30002F286ADC0021354A517066E00021334AD4
:100A4000517062E03E2817DA322815DB2F49897889
:100A5000022903DD02212D4A517056E02B49897885
:100A6000012905DD3B2850DC0121284A51704CE06A
:100A70000121264A517048E0502817DA3E2815DB3C
:100A800022498978032903DD0321204A51703CE083
:100A90001E498978022905DD4D2836DC02211B4AD2
:100AA000517032E00221194A51702EE0622817DAA3
:100AB000502815DB15498978042903DD0421134AE0
:100AC000517022E011498978032905DD5F281CDC7B
:100AD00003210E4A517018E003210C4A517014E0B2
:100AE00073280FDA62280DDB08498978042905DDAF
:100AF00070280ADC0421054A517006E00421034AEB
:100B0000517002E00521014A51707047BC09002074
:100B10000148007870470000070000200148006885
:100B2000704700008C1F00200148007870470000CB
:100B3000F10000200148007870470000F00000201C
:100B4000F8B5002600240025FCF740FE07460A21E0
:100B5000F7F7F6FA054609480068854200D303E036
:100B600006480068461B34467D200001844200D3BD
:100B70000446034804600068F8BD00002C01002012
:100B8000280100200148007870470000FD00002087
:100B900001480079704700003C2800200148407857
:100BA00070470000FD0000200148007A70470000F7
:100BB0003C28002001484079704700003C28002074
:100BC00001480088704700002200002010B5002472
:100BD000FFF7DEFF00280AD10A4800880A49884248
:100BE00002DB0846074908800648048808E00548F3
:100BF0000088FCF799FB84B20448844200DB044679
:100C0000204610BD3A000020C6070000CE040000B8
:100C1000002005490988054A914202DB1146024A33
:100C200011800149088870473A000020C60700007B
:100C3000F8B50027002500260024FFF7C3FE05466F
:100C4000FFF7D4FE0646F020284000110A2805DBF5
:100C5000F02028400011C01C044303E0F02028408D
:100C60000011044324022807000F0A2804DB280788
:100C7000000FC01C044302E02807000F04432402B5
:100C8000F020304000110A2805DBF0203040001130
:100C9000C01C044303E0F020304000110443240250
:100CA0003007000F0A2804DB3007000FC01C044384
:100CB00002E03007000F0443002C01D10248F8BDC8
:100CC00027463846FBE70000FFFF0000F8B5002785
:100CD000002500260024FFF77FFE0546FFF790FE63
:100CE0000646F020284000110A2805DBF0202840A5
:100CF0000011C01C044303E0F0202840001104430D
:100D000024022807000F0A2804DB2807000FC01C54
:100D1000044302E02807000F04432402F02030407F
:100D200000110A2805DBF02030400011C01C0443EC
:100D300003E0F02030400011044324023007000F8C
:100D40000A2804DB3007000FC01C044302E0300710
:100D5000000F0443002C01D10248F8BD2746384655
:100D6000FBE70000FFFF000010B50024FFF720FEA6
:100D70000446204610BD012070470000014800785D
:100D800070470000510700200148007870470000BC
:100D9000530700200148C07B70470000C8090020AD
:100DA0000148007A70470000C809002070B500248F
:100DB0000F48C07A012810D10D490868FBF704FFDD
:100DC0000546FF35F5357D21C9002846F7F7B8F906
:100DD00084B2632C0ADD632408E0054800883230C1
:100DE00084B264212046F7F7C1F984B2204670BD71
:100DF000C809002070B5002407490868FBF7E4FE25
:100E000005466421F7F79CF984B20448844200DD6A
:100E10000446204670BD0000C8090020DE03000023
:100E200010B5002400F016F8012801D103240CE0CD
:100E300000F010F8022802D1FF24373405E00A211F
:100E400003480088F7F792F984B2204610BD0000ED
:100E50000200002001480078704700000B000020CD
:100E600010B50024044804F0B9FB002801D0012487
:100E700000E00024204610BD0307000010B5002448
:100E8000044804F0ABFB002801D0012400E000245A
:100E9000204610BD0507000010B50024044804F0EA
:100EA0009DFB002801D0012400E00024204610BD55
:100EB0000707000010B50024062004F08FFB00286F
:100EC00001D0012400E00024204610BD10B500240C
:100ED000052004F083FB002801D0012400E0002459
:100EE000204610BD10B50024044804F077FB00280C
:100EF00001D0012400E00024204610BD06070000B8
:100F000010B50024044804F069FB002801D0012436
:100F100000E00024204610BD0305000010B50024A9
:100F2000044804F05BFB002801D0012400E0002409
:100F3000204610BD040500000148807A704700007B
:100F4000C809002001488078704700005C0A002032
:100F500001484068704700005C0A00200148407862
:100F6000704700005C0A002070B50024FFF710FEF7
:100F7000002803D1FCF72AFC04460DE0FFF708FE29
:100F8000012806D1FCF722FC0546FCF7CDF9044602
:100F900002E0FCF71BFC0446204670BD0148007CC3
:100FA00070470000C80900200148407A70470000DF
:100FB000C809002070B500240F48C07A012810D15C
:100FC0000D494868FBF700FE0546FF35F5357D21E4
:100FD000C9002846F7F7B4F884B2632C0ADD63240D
:100FE00008E005488088323084B264212046F7F753
:100FF000BDF884B2204670BDC809002070B5002439
:1010000007494868FBF7E0FD05466421F7F798F8C3
:1010100084B20448844200DD0446204670BD0000CE
:10102000C8090020DE0300000148007B7047000073
:10103000C80900200148007870470000F400002033
:1010400070B50024FFF7A4FD002803D1FCF7E0FBF6
:1010500004460FE0FFF79CFD012807D10020FCF7B4
:10106000D7FB0546FCF760F9044603E00020FCF7D7
:10107000CFFB0446204670BD014800787047000051
:101080004200002070B505460024032D00D170BD3C
:10109000002D01D0012D1BD181210320800204F0FD
:1010A0004DFA8021134804F049FA32211248FFF723
:1010B00025FB002409E0A200104BD2189178A20071
:1010C000985A04F03BFA601CC4B23B2CF3DB0FE0EF
:1010D000022D0DD1002409E0A200094BD21891780D
:1010E000A200985A04F02AFA601CC4B23B2CF3DB2D
:1010F00000BFCCE702060000A0860100F40D02004C
:10110000E00E0200F8B5002100240023002200BFF9
:101110000AE001258D40ABB205881D402C469C425B
:1011200000D10A464D1CA9B21029F2DB0588FF2D1B
:101130001FDC284D6D7E0688B543264E75763546F4
:101140002D7E0688B543234E357635466D7E8678EE
:10115000F607F60F964035431E4E757635462D7EC2
:10116000867802273E40760896403543194E3576FC
:1011700022E0184DED7E0688B543164EF5763546CD
:10118000AD7E0688B543134EB5768578ED07ED0F35
:101190001646083EB5400F4EF67E35430D4EF576A9
:1011A0008578022635406D081646083EB540094E42
:1011B000B67E3543074EB5760025009505E000BFA5
:1011C0006D462D786D1CEEB200966D462D78012D82
:1011D000F5D9F8BD206B0440C107C90F002905D01F
:1011E0000021394A1171002238490A710221014057
:1011F000002905D00021344A1172002233490A72B5
:1012000004210140002905D000212F4A117300223A
:101210002E490A7308210140002905D000212A4ADD
:101220001174002229490A7410210140002905D0B7
:101230000021254A1175002224490A752021014008
:10124000002905D00021204A117600221F490A7684
:1012500040210140002904D000221B494A711B494A
:101260004A7180210140002904D0002216494A72A7
:1012700016494A72FF2101310140002904D00022A1
:1012800011494A7311494A73012149020140002959
:1012900004D000220C494A740C494A740121890285
:1012A0000140002904D0002207494A7507494A75C0
:1012B0000121C9020140002904D0002202494A76D6
:1012C00002494A767047000000600040006100401B
:1012D000C107C90F002905D001223C490A7100212C
:1012E0003B4A117102210140002905D001223749F2
:1012F0000A720021364A117204210140002905D0EA
:10130000012232490A730021314A11730821014038
:10131000002905D001222D490A7400212C4A11749C
:1013200010210140002905D0012228490A75002119
:10133000274A117520210140002905D001222349A7
:101340000A760021224A117640210140002905D069
:1013500001221E494A7100221D494A718021014023
:10136000002905D0012219494A72002218494A72FF
:10137000FF2101310140002905D0012213494A73A0
:10138000002213494A73012149020140002905D076
:1013900001220E494A7400220D494A740121890232
:1013A0000140002905D0012208494A750022084958
:1013B0004A750121C9020140002905D001220349D3
:1013C0004A76002202494A767047000000610040D8
:1013D0000060004010B50C480078002803D00B4A8C
:1013E00050689168884708484078002803D0084A28
:1013F00050689168884704488078002803D0054ADF
:1014000050689168884710BD0060004000030020CC
:10141000800400200006002010B50848007900284C
:1014200003D0074A10695169884704484079002869
:1014300003D0044A50689168884710BD006000409E
:10144000000300208C04002010B50848007A002812
:1014500003D0074AD069116A88470448407A0028B7
:1014600003D0044A50689168884710BD006000406E
:10147000000300209804002010B50848007B0028D5
:1014800003D0074A906AD16A88470448407B002805
:1014900003D0044A50689168884710BD006000403E
:1014A00000030020A404002010B50848007C002898
:1014B00003D0074A506B916B88470448407C002852
:1014C00003D0044A50689168884710BD006000400E
:1014D00000030020B004002010B50848007D00285B
:1014E00003D0074A106C516C88470448407D00289F
:1014F00003D0044A50689168884710BD00600040DE
:1015000000030020BC04002010B50848007E00281D
:1015100003D0074AD06C116D88470448407E0028EC
:1015200003D0044A50689168884710BD00600040AD
:1015300000030020C804002010B50848407F0028A0
:1015400003D0074A5068916888470448007F002804
:1015500003D0044A906DD16D884710BD00600040F3
:10156000D40400200003002010B50848407800286B
:1015700003D0074A506891688847044800780028DB
:1015800003D0044A506E916E884710BD2060004021
:10159000E00400200003002010B50948007900286D
:1015A00003D0084A106F516F88470548001D4078E6
:1015B000002803D0044A50689168884710BD000095
:1015C0002060004000030020EC04002010B5034A16
:1015D000D06F78329168884710BD0000000300206A
:1015E00010B5024A50689168884710BD84030020F6
:1015F00010B50948007C002803D0084A506891685B
:101600008847054810304078002803D0044A5068C5
:101610009168884710BD00002060004090030020C2
:101620001005002010B5024A50689168884710BD27
:101630009C03002010B5024A50689168884710BD8D
:10164000A803002010B50948007F002803D0084AED
:1016500050689168884705481C304078002803D0BE
:10166000044A50689168884710BD0000206000401F
:10167000B40300203405002010B50C480078002881
:1016800003D00B4A50689168884708484078002882
:1016900003D0084A50689168884704488078002839
:1016A00003D0054A50689168884710BD40600040EB
:1016B000C003002040050020C006002010B50D48E2
:1016C0000079002803D00C4A50689168884709487F
:1016D000001D4078002803D0084A50689168884768
:1016E0000448001D8078002803D0054A506891689E
:1016F000884710BD40600040CC0300204C0500200E
:10170000CC06002010B50D48007A002803D00C4A02
:10171000506891688847094808304078002803D00D
:10172000084A506891688847044808308078002843
:1017300003D0054A50689168884710BD406000405A
:10174000D803002058050020D806002010B50D4809
:10175000007B002803D00C4A5068916888470948EC
:101760000C304078002803D0084A506891688847B8
:1017700004480C308078002803D0054A50689168EE
:10178000884710BD40600040E4030020640500204D
:10179000E406002010B50D48007C002803D00C4A58
:1017A000506891688847094810304078002803D075
:1017B000084A5068916888470448103080780028AB
:1017C00003D0054A50689168884710BD40600040CA
:1017D000F003002070050020F006002010B5024A3A
:1017E00050689168884710BDFC03002010B5094877
:1017F000007E002803D0084A506891688847054851
:1018000018304078002803D0044A5068916888470F
:1018100010BD000040600040080400208805002042
:1018200010B50948007F002803D0084A5068916825
:10183000884705481C304078002803D0044A506887
:101840009168884710BD00004060004014040020EB
:101850009405002010B508480078002803D0074AF6
:1018600050689168884704484078002803D0044AAB
:1018700050689168884710BD6060004020040020D7
:10188000A005002010B509480079002803D0084AB7
:101890005068916888470548001D4078002803D0AB
:1018A000044A50689168884710BD0000606000409D
:1018B0002C040020AC05002010B50948007A00284F
:1018C00003D0084A50689168884705480830407836
:1018D000002803D0044A50689168884710BD000072
:1018E0006060004038040020B805002010B5024AAE
:1018F00050689168884710BD4404002010B5024A22
:1019000050689168884710BD5004002010B5094800
:10191000007D002803D0084A506891688847054830
:1019200014304078002803D0044A506891688847F2
:1019300010BD0000606000405C040020DC05002059
:1019400010B50948007E002803D0084A5068916805
:101950008847054818304078002803D0044A50686A
:101960009168884710BD0000606000406804002056
:10197000E805002010B50948007F002803D0084A78
:1019800050689168884705481C304078002803D08B
:10199000044A50689168884710BD000060600040AC
:1019A00074040020F405002010B5FE48006880791A
:1019B000002806D001286ED002286DD003286CD1F3
:1019C00004E2F8480068407903000EF045FC0A067E
:1019D00014BC2BBC47BC67BC9BBC0AF0BFFC0020FE
:1019E000F0490968C873EF4800684079401CED4928
:1019F00009684871AEE0EC490969EA4A1268D27A8E
:101A0000885C0AF023FDE74800684079401CE549FE
:101A100009684871E34800684079401CE149096859
:101A2000487197E001F030FF002810D10AF00EFD58
:101A3000DC4800684079401CDA4909684871D94897
:101A400000684079401CD7490968487105E00AF0F0
:101A5000AFFC0020D349096848717BE001F014FF16
:101A6000002811D101200AF0F1FCCE48006840792D
:101A7000401CCC4909684871CA4800684079401C3C
:101A8000C8490968487105E00AF092FC0020C54980
:101A9000096848715EE05FE0FEE0A3E101F0F4FE5A
:101AA000002828D1BF490968C97A24225143BF4A76
:101AB00012688918BB4A1268D27B885C0AF0C6FC9F
:101AC000B8480068C07B401CB6490968C873B5486F
:101AD0000068C07B242814D3B24800684079401CB9
:101AE000B04909684871AF4800684079401CAD4969
:101AF0000968487105E00AF05BFC0020A949096803
:101B0000487127E001F0C0FE002815D1A548006803
:101B1000C07A401CA3490968C872A2480068C07A0C
:101B2000A1490978884207DB00209E490968C872EC
:101B300001209C49096888710AF03AFC0020994903
:101B40000968487106E00AF033FC002095490968ED
:101B5000487100BF00BF4FE1924800684079030020
:101B60000EF07AFB080513912A91479170910AF0C3
:101B7000F5FB00208B490968C8738A4800684079E2
:101B8000401C88490968487184E087490969854A89
:101B90001268D27A885C0AF059FC82480068407961
:101BA000401C8049096848717E4800684079401CA3
:101BB0007C49096848716DE001F066FE002811D18A
:101BC00026200AF043FC774800684079401C75499C
:101BD00009684871734800684079401C7149096878
:101BE000487105E00AF0E4FB00206E49096848717D
:101BF00050E001F049FE00281DD101200AF026FC2A
:101C000068480068C07B401C66490968C87365481D
:101C10000068C07B242814D3624800684079401CC7
:101C20006049096848715F4800684079401C5D4917
:101C30000968487105E00AF0BBFB002059490968B2
:101C4000487127E001F020FE002815D155480068B2
:101C5000C07A401C53490968C87252480068C07A6B
:101C600051490978884207DB00204E490968C8724B
:101C700002204C49096888710AF09AFB0020494902
:101C80000968487106E00AF093FB0020454909689D
:101C9000487100BF00BFAFE04248006840790300D0
:101CA0000EF0DAFA0805138B2A8B478B638B0AF048
:101CB00055FB00203B490968C8733A4800684079E1
:101CC000401C3849096848717EE037490969354A3E
:101CD0001268D27A885C0AF0B9FB32480068407911
:101CE000401C3049096848712E4800684079401C02
:101CF0002C490968487167E001F0C6FD002811D140
:101D000025200AF0A3FB274800684079401C25499C
:101D100009684871234800684079401C21490968D6
:101D2000487105E00AF044FB00201E49096848712B
:101D30004AE001F0A9FD002810D10AF087FB1948FC
:101D400000684079401C17490968487115480068C7
:101D50004079401C13490968487105E00AF028FBE6
:101D600000201049096848712EE001F08DFD00281F
:101D700015D10C480068C07A401C0A490968C8722D
:101D800008480068C07A08490978884207DB0020C3
:101D900004490968C87203200249096888710AF079
:101DA00007FB05E0D4070020182F0020D0070020F3
:101DB000002012490968487106E00AF0F9FA00208B
:101DC0000E490968487100BF00BF15E000200B49AB
:101DD0000968887109490968487106200749096836
:101DE000C87009E00AF0E4FA002004490968487163
:101DF00002490968887100BF00BF10BDD4070020E8
:101E000010B56A480068407903000EF025FA09060B
:101E100010C627C644C6608EC6000AF09FFA634803
:101E200000684079401C614909684871BCE060491C
:101E300009695E4A1268D27A885C0AF007FB5B483F
:101E400000684079401C5949096848715748006842
:101E50004079401C554909684871A5E001F014FD1E
:101E6000002811D14F200AF0F1FA5048006840795B
:101E7000401C4E49096848714C4800684079401C34
:101E80004A490968487105E00AF092FA002047497A
:101E90000968487188E001F0F7FC002810D10AF0C9
:101EA000D5FA424800684079401C404909684871A9
:101EB0003E4800684079401C3C490968487105E08B
:101EC0000AF076FA00203949096848716CE001F09F
:101ED000DBFC002822D135480068C07A401C334919
:101EE0000968C87231480068C07A31490978884267
:101EF0000FDB00202D490968C8722C480068407922
:101F0000401C2A490968487100202849096848622C
:101F100008E0002025490968487103E000202349B2
:101F2000096848710AF044FA3EE020480068407CA5
:101F3000002816D01E48C068002803D01C48C1687D
:101F4000192088470020194909684862174909681B
:101F50004871164909688871052014490968C870D4
:101F60001AE012480068406A282807D20F48006823
:101F7000406A401C0D49096848620DE000200B4989
:101F800009684862094909684871084909688871FF
:101F9000052006490968C87006E00AF009FA002021
:101FA00002490968487100BF00BF10BDD407002076
:101FB000182F002010B50024F7480068807A012807
:101FC0007ED1F5480068C07900287AD0F2480068D0
:101FD0008079002804D0012874D0022873D191E1BF
:101FE000ED480068007B24286ED2EB480068C07979
:101FF00001287AD1002475E0E7480068C07A2421DE
:102000004843E64909684018E3490968097B415C8F
:10201000E1480068C07A24225043E14A12688018DF
:10202000DD4A1268127B805C814229D0DA48006860
:10203000C07A24214843DA4909684018D64909681A
:10204000097B415CD4480068C07A24225043D34ABB
:1020500012688018D04A1268127B8154CE480068FA
:10206000407B242805D3CC480068007BCA49096816
:102070004873C9480068007BC7490968887308E04D
:10208000C5480068407B242803D20120C249096862
:102090008871C1480068007B401CBF49096808730B
:1020A000BD480068007B242808D3BB480068407BFB
:1020B000242803D20120B84909688871B64805E090
:1020C000D3E1CDE169E0BAE138E00EE00068007BE1
:1020D000242804D2B04800688079012800D103E0A8
:1020E000601CC4B2242C87D356E0002413E0AA4815
:1020F0000068C07A24214843A94909684018015D55
:10210000A5480068C07A24225043A44A1268801867
:102110000155601CC4B2242CE9D300209E490968F3
:10212000487323209C490968887301209A490968EB
:10213000887124209849096808732DE00020964989
:102140000968087394480068C07A401C924909687D
:10215000C87291480068C07A92490978884217DBB2
:102160008D480068007C012804D102208A49096852
:10217000887106E0002088490968887186490968E5
:10218000C871002084490968C872834909680874C5
:10219000002081490968487161E17F480068407901
:1021A00003000EF059F8080513A62AA651A68EA61C
:1021B00001207949096808740AF0D0F87648006867
:1021C0004079401C74490968487199E0754909696A
:1021D000714A1268D27A885C0AF038F96E48006851
:1021E0004079401C6C49096848716B480068407927
:1021F000401C69490968487182E001F045FB0028EC
:102200001BD165490968497B491CC8B20AF01EF90F
:1022100061480068407B60490968C8735E4800688F
:102220004079401C5C49096848715B480068407906
:10223000401C59490968487105E00AF0B9F80020C6
:102240005549096848715BE001F01EFB00282BD15D
:1022500051490968C97A24225143504A12688918A1
:102260004D4A1268D27B885C0AF0F0F84A48006850
:10227000C07B401C48490968C87347480068C07B58
:1022800045490968897B88421ADD434800684079DE
:10229000401C4149096848713F4800684079401C2A
:1022A0003D49096848710BE00AF082F83A48006835
:1022B000407B39490968C87300203749096848716B
:1022C0001EE001F0E1FA00280CD133490968887159
:1022D000242031490968C8732F49096848732E4979
:1022E000096888730AF064F800202B49096848716E
:1022F00006E00AF05DF8002027490968487100BF30
:1023000000BFACE024480068407903000DF0A4FF52
:1023100008050F8E268E4C8E688E0AF01FF81E4818
:1023200000684079401C1C490968487185E01D49D6
:102330000969194A1268D27A885C0AF087F8164847
:1023400000684079401C14490968487112480068C7
:102350004079401C1049096848716EE001F094FA18
:10236000002811D125200AF071F80B480068407947
:10237000401C094909684871074800684079401CB9
:1023800005490968487105E00AF012F80020024981
:102390000968487151E00000D4070020D0070020F0
:1023A000CC070020182F002001F06EFA002810D171
:1023B0000AF04CF8644800684079401C624909689A
:1023C0004871614800684079401C5F49096848715C
:1023D00005E009F0EDFF00205B49096848712CE039
:1023E00001F052FA00281AD157480068C07A401C00
:1023F00055490968C87254480068C07A5349097839
:1024000088420CDB002050490968C8724E490968AF
:1024100088714D49096848714B490968C87109F0CC
:10242000C7FF002048490968487106E009F0C0FF6D
:10243000002045490968487100BF00BF0FE009F05E
:10244000B7FF00204049096848713F490968887111
:102450003D49096808733C490968C87200BF71E0CA
:1024600000203949096888726CE037480068807A32
:10247000022867D134480068007A00285ED03248CC
:1024800000684079002804D001280CD0032846D1E8
:102490001BE009F063FF2C4800684079401C2A4982
:1024A0000968487149E0002009F0D0FF264800681B
:1024B0004079401C244909684871234800684079E4
:1024C000401C21490968487137E009F011FF0028D4
:1024D00012D11D4800684078401C1B4909684870AB
:1024E000194800684078032812D301F06DFA0020E3
:1024F0001549096848700BE0002013490968087203
:10250000AA2011490968887000200F49096848709D
:1025100009F04EFF00200C49096848710DE009F0F0
:1025200047FF002008490968487107490968487051
:10253000AA2005490968887000BF03E0002002490D
:102540000968887210BD0000D4070020182F0020F1
:10255000F8B504460D4600260C2060431D49085C72
:10256000002801D00120F8BD0C2060431949401813
:1025700085600C20604340188068002801D101204C
:10258000F1E701210C206043124A11540022204639
:10259000E317DB0E1B185B115B01E31A9B000E4F68
:1025A000DB19E717FF0E3F197F11DA550DF086FE94
:1025B00000222046E317DB0E1B185B115B01E31AB8
:1025C0009F00064BFB18E717FF0E3F197F11DA55E6
:1025D0003046C8E700030020006000400061004072
:1025E00000BFFEE709480088401C084908800846EB
:1025F00000880749884208DD06480078002804D092
:10260000084602490880012088707047EC000020CD
:10261000DC050000F000002010B515488078012886
:1026200024D11448007801280CD1134800780128DF
:1026300008D1002011498870084602F09DFD002055
:102640000D4908700B48007802280CD10C4800781E
:10265000012808D1002009498870084602F08CFD45
:1026600000200749087000200249087010BD0000D2
:10267000EC000020F0000020F2000020FD0000200F
:10268000F30000207047000010B500F077FE01282D
:1026900003D1002001490880887010BDEC000020A3
:1026A000F0B505460E46174600243A463146284600
:1026B00000F072FE00BF42E000202101394A12689A
:1026C00050522101374A12688918488000212001A0
:1026D000344A1268801881802001324A12688018BA
:1026E000C18020012F4A12688018017220012D4AF2
:1026F00012688018417220012A4A1268801881727B
:102700002001284A12688018C17200202101254A40
:1027100012688918087300212001224A1268801863
:102720004173002021011F4A126889188873002113
:1027300020011C4A12688018C173601CC4B21A4878
:102740004078A042B8DC64201849096808807D20E0
:10275000C0001649096848801548144909688880EE
:102760007D20000111490968C88010490968088165
:1027700010480E49096848810F480C49096888814A
:1027800040000A490968C88132200849096808825E
:10279000FF20F530054909684882044909688882A4
:1027A000F0BD00009407002088070020900700205B
:1027B0004C040000102700003075000038B50024DC
:1027C00004E0002013490855601C84B2282CF8D37B
:1027D00001216846417001706A460F490D48FFF7B4
:1027E0005FFF7D21C900322000F0C6F90B490C487B
:1027F00000F0E0F90948643000F072F90748C83089
:1028000000F07EF9074800F091F9074800F0A4F9BC
:1028100038BD00004C280020AC1302002823000023
:10282000B80B0000542400001027000010B5284801
:102830000078002803D101202549087046E024488B
:102840000078012810D123480078012808D1002001
:1028500021498870084602F08FFC00201D4908704D
:1028600002201B49087031E019480078022810D175
:102870001A480078012808D10020174988700846B6
:1028800002F07AFC002015490870032010490870F6
:102890001CE00F480078032803D104200C4908707D
:1028A00014E00B480078042803D10520084908707B
:1028B0000CE007480078052803D005480078062872
:1028C00004D10020024908700549087010BD0000BD
:1028D000F0000020F2000020FD000020F3000020A6
:1028E000F4000020F8B50024002500263E480078BA
:1028F00000281ED13D480078002803D101203B4923
:10290000087016E039480078012803D102203749C1
:1029100008700EE035480078022803D103203349BF
:10292000087006E031480078032802D100202F49C2
:1029300008702D48007801280ED1012417250026A3
:102940002B480123324629460090204601F034FEF0
:1029500001202849087046E02348007802280FD15A
:1029600001243B2500262248401C012332462946EB
:102970000090204601F020FE01201F49087032E03F
:102980001948007803280DD1FEF702F9002803D179
:1029900001201A49087102E00020184908710DF061
:1029A0002DFC20E01048007804280DD1FEF702F934
:1029B000002803D101201149487102E000200F498D
:1029C00048710DF01BFC0EE007480078052803D184
:1029D00006200549087006E003480078062802D161
:1029E000052001490870F8BDF0000020F10000202A
:1029F000FD000020F2000020F30000203C28002011
:102A000010B5044623000DF027FC095B060E1617CF
:102A10001819595A5E00F9F79DFF2C49884201D3D5
:102A2000FFF760FF50E0F9F795FF2849884201D38E
:102A3000FFF7FCFE48E047E046E045E0F9F78AFF93
:102A40002249884239D301F071FD214800780328DA
:102A500014D120480078002810D1FEF7A5F80028EE
:102A600006D101201C4988608868FAF737FF05E025
:102A70000020194988608868FAF730FF1448007808
:102A8000012805D113480078002801D1FAF7F4F89D
:102A900010480078052803D10120104908700AE089
:102AA0000C480078062803D102200C49087002E087
:102AB00000200A4908700BF067F905E004E003E024
:102AC000FFF790FD00E000BF00BF10BDB80B000095
:102AD000F1000020F00000203C280020F40000203D
:102AE00001460020054A126852898A4201DC012011
:102AF00002E0024A1268118170470000900700202E
:102B000001460020084A126812898A4201DB01202E
:102B100009E0054A126892898A4201DC012002E03C
:102B2000014A126851817047900700200146002039
:102B3000084A126852898A4201DB012009E0054AED
:102B40001268D2898A4201DC012002E0014A12683F
:102B5000918170479007002001460020054A1268C5
:102B600092898A4201DB012002E0024A1268D18187
:102B70007047000090070020024600200C4B1B68A5
:102B80001B8A934201DD012010E08A4201DB012013
:102B90000CE0074B1B689B888B4201DC012005E0A1
:102BA000034B1B681A80024B1B685980704700005A
:102BB00090070020024600200C4B1B681B8A9342A2
:102BC00001DD012010E08A4201DB01200CE0074B0F
:102BD0001B685B88934201DB012005E0034B1B6807
:102BE0009A80024B1B68D980704700009007002034
:102BF00070B5044600250C206043FE490968401862
:102C00004068002807D00C216143FA4A12688918ED
:102C10004868804705460C206043F6490968085C0F
:102C2000002873D10C206043F2490968401880687D
:102C3000002874D02001F04909684018C07A0228A1
:102C40000AD1032D08D10C206043EA4A126880188B
:102C500081680120884762E02001E749096840183F
:102C6000C07A02280AD1042D08D10C206043E14A21
:102C70001268801881680220884750E02001DE49F0
:102C800009684018C07A02280AD1052D08D10C2005
:102C90006043D84A126880188168032088473EE064
:102CA0002001D54909684018C07A02280AD1062DAA
:102CB00008D10C206043CF4A126880188168042034
:102CC00088472CE02001CC4909684018C07A0228C6
:102CD0000AD1072D08D10C206043C64A126880181B
:102CE0008168052088471AE02001C3490968401817
:102CF000C07A02280BD1082D09D10C206043BD4AAF
:102D00001268801881680620884708E00DE00C20D2
:102D10006043B84A12688018816800208847200103
:102D2000B54909684018C5720CE30C206043B149ED
:102D30000968085C012873D10C206043AD4909681B
:102D400040188068002874D02001AB4909684018F9
:102D5000C07A03280AD1022D08D10C206043A54A6D
:102D60001268801881680120884762E02001A2492A
:102D700009684018C07A04280AD1022D08D10C2015
:102D800060439C4A1268801881680220884750E09E
:102D90002001994909684018C07A05280AD1022DF6
:102DA00008D10C206043934A126880188168032080
:102DB00088473EE02001904909684018C07A0628FB
:102DC0000AD1022D08D10C2060438A4A126880186B
:102DD0008168042088472CE0200187490968401851
:102DE000C07A07280AD1022D08D10C206043814AFD
:102DF000126880188168052088471AE020017E4902
:102E000009684018C07A08280BD1022D09D10C207E
:102E10006043784A1268801881680620884708E075
:102E20000DE00C206043734A12688018816800200E
:102E300088472001704909684018C57282E20C2059
:102E400060436C490968085C0228F7D1002D7DD1E8
:102E5000200169490968085A68490968098A88424D
:102E600075DA200164490968085A0A3081B22001E4
:102E7000614A1268115220015F490968085A5F4986
:102E80000968098A884231DB20015B4909684018DA
:102E900040885A4909680988884227DB2001564939
:102EA00009684018408855490968498888421DDCEE
:102EB00000202101504A12688918488020014E499B
:102EC00009684018807A0028B8D10C20604349492D
:102ED0000968401880680028B0D00C206043454A3B
:102EE000126880188168012088472BE2200142493E
:102EF0000968085A41490968098A88429EDB20010D
:102F00003D490968401840883C49096889888842D9
:102F100094DB20013849096840184088374909681E
:102F2000C98888428ADC00202101334A1268891846
:102F300048802001304909684018807A0028D4D19F
:102F40000C2060432B490968401801E063E00BE066
:102F500080680028C9D00C206043264A1268801877
:102F6000816802208847EDE100202101224A126891
:102F7000891848802101204A12688918C8720021E6
:102F800020011D4A12688018C18020011A4A126867
:102F9000801841722001184A1268801881721848FE
:102FA00001782001144A1268801801720020210162
:102FB000114A12688918888021010F4A12688918FD
:102FC000087321010C4A12688918487321010A4AC2
:102FD00012688918887300212001074A1268801836
:102FE000C1730C20604303490968401880680028B9
:102FF000B9D007E08C07002094070020900700203C
:10300000880700200C206043CF4A1268801881682E
:103010000020884796E1012DA5D12001CB49096800
:103020004018C07AA84225D000212001C74A126862
:103030008018418000202101C44A12688918C88084
:103040002001C24909684018C572C14800782101B1
:10305000BE4A12688918487200202101BB4A1268D2
:1030600089188880BA4801782001B84A1268801807
:10307000017267E12001B54909684018007AB44936
:103080000978884220D0B24800782101AF4A1268FE
:10309000891808722001AD4909684018407AAC4986
:1030A0000978884209D02001A84909684018808819
:1030B0002101A64A12688918C88000212001A34A6C
:1030C00012688018818012E02001A0490968401828
:1030D0008088A04988420AD220019C49096840188A
:1030E00080880A302101994A126889188880200155
:1030F0009649096840184088964988420AD22001BA
:1031000092490968401840880A3021018F4A1268A4
:103110008918488020018D4909684018407A8C49F7
:103120000978884205D001202101884A126889184F
:1031300088722001854909684018408886490968D5
:103140000988884204DB00212001804A126811525C
:1031500020017E4909684018807A00287ED10C2021
:1031600060437949096840188068002877D02001B9
:103170007649096840184088774909680989884272
:1031800014DB2001714909684018007B00280DD12B
:103190000C2060436C4A12688018816803208847BD
:1031A00001202101694A12688918087320016749C2
:1031B000096840184088684909684989884214DBD1
:1031C0002001624909684018407B00280DD10C207D
:1031D00060435D4A12688018816804208847012096
:1031E00021015A4A12688918487320015749096811
:1031F00040184088584909688989884214DB2001B1
:10320000524909684018807B00280DD10C2060438A
:103210004D4A1268801881680520884701202101E5
:103220004A4A126889188873200148490968401879
:10323000408849490968C989884210DB200143490F
:1032400009684018C07B00287CD10C2060433E4AAE
:103250001268801881680620884701E007E03BE09B
:1032600001202101394A12688918C8736AE02001D7
:10327000364909684018407A01282ED13448007830
:1032800002282AD12001314909684018C0883249F2
:103290000968498A884255DB20012C490968401891
:1032A00080882D490968898A88424BDB0C2060435D
:1032B0002549096840188068002843D00C206043E5
:1032C000214A126880188168072088470020210160
:1032D0001E4A12688918487234E020011B490968A7
:1032E0004018407A02282DD119480078012829D1A8
:1032F0002001164909684018C08817490968898A59
:1033000088421FDB20011149096840188088124952
:103310000968498A884215DB0C2060430A4909681C
:103320004018806800280DD00C206043064A1268BF
:10333000801881680820884700202101034A12680C
:103340008918487270BD00008C0700209407002087
:1033500088070020F0FF00009007002010B500242F
:1033600000BF04E02046FFF743FC601CC4B20248E3
:103370004078A042F6DC10BD8807002010B500247C
:10338000044802F02BF9002800D000E00124204678
:1033900010BD00000304000010B5074B14781C702A
:1033A00054785C70054B1960054B18600346183360
:1033B000044C236010BD0000880700208C0700200B
:1033C000900700209407002010B50446012C09D175
:1033D000BA220C21002000F0EFF80121022004F0B5
:1033E00021FE08E000220C21104600F0E5F8002143
:1033F000022004F017FE10BD10B500240421084877
:10340000F7F79AFE552801D1012407E0042000F0C7
:10341000FFFF002801D0002400E00124204610BD59
:103420005408002010B50446012C09D1BA221C21F1
:10343000002000F0C1F80121062004F0F3FD08E0AF
:1034400000221C21104600F0B7F80021062004F0ED
:10345000E9FD10BD10B50024062000F0D9FF0028BA
:1034600001D0012400E00024204610BD10B5044620
:10347000012C09D1BA221721002000F09DF801216A
:10348000042004F0CFFD08E000221721104600F0D0
:1034900093F80021042004F0C5FD10BD002004496C
:1034A000097A002901D0012000E0002070470000C7
:1034B0005C0A002010B50446022C1CD100220D210C
:1034C000104600F079F8FDF759FC002809D0BA221F
:1034D0000B21002000F070F801210D2004F0A2FD66
:1034E00058E000220B21104600F066F800210D2064
:1034F00004F098FD4EE0032C1CD100220B21104655
:1035000000F05AF8FDF73AFC002809D0BA220D2144
:10351000002000F051F801210D2004F083FD39E076
:1035200000220D21104600F047F800210D2004F084
:1035300079FD2FE0042C0ED1BA220D21002000F0DD
:103540003BF800220B21104600F036F801210D2037
:1035500004F068FD1EE0012C0ED100220D21104662
:1035600000F02AF8BA220B21002000F025F80121F2
:103570000D2004F057FD0DE000220D21104600F053
:103580001BF800220B21104600F016F800210D2038
:1035900004F048FD10BD10B50024FCF74DFD0228D5
:1035A00001D1022406E0FCF747FD012801D10324E4
:1035B00000E00424204610BD10B5064B1B78834262
:1035C00007DD242905D224234343034C24681B1917
:1035D0005A5410BD182F0020CC07002010B5744895
:1035E0000068407903000CF037FE0B0711D325D398
:1035F0005A6D77D38DA8D30008F0B0FE6C480068F0
:103600004079401C6A4909684871CFE069494969B5
:10361000087808F01BFF664800684079401C644940
:1036200009684871624800684079401C604909682F
:103630004871BBE000F028F9002811D17F2008F084
:1036400005FF5B4800684079401C5949096848718A
:10365000574800684079401C5549096848711DE089
:10366000534800684078401C5149096848705048E8
:103670000068407803280BD300204D490968487042
:10368000AA204B4909688870032049490968C87015
:1036900008F08EFE002046490968487186E000F077
:1036A000F3F8002807D1424800684079401C40499F
:1036B0000968487103E000203D490968487108F035
:1036C00077FE73E008F04AFE394800684079401CF4
:1036D00037490968487169E0364949690978491CE0
:1036E000C8B208F0B3FE324800684079401C304947
:1036F000096848712E4800684079401C2C490968C7
:10370000487153E000F0C0F800280FD108F0F8FD30
:10371000274909688870012008F06CFE2448006879
:103720004079401C22490968487105E008F040FED4
:1037300000201F490968487138E01D4800688078FA
:1037400018280CD102201A4909680870002018496D
:1037500009684870042016490968C87011E01448C7
:1037600000684078401C1249096848701048006899
:103770004078032805D300F027F900200C49096898
:10378000487008F015FE00200949096848710DE0ED
:1037900008F00EFE002006490968487104490968CE
:1037A0004870AA2002490968887000BF00BF10BD98
:1037B000D4070020182F002010B531480068407948
:1037C000002804D001280CD0032848D11DE008F0BF
:1037D000C5FD2B4800684079401C2949096848719B
:1037E0004BE028490969087808F030FE2448006851
:1037F0004079401C22490968487121480068407995
:10380000401C1F490968487137E000F03DF8002866
:103810000CD101201A49096808700020184909686C
:103820004870042016490968C87011E014480068FF
:103830004078401C12490968487011480068407877
:10384000032805D300F0C0F800200D49096848702E
:1038500008F0AEFD00200A49096848710DE008F043
:10386000A7FD0020064909684871054909684870A4
:10387000AA2003490968887000BF00BF10BD00007E
:10388000D4070020182F002010B508F031FD0446A1
:103890001F4800680078002838D01D480068C078AC
:1038A000042833D3002C09D1002119480068C07ABC
:1038B0008200174800681430815027E014480068DF
:1038C000C07A81001248006814304058114988427B
:1038D00011D20F480068C07A81000D48006814308A
:1038E0004058401C0A490968C97A8A000849096891
:1038F000143188500AE000F067F80021044800689D
:10390000C07A82000248006814308150204610BD01
:10391000D4070020B80B000000B587B0012069462D
:103920000871084802900848039008480490084825
:1039300005900848069001A9074800F00FF807B065
:1039400000BD0000813C0100C9570100E5030200F1
:103950001914020018140200B4280020F8B5064615
:103960000F46002400253946304600F0EFF900BF2D
:1039700014E000250EE00021242060430B4A126869
:103980008018415524206043094A12688018415527
:10399000681CC5B2242DEED3601CC4B20548007863
:1039A000A042E6DC00F010F8F8BD0000CC070020D3
:1039B000D0070020182F0020012002490968087153
:1039C00070470000D407002010B500F073F9002004
:1039D00003490968087002490968C87010BD0000F1
:1039E000D407002007480068C078062808D1054899
:1039F0000068C079002803D1012002490968C87114
:103A000070470000D407002010B555480068C07802
:103A100003000CF021FC08671D1A1714110E05662F
:103A200050484068002803D04E484168002088472D
:103A300093E000F0E5F890E000F0C6F88DE000F0CB
:103A4000D1F88AE0FFF7B8FE87E0FFF7C7FD84E012
:103A500044484068002803D0424841680120884714
:103A60003F480068407C00281AD03E48C0680028C3
:103A700003D03C48C168C8208847002038490968FD
:103A80004862374800680078002804D00420344990
:103A90000968C87024E0022031490968C8701FE035
:103AA0002F480068406A401C2D49096848622C482C
:103AB0000068406A7D21C900884211D3002028494E
:103AC00009684862264800680078002804D004206D
:103AD00023490968C87003E0022021490968C870B9
:103AE0003BE000BF1F484068002803D01D484168E4
:103AF000002088471A480068407C002813D01948E5
:103B0000C068002803D01748C168C8208847002033
:103B100013490968486212480068C078401C10497F
:103B20000968C87018E00E480068406A401C0C49DB
:103B3000096848620A480068406A7D21C9008842D5
:103B40000AD3002006490968486205480068C07821
:103B5000401C03490968C87000BF00BF10BD0000C9
:103B6000D4070020182F002010B515480068C07831
:103B7000072824D0012012490968487408E0114838
:103B80008068002802D00F4988688047FFF73CFF13
:103B90000B480068C0780628F1D109480068007A0F
:103BA0000028ECD106480068C0790028E7D1044815
:103BB0000068807A0028E2D101490968487410BD84
:103BC000D4070020182F002010B5054800680078A1
:103BD000012802D1FDF7E8FE01E0F5F789FD10BDEF
:103BE000D407002010B5054800680078012802D1EC
:103BF000FEF706F901E0F6F759F910BDD4070020E9
:103C000010B51D480068807A002829D11A4800683C
:103C1000007A002803D002201749096888721648E4
:103C20000068C079002803D0012013490968887210
:103C3000114800680079012812D100200E49096856
:103C400008710D490968887207200B490968C87016
:103C50000A484068002803D0084841680020884787
:103C6000054800680078012802D1FEF7A3F901E0B9
:103C7000F6F7F6F910BD0000D4070020182F002039
:103C800010B504462146084801F0C4FC07480078F6
:103C9000002805D1002C03D032210548FCF72EFD69
:103CA0000248047010BD000001030000060100205E
:103CB00050C300000020244909684870AA20224906
:103CC0000968887000202049096848621E4909680F
:103CD00008711D49096848711B49096888711A49AA
:103CE0000968C87118490968087217490968887213
:103CF00015490968C87214490968087324201249D3
:103D0000096848731049096888730F490968C873BE
:103D100000200D49096808740B49096848740A496C
:103D20000968887408490968C874074909684861BE
:103D3000002105480068816103480068C1610248AC
:103D40000068016270470000D407002010B50A78AF
:103D50000D4B1860034628330C4C23602423534337
:103D6000044628341B190A4C23600A4C4B686360D4
:103D70008B68A360CB68E3604B6963610B69236167
:103D80000B78237010BD0000D4070020CC07002062
:103D9000D0070020182F002007480068C0780628A8
:103DA00008D105480068007A002803D101200249A3
:103DB0000968087270470000D407002010B5044657
:103DC000012C09D1BA2220210020FFF7F5FB0121A7
:103DD000084604F027F908E0002220211046FFF7EA
:103DE000EBFB0021012004F01DF910BD10B50024EB
:103DF000032000F00DFB002801D0012400E0002486
:103E0000204610BD10B50446032C0ED1BA22152150
:103E10000020FFF7D1FB002214211046FFF7CCFB56
:103E200001210E2004F0FEF839E0022C1CD1FCF731
:103E3000A5FF002809D0BA2214210020FFF7BCFBFF
:103E400001210E2004F0EEF808E0002214211046B3
:103E5000FFF7B2FB00210E2004F0E4F80022152148
:103E60001046FFF7A9FB1AE0012C0ED1BA2214214B
:103E70000020FFF7A1FB01210E2004F0D3F800225F
:103E800015211046FFF798FB09E000221521104686
:103E9000FFF792FB002214211046FFF78DFB10BDA7
:103EA00010B50024F8F756FD094988420DD3FCF7F8
:103EB000D1FF002807D1FCF72BFE012801DD0324E8
:103EC00004E0022402E0022400E00124204610BDA8
:103ED000B80B000010B50446012C09D1BA221D21EF
:103EE0000020FFF769FB0121002004F09BF808E0A7
:103EF00000221D211046FFF75FFB0021084604F059
:103F000091F810BD10B50024022000F081FA0028BD
:103F100001D0012400E00024204610BD10B5044665
:103F2000012C09D1BA221E210020FFF745FB0121F7
:103F3000092004F077F808E000221E211046FFF760
:103F40003BFB0021092004F06DF810BD70B5002482
:103F500000250026FCF798FC0546FCF7A1FC064668
:103F600002210848F7F7E8F8552800D108E0012EAB
:103F700001D1002404E0012D01D1012400E000243E
:103F8000204670BD5408002010B50446012C09D10C
:103F9000BA221F210020FFF70FFB0121082004F0A7
:103FA00041F808E000221F211046FFF705FB002121
:103FB000082004F037F810BD70B500240025FCF788
:103FC000EDFC054603211A48F7F7B6F8552806D147
:103FD00001201849088000201749088023E016486E
:103FE0000088012811D114490880FCF7F1FB7628DC
:103FF00003DA01200F49088015E0FCF7E9FB782877
:1040000011DB00200B4908800DE001200A490880DF
:10401000FCF7DEFB762803DA01200649088002E07F
:1040200000200449088003480488204670BD000031
:1040300054080020240100202601002010B5044669
:10404000012C09D1BA2221210020FFF7B5FA012164
:10405000072003F0E7FF08E0002221211046FFF7C8
:10406000ABFA0021072003F0DDFF10BD10B50024DE
:10407000FCF766FD002801D1012400E00024204661
:1040800010BD10B50446012C09D1BA22162100201A
:10409000FFF792FA0121032003F0C4FF08E0002299
:1040A00016211046FFF788FA0021032003F0BAFF1B
:1040B00010BD10B50024052000F0AAF9002801D099
:1040C000012400E00024204610BD10B50446012C58
:1040D00009D1BA2219210020FFF76EFA012105202B
:1040E00003F0A0FF3CE0022C17D1FCF747FE0028AC
:1040F00009D0BA2219210020FFF75EFA012105201C
:1041000003F090FF2CE0002219211046FFF754FA2B
:104110000021052003F086FF22E0032C17D1FCF7D5
:1041200033FE002809D0BA2219210020FFF744FAF3
:104130000121052003F076FF12E00022192110462C
:10414000FFF73AFA0021052003F06CFF08E0002297
:1041500019211046FFF730FA0021052003F062FF15
:1041600010BD000010B50024FCF71EFD01282FD162
:1041700004211948F6F7E0FF552801D1012428E071
:10418000FCF79AFB01280BD0FCF796FB022807D01E
:10419000FCF792FB032803D0FCF78EFB052801D126
:1041A000012416E0FCF788FB042801D1022410E06A
:1041B000FCF782FB062801D103240AE0FCF77CFB14
:1041C000002803D0FCF778FB072802D1002400E088
:1041D0000024204610BD00005408002010B50446FD
:1041E000012C0ED1BA221B210020FFF7E5F9002295
:1041F0001A211046FFF7E0F901210A2003F012FF0F
:104200001EE0022C0ED1BA221A210020FFF7D4F9A9
:1042100000221B211046FFF7CFF901210A2003F0ED
:1042200001FF0DE000221A211046FFF7C5F9002218
:104230001B211046FFF7C0F900210A2003F0F2FE0F
:1042400010BD10B50024FCF7A5FD022803D0FCF733
:10425000A5FE022807D1FCF76FFE012801D1012439
:1042600002E0022400E00224204610BD10B5F8F759
:104270008BFB0446204610BD10B5034B08220349B2
:10428000034800F013F910BD6D420100B81302009D
:104290007428002070B506465C488068002804D069
:1042A0005A4988688047054600E000250024A6E0BA
:1042B000564841680C20604308184088A84207D03F
:1042C000524841680C2060430818408802287DD17C
:1042D0004E4841680C2060430818806800280CD0C4
:1042E0004A494A680C216143511888688047474908
:1042F0000968E2008918487009E0444841680C20C8
:104300006043095C41480068E200801841703F4802
:104310000068E100401840783C490968E200895C87
:1043200088420FD039480068E1004018417837488A
:104330000068E2008154002034490968E2008918CD
:1043400048605AE031480068E100401841782F4841
:1043500042680C2060431018407881421FD12B48DE
:104360000068E10040184168284842680C2060431A
:104370001018808881420BD824480068E10040185A
:104380004068801921490968E2008918486034E0D2
:1043900001201E490968E200891848802DE01B4869
:1043A0000068E10040184168184842680C206043EA
:1043B0001018C08881420DD814480068E1004018E8
:1043C0004068811911480068E20000E009E08018A7
:1043D000416012E000200D490968E2008918488018
:1043E0000BE0002009490968E20089184880002193
:1043F00006480068E20080184160601C84B20348EF
:104400008089A04200DD53E770BD0000D02E00205F
:104410000146064A92898A4205DD044A1268CB00A9
:10442000D218508800E0002070470000D02E0020F5
:10443000002000BF14E00D494A680C214143511887
:10444000498801290AD10021084A1268C300D218FC
:104450005180064A1268C300D2185160411C88B2CC
:10446000024989898142E6DC70470000D02E002095
:10447000002000BF13E00C494A680C214143511849
:104480004988002909D1084A1268C300D21851800E
:10449000054A1268C300D2185160411C88B2024913
:1044A00089898142E7DC7047D02E0020F0B50446B0
:1044B0000020164DAB6069602C60AA8100BF1FE030
:1044C000124D6E680C254543755D104E3668C70069
:1044D000F61975700D4D6E680C254543755D0B4ED4
:1044E0003668C700F5550025084E3668C700F6192E
:1044F0007580064E3668C700F6197560451CA8B26F
:10450000024DAD898542DBDCF0BD0000D02E0020DD
:1045100070B505460E46002E05D031462846F3F705
:104520000FFE044600E02C46204670BD10B5FCF797
:1045300007FB00280DD107480078012809D005485D
:104540000078032805D004480078002801D1F8F746
:10455000F7FE10BDF1000020F000002008B500209B
:104560000090012269460520F9F7D8FD0549009819
:1045700088600020044908700449087004490870E4
:1045800008BD00003C280020F0000020F2000020C0
:10459000F300002008B500200090012269460520A4
:1045A000F9F7BCFD00200349087148710098886044
:1045B00008BD00003C28002070B5049C257891427D
:1045C00016DD01280AD18D4206DAFF26F61AAE4220
:1045D0000ED3EE18F5B20BE0154609E0022807D11C
:1045E000954204DD9D4203DBEE1AF5B200E00D4674
:1045F000257070BD0D4A4168516081699161C16843
:10460000D160416A5162016A1162016811604169B9
:10461000516181689160C169D16101691161816AEB
:1046200091620021024A117070470000EC2E0020B8
:10463000C807002010B5FFF7FBFEF7F7F5FF0021D4
:104640000148F6F779FE10BD6008002010B5F7F7B5
:10465000EBFFFFF70DFF09F0D9FD09F075FEFBF741
:1046600091FBFAF7C3F8FFF779FFF8F70DFCF6F7BF
:1046700069FCF9F73FF955210448F6F75DFEF8F7B4
:104680003BFAF9F7B5F8FBF73DF810BD60080020DC
:104690001CB500203149087007F010FE0020FCF71F
:1046A000F1FC0CF001F9F7F745F955212C48F6F724
:1046B00043FEF8F721FAF9F79BF8F6F73BF8F6F71F
:1046C000B9FAE12040020BF031FD00F069FAF6F78B
:1046D00039FC07F0D1FFF7F7A7FFF9F7CDFEF8F7A0
:1046E0005FFCF8F7DDFBFFF7C7FDFEF767F8FFF7A4
:1046F00013F9FFF739FAF9F7B1FDFBF76FFBFAF79A
:1047000075F8184AFF219131012009F0E9FE0022D5
:104710001146012009F028FE09F05EFD09F014FEA3
:10472000FFF738FFF9F714F900200F498871487135
:1047300008710120887048701420087007226846AC
:10474000F3F795FD0199009800F0B4FF02210120D4
:1047500000F08CFEFAF7D6FF1CBD0000050100201A
:10476000600800200090D003160100207047000070
:1047700010B50446552C03D105494869804702E02D
:1047800003490868804700200249087010BD0000F6
:10479000EC2E0020C807002010B546480078030022
:1047A0000BF05AFD0A06111B26303B46505173810F
:1047B00041484068002802D03F49486880470120AE
:1047C0003C49087000BF3C488068002804D03A4942
:1047D000886880473749087069E03748C068002812
:1047E00002D03549C868804703203249087000BFAD
:1047F00031480069002804D02F49086980472D49B5
:10480000087054E02C484069002802D02A494869C1
:10481000804700202749087049E027488069002820
:1048200002D025498869804706202249087000BFC8
:104830002148C069002804D01F49C86980471D4924
:10484000087034E000BF1B48007807280AD11A48D6
:10485000006A002802D01849086A804709201549D3
:10486000087011E01348007808280AD11248406AFD
:10487000002802D01049486A804709200D49087075
:1048800002E000200B49087000BF0A4800780028A9
:1048900008D00948806A002804D00749886A804700
:1048A0000449087003E000200249087000BF00BFFF
:1048B00010BD0000C8070020EC2E0020704700004B
:1048C00010B500200CF0ACF808F0B0FD08F004FEC4
:1048D00008F01AFE00F0BEFCF6F73CFA0220FCF7E6
:1048E000D1FB002007490870FFF73EF9FFF764F895
:1048F000FFF78AF8F6F78EF810200AF007FA00F0B2
:10490000A9FD10BD9C01002010B5012408F05CF940
:10491000012801D1052407E0F8F716F80349884279
:1049200001D2012400E00224204610BD204E0000E8
:1049300010B5062408F048F9002800D1002408F03A
:1049400049F9012803D008F045F9072800D90924BE
:10495000204610BD10B5F6F7FDF9002211460120E2
:1049600009F034FE00213B48F6F7E6FC002400BFC6
:1049700000F02AFF32217D200001FBF7BFFE00205E
:10498000354908700AE00022334801781046FEF7E6
:1049900013FE31480078401C2F4908702E480078DB
:1049A0002428F0DB00202D49087009E000212B4865
:1049B000007809F019FA29480078401C2749087046
:1049C000264800780D28F1DBFFF71EF8F5F7F8FE12
:1049D00008F04CF822480078401C2149087008462D
:1049E0000078052812D300200870FEF7FBFF1D4851
:1049F00000780A2805D300201A490870FFF7CCF97F
:104A000004E018480078401C1649087008F0E2F8E5
:104A10000128ADD908F0DEF80728A9D200200F49F7
:104A2000087008E00D48007809F0F8F90B480078A4
:104A3000401C0A490870094800780D28F2DBF6F797
:104A4000F9F855210348F6F777FCF7F753FF2046AE
:104A500010BD0000600800201F0100201D01002083
:104A60001E0100202001002010B5032408E000F002
:104A7000ABFE012000F0B2FD002801D0042400E0CC
:104A8000F5E700BF204610BD10B50020284908609A
:104A900007F014FC0120FCF7F5FAF6F74BFF55215F
:104AA0002448F6F749FCF8F727F8F8F7A1FE0BF0D1
:104AB000FBFEF5F73FFEF9F7A7FCF6F7BBF807F0AA
:104AC000E5FFF9F7D9FCF9F775FEF8F769FAFFF792
:104AD000D3FBFDF773FEFFF7CBFCFFF73FFDFEF7BF
:104AE0001BFFFFF741F800F05BF8E12040020BF0FC
:104AF0001DFBF6F727FAFBF771F9F9F777FE0E4A77
:104B0000FF219131012009F0EBFC00221146012028
:104B100009F02AFC09F060FB09F016FCF8F7EAFE40
:104B20000221012000F0A2FCFAF7ECFD10BD00000C
:104B300050000020600800200090D00370B50646A9
:104B40000D4614460E4806600E4805600E49206862
:104B500008600E49606808600D49A06808600D494A
:104B6000206908600C49E06808600C4960690860C9
:104B700005480068002802D003480068804770BDDF
:104B8000C4000020CC000020AC000020B0000020B9
:104B9000B4000020B8000020BC000020C0000020AD
:104BA00000B587B00C4801900C4802900C48039067
:104BB0000020049005900B48069000200A490860E8
:104BC00048600A490860486001AA0121C9020848F2
:104BD000FFF7B4FF07B000BDF54B0100994F01008E
:104BE000214F01004D4E010070120020680A002084
:104BF0007817002001207047F3B5C3B00446449EE7
:104C00000020009057E002E0641C761E00BF022ED8
:104C100005D32078EB28F7D160789028F4D1072EBF
:104C200000D24AE0A778FD1CB54200D945E0A81E95
:104C3000205C0002691E615C08434290042D38D953
:104C4000291FA01C0BF04AFE4299884226D11D481C
:104C50000068002804D0B91EE01C1A4A1268904768
:104C600019480068002824D0E1786846017120794D
:104C700081116846417120798106890E68468171EB
:104C8000381FC1B26846C171C279611D02A8F3F72D
:104C9000EEFA01A80C49096888470AE00020009054
:104CA00002E00098401C00900098A842F9D3002030
:104CB00000906419761B072EA5D200BF4498801B74
:104CC00045B0F0BDB8000020C0000020F7B5C0B06E
:104CD000154600260027E81DFF210131884202DD2C
:104CE000002043B0F0BDEB21684601709021417077
:104CF000281DC1B2684681700021C1704098C1B2C0
:104D0000684601710524002605E04198805D6946EA
:104D10000855641C761CAE42F7DBA11E00A80230C9
:104D20000BF0DCFD0746381269460855641C0F5528
:104D3000641C06480068002805D021466846034ADE
:104D400012689047CDE70020CBE70000B0000020BC
:104D500070B50024002500261B4840681A490968E0
:104D6000884200D170BD18484068174909688842D8
:104D700005D91548406814490968451A07E01248E2
:104D8000006811494968401A012189020D1AFF2D56
:104D900001D9FF2600E02E4600240DE00A480168F4
:104DA0000830405C0949085507480088401C8005C8
:104DB000800D05490860641CB442EFD3B1B20348CA
:104DC0000BF010FA00BFCDE770120020781600201B
:104DD00070B500251A480068002830D0194A12889A
:104DE000FF230133991A184A1268164B1B88D018F2
:104DF000134A126890470546002D20D011480088BC
:104E0000401910490880084601880F480068FFF7DC
:104E1000F3FE0446002C0DDD0A480088844209DABE
:104E200008480088021B0848006801190648006805
:104E3000F3F71DFA03480088001B0249088070BD83
:104E4000B4000020C8000020C400002038B504468B
:104E500000200090A07810280CD120792D490870EE
:104E600008460078012853D1002211462020FFF780
:104E70002DFF4DE0A078122803D120792549087232
:104E800046E0A078052803D12079224988723FE0C6
:104E9000A07802281DD120791E4948720846407A20
:104EA000012806D10090012269460420FFF70EFF79
:104EB0002EE01848407A02282AD100BFBFF34F8F56
:104EC00015481649C860BFF34F8F00BF00BF00BF31
:104ED000FDE7A07801281BD12079332803D10120D8
:104EE0000C49487005E02079352802D10020094995
:104EF0004870607907498870607A0006217A090451
:104F00000843E17909020843A1790843014948604F
:104F100038BD00005C0A00200400FA0500ED00E046
:104F200070B503460022002400251A484068194E37
:104F30003668B04201D1002070BD16484068154E59
:104F40003668B04205D913484068124E3668841B53
:104F500007E0104800680F4E7668801B0126F602B5
:104F6000341AA14201D9254600E00D4600220CE08A
:104F7000084806680830805D985406480088401C40
:104F80004005400D034E3060521CAA42F0D3284623
:104F9000D2E70000680A002070B503460022002412
:104FA00015484068144D2D68A84208D3124840683F
:104FB000114D2D68401B0125AD022C1A04E00E484E
:104FC00000680D4D6D68441BA14201D9012070BDE0
:104FD00000220CE09D5C084846680830855508387A
:104FE0008088401C8005800D034D6860521C8A42F9
:104FF000F0D30020EBE700007012002010B502484B
:10500000FFF7F8FA10BD0000A01402000021014AC9
:105010001175704740600040014600BFF020084015
:1050200000110A23584302460807000F8018C0B237
:1050300070470146002204E0501CC2B208460A38FC
:10504000C1B20A29F8DA1007000E084370470000C1
:1050500010B5044601218020F6F7F8F9607A01289E
:1050600005D14248C078102108434049C870607A91
:10507000A22805D13E48007F802108433C4908779B
:10508000607A3B49087700203A4948770846407FD4
:105090002178084337494877E07B002805D0084647
:1050A000407F20210843334948773248407FC00879
:1050B000C000A17A08432F4948770846807FF7212E
:1050C00008402C498877E078FFF7B3FF29498874B6
:1050D000A078FFF7AEFF2749C8746078FFF7A9FFF3
:1050E000244908752078002805D10846007D2179DB
:1050F000084320490875E079FFF79BFF1D49887533
:105100006079FFF796FF1B494875A079FFF791FF7B
:105110001849C875207AFFF78CFF164908760846AB
:10512000807F4006400E8877E07A002806D0084647
:10513000807F402108430F49887703E00D48807F36
:105140000C498877A07BFFF774FF0A498876607B5B
:10515000FFF76FFF0749C876207B08770846807FF6
:10516000102188430349887710BD000020040240C5
:1051700060040440404F044010B504461B48807F43
:1051800001210843194988772078FFF752FF174912
:1051900008756078FFF74DFF1449C874A078FFF7D1
:1051A00048FF1249887420780C2806DD0846407FA5
:1051B000082108430D49487709E00C48407F0B4916
:1051C00048770846007DE178084308490875074894
:1051D000807F400840000549887700BF0348807FF2
:1051E000022108400028F9D110BD0000404F0440C2
:1051F00010B500201449087616200BF053F8002152
:10520000124801761248407F8021084310494877B0
:105210000846807F012108430D49887700BF0C486C
:10522000807F022108400028F9D00948807F40088B
:1052300040000749887700BF0548807F0221084069
:105240000028F9D110BD00004060004040610040DE
:10525000404F044010B5002007490870002120206D
:10526000F6F7F4F801210548017500200449087596
:1052700015200AF0FFFF10BD0050044040610040BF
:105280004060004070B504460D46002C14D0002D3F
:1052900012D0042D10D800F013F800280CD10026ED
:1052A00008E00649885D22460121F4F75FF8A41C56
:1052B000701CC6B2AE42F4DB70BD00001C140200CC
:1052C00000200549897DC907C90F002901D00120A7
:1052D00000E00020704700000050044030B585B069
:1052E00005460C4600200390049000900190029027
:1052F000072C0BDC0120A04081B26846818101218E
:10530000C17303A90220FAF7A9FE3EE0082C01D0E0
:10531000092C0BD10120A04081B268468181012176
:10532000C17303A90120FAF799FE2EE00A2C03D0DD
:105330000B2C01D00D2C0BD10120A04081B268466E
:1053400081810121C17303A90020FAF787FE1CE0C7
:105350000C2C01D00F2C0BD10120A04081B268464B
:1053600081810121C17303A90E20FAF777FE0CE0B9
:105370000E2C0AD10120A04081B268468181012112
:10538000C17303A90C20FAF769FE00216846017079
:10539000C17041700121817000210171C1720D2124
:1053A0008172FF21017200214172F4F73FF8034935
:1053B0001520FDF7CDF805B030BD00000D500100FF
:1053C00010B500201049087515200AF053FF002180
:1053D0000E4801751520002809DB00BF00BFC2067A
:1053E000D20E012191400A4A116000BF00BF00BFE8
:1053F000084880798011032805D00648007880216C
:1054000008430449087010BD4060004040610040FE
:1054100000E100E00050044010B5F4F701F910BDC0
:1054200010B501231A4600211846F5F7CBFF0122DB
:1054300011461046F6F73CF8F6F728F803480BF04B
:1054400025FA02480249086010BD00000090D00310
:105450004C07002000BF04480069042108430249AA
:10546000086130BF00BF704700ED00E0F3B585B0C4
:105470000546002400270026002003900490EEB289
:105480002804070E0F2F54DA082E52DA002009E004
:105490000C214143284A515AA94201D1044603E054
:1054A000411CC8B21728F3D300BF0120B04086B218
:1054B0000C20604320494018C3780C2060434018FA
:1054C0008278F8B231460190FAF76CFE6846868120
:1054D000012181730021C17302214174F8B203A933
:1054E000FAF7BCFD0C216143134A8918C888FBF701
:1054F000EFFE0C20604310494018C18868460181C6
:1055000069460698887202A8FBF7FCFD0C226243EC
:10551000094BD21891680C226243D218042010560D
:10552000FDF716F80C216143034A8918C888FBF778
:1055300053FE07B0F0BD000038160200FEB5054668
:105540000C460020C0430290EFB22804060E0F2E36
:1055500042DA082F40DA0120B840694608808020EE
:105560002040002816D101208870A007800F022853
:1055700001D1487109E0A007800F012802D16946D6
:10558000487102E0002069464871F0B26946FAF7B6
:1055900065FD1FE00020694688700E20204000282D
:1055A00000D000BF10202040002802D169460871B9
:1055B00002E0012069460871E007C00F002802D10F
:1055C0006946887102E0012069468871F0B2694637
:1055D000FAF744FD002002900298FEBD30B5014666
:1055E000CAB20C04230E00200F2B0FDA082A0DDAA2
:1055F00001249440A2B2064C03252D026419E45CF8
:105600001440002C01D0012000E0002030BD00003B
:1056100000000440F8B504460F460020C043009047
:10562000E6B22004050E0F2D11DA082E0FDA012044
:10563000B04086B2002F04D1E8B23146FAF70AFE34
:1056400003E0E8B23146FAF715FE0020009000981A
:10565000F8BD00001649897F01221143144A917751
:1056600000BF1349897F022211400029F9D0104957
:10567000897C81700E49C97C41700D49097D01709A
:105680000B498A7D8271497D01710949CA7D427148
:105690000A7EC271897F49084900054A917700BF97
:1056A0000349897F022211400029F9D17047000087
:1056B000404F044003B585B0002001900290039054
:1056C0000490002168464173817E01A8C17068463C
:1056D000417E01A881706846017E4171002101A8C8
:1056E0000171082168460171817D01A8C171684678
:1056F000C17D4172417D01A881716846017D01A88B
:105700000172002168468173C17301A881730C2165
:1057100041734121684601740021C17401A8FFF75B
:1057200097FC1A200449888204491620FCF710FFD0
:1057300000F006F807B000BD204F0440D909020070
:1057400010B5FFF755FD10BD70B504460D46601E3F
:105750000D49884200D90124002C00D101244020A9
:105760000A490870084600786043094948610321E6
:10577000081F0AF0AFFD0020054988610720086175
:105780000448056070BD0000FFFFFF0078010020A5
:1057900000E000E0740100200020C043002809DB85
:1057A000C206D20E01219140054A1160BFF34F8F0E
:1057B000BFF36F8F00BF0020024908618861704706
:1057C00080E100E000E000E010B50AF029FD10BD26
:1057D0001A20084908722B2048723C2088724D20FC
:1057E000C8727F20044909680860AC2003494870EA
:1057F00070470000000402407C01002000100240BD
:1058000010B51C480078012812D11B480078642884
:1058100009DB0220194948710871002016490870F7
:105820001449087004E014480078401C12490870BC
:105830001348007801281CD112480078012804D1AF
:10584000002010490870104908700F48007832286D
:105850000ADBF7F799F900210C48F5F727FD5521E8
:105860000B48F5F769FD04E007480078401C06493D
:10587000087010BD19070020180700200807002035
:1058800012070020140700201307002054080020EE
:1058900060080020F8B504460D460027002000905F
:1058A00003200003204000130090102C04D0122C81
:1058B00002D01148844217D122202840222806D144
:1058C00027073F0F39460098F4F720FF06461220BD
:1058D000284012280ED12007000F471C3946009897
:1058E000F4F714FF064605E02107090F0098F4F7C6
:1058F0000DFF06463046F8BD10100000F8B504460E
:105900000D46002600270120000320400713102C1D
:1059100004D0122C02D00F48844215D122202840F6
:10592000222805D12607360F31463846FAF78EF879
:105930001220284012280CD12007000F461C3146A7
:105940003846FAF783F804E02107090F3846FAF7DA
:105950007DF8F8BD10100000FFB58BB01C4600208C
:105960000790069005903848049010210B98084045
:10597000002801D0022707E040210B9808400028AA
:1059800001D0012700E00027002C04D014980470F7
:105990000120089001E010200890002548E0002C2C
:1059A00008D025466000294A115A0C98F2F7C8FB26
:1059B000079006E06800254A115A0C98F2F7C0FBE0
:1059C00007903E4630E0711C0798F2F7B9FB40089B
:1059D00006900D98F2F70AFD03900D9A0699881A21
:1059E000F2F704FD18490190F2F785FC0290039943
:1059F000F2F7BEFC05900598F2F7FFFC4900490854
:105A0000039102900498F2F7F8FC490049080191CB
:105A10000090039B029AF2F705FD03D20A950996BE
:105A200005980490701CC6B27F2ECCDD681CC5B2F0
:105A300008988542B3DB14990A980870149909985C
:105A4000487004980FB0F0BD0000C8424C17020027
:105A50000246412A2ED010DC212A2AD006DC102A48
:105A600045D0122A4BD0202A59D11CE0222A26D018
:105A7000232A2AD0402A52D116E081235B01D01A72
:105A80009A4228D008DC422A1AD0432A1ED0254840
:105A90001018002843D13AE0012822D020281BD03A
:105AA00021283CD11EE000BF1F4803890B4303811E
:105AB00036E000BF1C4843890B43438130E000BF00
:105AC000194883890B4383812AE000BF1648C389A4
:105AD0000B43C38124E000BF144883880B438380B9
:105AE0001EE000BF1148C3880B43C38018E00E4876
:105AF00043890B43438103890B43038110E00A4828
:105B0000C3890B43C38183890B43838108E0074822
:105B1000C3880B43C38083880B43838000E000BFAE
:105B200000BF7047F0EFFFFF001104400014044075
:105B3000F0B505460E46412D30D010DC212D2CD07D
:105B400006DC102D51D0122D56D0202D62D11CE034
:105B5000222D2AD0232D30D0402D5BD116E081217B
:105B60004901681A8D4230D008DC422D1ED0432DE9
:105B700024D02A48281800284CD144E001282CD0F1
:105B8000202823D0212845D128E000BF244F388881
:105B9000314600F049F804463DE000BF204F7888C8
:105BA000314600F041F8044635E000BF1C4FB8888C
:105BB000314600F039F804462DE000BF184FF88850
:105BC000314600F031F8044625E000BF154F388813
:105BD000314600F029F804461DE000BF114F7888D7
:105BE000314600F021F8044615E00D4F7888314623
:105BF00000F01AF804460EE0094FF888314600F02C
:105C000013F8044607E0074F7888314600F00CF897
:105C1000044600E000BF00BF2046F0BDF0EFFFFFEC
:105C200000110440001404400246002013460B40BB
:105C3000002B01D0012000E000207047FFB581B0AB
:105C40000E461746012F07D1F748407D0009000195
:105C5000C01DF549487505E0F348407D0009000185
:105C6000F1494875049801287ED10A210198F2F77C
:105C700067FA0546ED48445DE007C00F002807D0ED
:105C8000E948007C00090001C01DE749087405E0EF
:105C9000E548007C00090001E34908740220204027
:105CA000002807D0E048C07BF02188437030DE49EF
:105CB000C87305E0DC48C07BF0218843DA49C8732B
:105CC00004202040002807D0D748807C000900012C
:105CD000C01DD549887405E0D348807C00090001C7
:105CE000D149887408202040002807D0CE48407C45
:105CF000F02188437030CC49487405E0CA48407CA4
:105D0000F0218843C849487410202040002807D05B
:105D1000C548407C00090001C01DC349487405E026
:105D2000C148407C00090001BF4948742020204040
:105D3000002807D0BC48007CF02188437030BA4965
:105D4000087405E0B848007CF0218843B64908741F
:105D500040202040002808D0B348807CF0218843B0
:105D60007030B149887406E08BE0AF48807CF02148
:105D70008843AD4988740A210198F2F7E1F90D468C
:105D8000AA48445DE007C00F002807D0A648807BE2
:105D9000F02188437030A449887305E0A248807BD5
:105DA000F0218843A049887302202040002807D0B2
:105DB0009D48807B00090001C01D9B49887305E058
:105DC0009948807B0009000197498873042020408E
:105DD000002807D09448007DF02188437030924914
:105DE000087505E09048007DF02188438E490875CC
:105DF00008202040002807D08B48007D00090001C2
:105E0000C01D8949087505E08748007D000900012B
:105E10008549087510202040002807D08248C07CA2
:105E2000F021884370308049C87405E07E48C07C0A
:105E3000F02188437C49C87420202040002807D0E6
:105E40007948C07B00090001C01D7749C87305E08F
:105E50007548C07B000900017349C8734020204089
:105E6000002807D07048C07C00090001C01D6E49A1
:105E7000C87454E06C48C07C000900016A49C874C9
:105E80004DE06948007C0009000167490874084634
:105E9000C07BF02188436449C8730846807C0009B0
:105EA000000188740846407CF02188435E494874AC
:105EB0000846407C0009000148740846007CF02137
:105EC0008843594908740846807CF0218843564924
:105ED00088740846807BF0218843534988730846BC
:105EE000807B0009000188730846007DF02188430B
:105EF0004D4908750846007D0009000108750846EF
:105F0000C07CF02188434849C8740846C07B00091A
:105F10000001C8730846C07C00090001C8740A98D3
:105F200001287DD10A213046F2F70AF905463F489B
:105F3000445DE007C00F002807D03B48407B0009C4
:105F40000001C01D3849487305E03748407B00090F
:105F500000013549487302202040002807D032480C
:105F6000007BF021884370302F49087305E02E48EC
:105F7000007BF02188432C4908730420204000282E
:105F800007D02948807DF0218843703026498875E4
:105F900005E02548807DF021884323498875082045
:105FA0002040002807D02048807D00090001C01D46
:105FB0001D49887505E01C48807D000900011A49CB
:105FC000887510202040002807D01748407DF02118
:105FD000884370301449487505E01348407DF0212E
:105FE00088431149487520202040002807D00E48DA
:105FF000407BF021884370300B49487305E00A4824
:10600000407BF02188430849487340202040002805
:106010000ED00548C07D00090001C01D024900E006
:1060200092E0C8750AE000004C2600208C110200A6
:106030006D48C07D000900016B49C8750A213046D2
:10604000F2F77EF80D466948445DE007C00F00286E
:1060500007D06548C07AF021884370306249C87221
:1060600005E06148C07AF02188435F49C872022088
:106070002040002807D05C48C07A00090001C01DFC
:106080005949C87205E05848C07A000900015649CC
:10609000C87204202040002807D05348407E0009E1
:1060A0000001C01D5049487605E04F48407E000978
:1060B00000014D49487608202040002807D04A4872
:1060C000007EF021884370304749087605E0464855
:1060D000007EF021884344490876102020400028A3
:1060E00007D04148007E00090001C01D3E490876E6
:1060F00005E03D48007E000900013B49087620206C
:106100002040002807D03848007B00090001C01D4E
:106110003549087305E03448007B00090001324925
:10612000087340202040002807D02F48C07DF02170
:10613000884370302C49C87554E02B48C07DF0214D
:1061400088432949C8754DE02748407B0009000174
:10615000254948730846007BF0218843224908738B
:106160000846807DF02188431F4988750846807D58
:106170000009000188750846407DF02188431A49CE
:1061800048750846407BF021884317494873084604
:10619000C07D00090001C8750846C07AF021884317
:1061A0001149C8720846C07A00090001C872084641
:1061B000407E0009000148760846007EF0218843B1
:1061C000094908760846007E00090001087608465D
:1061D000007B0009000108730846C07DF021884358
:1061E0000149C87505B0F0BD4C2600208C11020095
:1061F000FFB581B00E461746019801287ED104985C
:10620000002828D1FB480078012824D0F6F7A2FB0B
:10621000F94988421FD3FAF7B1FD00280DD0F7489D
:10622000807DF02188437030F44988750846C07C31
:1062300000090001C01DC8741AE0F048807DF021FB
:1062400088431030ED4988750846C07C000900017C
:10625000401CC8740CE0E948807DF0218843703010
:10626000E64988750846C07C00090001C01DC87455
:10627000E248C07CF02188437030E049C874084689
:10628000007EF02188437030DC4908760846807D26
:1062900000090001401C88750846407DF0218843B4
:1062A0001030D64948750846407D00090001401C61
:1062B00048750846007DF02188431030CF490875A5
:1062C0000846007D00090001401C0875330009F0F4
:1062D000C3FF062E261E140C042FC848007D00099B
:1062E0000001C01DC549087500BFC448007DF021EC
:1062F00088437030C149087500BF00E0AFE1BF4876
:10630000407D00090001C01DBC49487500BFBB4865
:10631000407DF02188437030B849487500BFB748C8
:10632000807D00090001C01DB449887500BF00E0F0
:1063300000BF00BF049800285ED1AE480078012855
:106340005AD0F6F707FBAC49884255D3AB48C07F1B
:10635000F0218843A949C8770846807F00090001D9
:1063600088770846407FF0218843A449487708464B
:10637000007FF0218843A14908770846C07DF021BD
:1063800088439E49C8750846C07F00090001C87748
:106390000846807FF0218843984988770846407FE7
:1063A00000090001C01D48770846807EF02188431F
:1063B000924988760846807E000900018876084662
:1063C000407E0009000148760846007E0009000171
:1063D00008760846007F0009000108770846C07E5D
:1063E000F02188438549C8760846407EF0218843DD
:1063F000703082494876B8E164213846F1F7A0FE52
:106400000546012D07D17D48C07FF02188437030BB
:106410007A49C87705E07948C07FF02188437749F9
:10642000C8770A213846F1F78BFE0A210090F1F770
:1064300087FE0D46642F02D37148445D01E0714828
:10644000445DE007C00F002807D06C48807F00093A
:106450000001C01D6949887705E06848807F000910
:1064600000016649887702202040002807D0634851
:10647000407FF021884370306049487705E05F48ED
:10648000407FF02188435D49487704202040002860
:1064900007D05A48007FF021884370305749087769
:1064A00005E05648007FF0218843544908770820CA
:1064B0002040002807D05148C07DF021884370302B
:1064C0004E49C87505E04D48C07DF02188434B49D1
:1064D000C87510202040002807D04848C07F000918
:1064E0000001C01D4549C87705E04448C07F000948
:1064F00000014249C87720202040002807D03F48AB
:10650000807FF021884370303C49887705E03B4824
:10651000807FF02188433949887740202040002837
:1065200007D03648407F00090001C01D3349487735
:1065300005E03248407F00090001304948770A21D0
:106540003846F1F7FDFD0D462D48445DE007C00FCC
:10655000002807D02948807EF021884370302749E1
:10656000887605E02548807EF02188432349887697
:1065700002202040002807D02048807E000900012A
:10658000C01D1E49887605E01C48807E0009000178
:106590001A49887604202040002807D01748407EFA
:1065A00000090001C01D1549487605E01348407EEA
:1065B000000900011149487608202040002807D032
:1065C0000E48007E00090001C01D0C49087605E058
:1065D0000A48007E00090001084908761020204082
:1065E000002811D00548007F00090001C01D0349A3
:1065F00008770FE005010020B80B000020270020DD
:106600008C1102009F1102005948007F000900010F
:106610005749087720202040002807D05448C07EE2
:10662000F021884370305249C87605E05048C07E5A
:10663000F02188434E49C87640202040002807D0EA
:106640004B48407EF02188437030494948768CE0C1
:106650004748407EF02188434549487685E04448D4
:10666000807D00090001424988750846407DF0217F
:1066700088433F4948750846407D00090001487538
:106680000846007DF0218843394908750846007D99
:106690000009000108750846C07C00090001C874A3
:1066A0000846807DF0218843314988750846C07CC2
:1066B000F02188432E49C8740846007EF0218843A3
:1066C0002B4908760846C07FF02188432849C877BF
:1066D0000846807F0009000188770846407FF02146
:1066E0008843234948770846007FF02188432049A2
:1066F00008770846C07DF02188431D49C8750846C3
:10670000C07F00090001C8770846807FF0218843D8
:10671000174988770846407F0009000148770846F6
:10672000807EF0218843124988760846807E0009E1
:10673000000188760846407E000900014876084638
:10674000007E0009000108760846007F000900016C
:1067500008770846C07EF02188430549C876084678
:10676000407EF02188430249487605B0F0BD000024
:106770002027002010B50146002200200A0EFE4B03
:10678000985CC307DB0F002B07D0FC4BDB7FF024AA
:10679000A3437033F94CE37705E0F84BDB7FF0243B
:1067A000A343F64CE37702230340002B07D0F34BBF
:1067B000DB7F1B091B01DB1DF04CE37705E0EF4B92
:1067C000DB7F1B091B01ED4CE37704230340002B07
:1067D00007D0EA4B9B7F1B091B01DB1DE74CA3770E
:1067E00005E0E64B9B7F1B091B01E44CA3770823C4
:1067F0000340002B09D0E14B20335B781B091B01C0
:10680000DB1DDE4C2034637007E0DC4B20335B780B
:106810001B091B01D94C2034637010230340002B4B
:1068200009D0D64B20331B78F024A3437033D34CCC
:106830002034237007E0D14B20331B78F024A3438E
:10684000CE4C2034237020230340002B09D0CB4BA7
:1068500020331B781B091B01DB1DC84C203423701F
:1068600007E0C64B20331B781B091B01C34C2034A7
:10687000237040230340002B07D0C04B9B7FF024A4
:10688000A3437033BD4CA37705E0BC4B9B7FF02442
:10689000A343BA4CA377FF231B040B401A0CB64B3F
:1068A000985CC307DB0F002B07D0B44B1B7F1B0981
:1068B0001B01DB1DB14C237705E0B04B1B7F1B098F
:1068C0001B01AE4C237702230340002B07D0AB4BB8
:1068D000DB7EF024A3437033A84CE37605E0A74B9E
:1068E000DB7EF024A343A54CE37604230340002B76
:1068F00007D0A24B9B7EF024A34370339F4CA3761A
:1069000005E09E4B9B7EF024A3439C4CA37608237A
:106910000340002B07D0994B5B7FF024A3437033D7
:10692000964C637705E0954B5B7FF024A343934C33
:10693000637710230340002B07D0904B5B7F1B092C
:106940001B01DB1D8D4C637705E08C4B5B7F1B09C6
:106950001B018A4C637720230340002B07D0874B11
:106960001B7FF024A3437033844C237705E0834BD3
:106970001B7FF024A343814C237740230340002B4B
:1069800007D07E4BDB7E1B091B01DB1D7B4CE376B6
:1069900005E07A4BDB7E1B091B01784CE376FF2375
:1069A0001B020B401A0A744B985CC307DB0F002BC9
:1069B00007D0724B1B7EF024A34370336F4C2376B9
:1069C00005E06E4B1B7EF024A3436C4C2376022320
:1069D0000340002B07D0694B1B7E1B091B01DB1DED
:1069E000664C237605E0654B1B7E1B091B01634C3F
:1069F000237604230340002B07D0604BDB7D1B096B
:106A00001B01DB1D5D4CE37505E05C4BDB7D1B0969
:106A10001B015A4CE37508230340002B07D0574B4A
:106A20009B7E1B091B01DB1D544CA37605E0534BD9
:106A30009B7E1B091B01514CA37610230340002BA6
:106A400007D04E4B5B7EF024A34370334B4C6376F0
:106A500005E04A4B5B7EF024A343484C6376202339
:106A60000340002B07D0454B5B7E1B091B01DB1D40
:106A7000424C637605E0414B5B7E1B091B013F4C9A
:106A8000637640230340002B07D03C4BDB7DF02492
:106A9000A3437033394CE37505E0384BDB7DF024BC
:106AA000A343364CE375CAB2334B985CC307DB0F84
:106AB000002B07D0314B1B7DF024A34370332F4CA8
:106AC000237505E02D4B1B7DF024A3432B4C237530
:106AD00002230340002B07D0284B1B7D1B091B0101
:106AE000DB1D264C237505E0244B1B7D1B091B0178
:106AF000224C237504230340002B07D01F4BDB7C63
:106B00001B091B01DB1D1D4CE37405E01B4BDB7CEB
:106B10001B091B01194CE37408230340002B07D009
:106B2000164B9B7CF024A3437033144CA37405E0F4
:106B3000124B9B7CF024A343104CA37410230340FE
:106B4000002B07D00D4B5B7DF024A34370330B4C1F
:106B5000637505E0094B5B7DF024A343074C637527
:106B600020230340002B0BD0044B5B7D1B091B0132
:106B7000DB1D024C637509E08C1102000027002028
:106B80000C4B5B7D1B091B010A4C637540230340C2
:106B9000002B07D0074BDB7CF024A3437033054C5C
:106BA000E37405E0034BDB7CF024A343014CE37466
:106BB00010BD00000027002000B501287ED1FE4A4C
:106BC000D278F0239A437032FB4BDA701A4612796E
:106BD00012091201D21D1A711A461279F0239A4332
:106BE0007032F54B1A711A46527912091201D21DF0
:106BF0005A711A465279F0239A437032EE4B5A7109
:106C00001A46D27912091201D21DDA711A46D279C6
:106C1000F0239A437032E84BDA711A46527A12091D
:106C20001201D21D5A721A46527AF0239A437032D8
:106C3000E14B5A721A46927AF0239A437032DE4B35
:106C40009A721A469278F0239A437032DA4B9A700D
:106C50001A46D27A12091201D21DDA721A465278F5
:106C600012091201D21D5A701A46D27AF0239A43A1
:106C70007032D14BDA721A46203AD27FF0239A430F
:106C80007032CD4B203BDA77CB4A127B12091201CE
:106C9000D21D20331A731A46203A927F120912012C
:106CA000D21D203B9A77C44A127BF0239A4370325C
:106CB000C14B1A731A46203A127F00E0F2E1F0232A
:106CC0009A437032BC4B203B1A77BB4A527B120965
:106CD0001201D21D20335A731A46203AD27E12096D
:106CE0001201D21D203BDA76B44AD278F0239A43BF
:106CF0007032B24BDA701A46127B12091201D21DA1
:106D00001A731A46127912091201D21D1A711A4603
:106D1000927AF0239A437032A84B9A721A461279EB
:106D2000F0239A437032A54B1A711A465279120910
:106D30001201D21D5A711A46927912091201D21DFE
:106D40009A711A46127A12091201D21D1A721A4643
:106D5000127AF0239A437032984B1A721A46527A7A
:106D600012091201D21D5A72934A92791209120124
:106D7000521C914B9A711A469279F0239A43103221
:106D80008D4B9A711A46127A12091201521C1A720C
:106D90001A46127AF0239A431032874B1A721A4617
:106DA000927A12091201521C9A721A46D27812096A
:106DB0001201521CDA701A46927812091201521C02
:106DC0009A701A465278F0239A4310327A4B5A70CE
:106DD0001A461278F0239A431032774B1A701A46EB
:106DE000127812091201521C1A701A46203AD27FE8
:106DF00012091201521C203BDA771A46927FF023C7
:106E00009A4310326C4B203B9A771A46527FF023FC
:106E10009A431032684B203B5A771A46527F120928
:106E20001201521C5A771A46127F12091201521C83
:106E30001A771A46D27EF0239A4310325E4B203BDB
:106E4000DA761A46927EF0239A4310325A4B203B50
:106E50009A765A4A127BF0239A431032574B1A7390
:106E60001A46D27AF0239A431032544BDA721A46F9
:106E7000D27A12091201521CDA721A46927A120957
:106E80001201521C9A721A46527AF0239A43103217
:106E90004A4B5A721A465279F0239A431032474BA2
:106EA0005A711A46D279F0239A431032434BDA7161
:106EB0000B0009F0D1F919F3E9DFD5CBC1B7ADA3C8
:106EC000998F87786E645A50463E362E261E160ECF
:106ED000F5003A4AD279F0239A437032374BDA718F
:106EE00000BF364A5279F0239A437032334B5A71BD
:106EF00000BF324A527AF0239A4370322F4B5A72B3
:106F000000BF2E4A927A12091201D21D2B4B9A729F
:106F100000BF2A4AD27A12091201D21D274BDA7217
:106F200000BF264AD27AF0239A437032234BDA729A
:106F300000BF224A127BF0239A4370321F4B1A7310
:106F400000BF1D4A203A927EF0239A4370321A4BBA
:106F5000203B9A7600BF184A203AD27EF0239A430B
:106F60007032154B203BDA7600BF134A203A127F6D
:106F700012091201D21D104B203B1A7700BF0E4A96
:106F8000203A527F12091201D21D0B4B203B5A7737
:106F900000BF094A203A527FF0239A437032064BD1
:106FA000203B5A7700BF044A203A927FF0239A434D
:106FB0007032014B203B03E06C260020402700206C
:106FC0009A7700BFDC4AD27F12091201D21DDA4B38
:106FD000DA7700BFD84A2032127812091201D21D86
:106FE000D54B20331A7000BFD34A20321278F023D9
:106FF0009A437032D04B20331A7000BFCE4A2032F1
:107000005278F0239A437032CB4B20335A7000BF32
:10701000C94A2032927812091201D21DC64B203380
:107020009A7000BFC44A2032D27812091201D21DD0
:10703000C14B2033DA7000BFBF4A2032927A120966
:107040001201D21DBC4B20339A7200BFBA4A2032C3
:10705000127AF0239A437032B74B20331A7200BF72
:10706000B54A2032127A12091201D21DB24B2033D6
:107070001A7200BFB04A20329279F0239A437032DC
:10708000AD4B20339A7100BFAB4A2032927912097E
:107090001201D21DA84B20339A7100BF01E0FFE717
:1070A00000BF47E1A44A2032D278F0239A43A24B92
:1070B0002033DA701A461279120912011A711A462F
:1070C0001279F0239A439C4B20331A711A46527955
:1070D000120912015A711A465279F0239A43964BBB
:1070E00020335A711A46D27912091201DA711A46FE
:1070F000D279F0239A43904B2033DA711A46527AB0
:10710000120912015A721A46527AF0239A438A4B94
:1071100020335A721A46927AF0239A43864B2033D0
:107120009A721A469278F0239A43834B20339A70CE
:107130001A46D27A12091201DA721A4652781209E4
:1071400012015A701A46D27AF0239A437A4B2033AE
:10715000DA72794AD27FF0239A43774BDA771A466C
:107160002032127B1209120120331A73724A927F65
:1071700012091201203B9A771A462032127BF02323
:107180009A436D4B20331A736B4A127FF0239A4354
:10719000694B1A771A462032527B120912012033AA
:1071A0005A73654AD27E12091201203BDA76634A8D
:1071B000D278F0239A43614BDA701A46127B120997
:1071C00012011A731A461279120912011A711A461B
:1071D000927AF0239A43594B9A721A461279F02305
:1071E0009A43564B1A711A465279120912015A7172
:1071F0001A469279120912019A711A46127A1209E4
:1072000012011A721A46127AF0239A434B4B1A72E1
:107210001A46527A120912015A72474A203292795A
:1072200012091201444B20339A711A469279F023C5
:107230009A43414B20339A711A46127A120912016D
:107240001A721A46127AF0239A433B4B20331A7271
:107250001A46927A120912019A721A46D2781209C3
:107260001201DA701A469278120912019A701A46BF
:107270005278F0239A43304B20335A701A461278D2
:10728000F0239A432C4B20331A701A4612781209B5
:1072900012011A70284AD27F12091201203BDA77B4
:1072A0001A46927FF0239A43234B9A771A46527FCD
:1072B000F0239A43204B5A771A46527F1209120143
:1072C0005A771A46127F120912011A771A46D27E8D
:1072D000F0239A43184BDA761A46927EF0239A43AB
:1072E000154B9A76154A127BF0239A43134B1A7367
:1072F0001A46D27AF0239A43104BDA721A46D27A9F
:1073000012091201DA721A46927A120912019A725D
:107310001A46527AF0239A43084B5A721A46527907
:10732000F0239A43054B5A711A46D279F0239A43B7
:10733000024BDA7100BD00004C26002040270020DF
:10734000F7B582B006461746002500200190002EB2
:107350007ED1F9F7EFFB05285FD1F9F70FFD002883
:107360000DD0FA484079F02188437030F7494871D0
:107370000846807800090001C01D88700AE0F348C3
:107380004079F0218843F149487108468078000926
:1073900000018870ED48C07900090001EB49C8710F
:1073A0000846807900090001887108464079000983
:1073B000000148710846007AF0218843E3490872C9
:1073C0000846007A0009000108720846C079F021D9
:1073D0008843DE49C8710846C07800090001C870BA
:1073E00008468078F0218843D8498870084640785C
:1073F000F0218843D54948700846407800090001CB
:107400004870084600790009000108710846C078F4
:10741000F0218843CD49C87029E2CC484079F02159
:1074200088437030C94948710846807800090001D6
:10743000C01D88700846C07900090001C87108465F
:10744000807900090001887108464079000900E050
:1074500034E0000148710846007AF0218843BB49B6
:1074600008720846007A0009000108720846C079CF
:10747000F0218843B549C8710846C0780009000169
:10748000C87008468078F0218843B0498870084663
:107490004078F0218843AD4948700846407800099B
:1074A000000148700846007900090001087108468B
:1074B000C078F0218843A549C870ADE7012E5FD19F
:1074C000F9F75CFC00280DD0A0484079F0218843F2
:1074D00070309E4948710846807800090001C01D3F
:1074E00088700AE099484079F021884397494871AB
:1074F000084680780009000188709448C079000926
:1075000000019249C871084680790009000188711C
:10751000084640790009000148710846007AF021C8
:1075200088438A4908720846007A000900010872F7
:107530000846C079F02188438449C8710846C0785C
:1075400000090001C87008468078F02188437F490F
:10755000887008464078F02188437C494870084686
:1075600040780009000148700846007900090001D0
:1075700008710846C078F02188437449C870DAE37E
:10758000022E7DD1F9F7D6FA05287AD1F9F7F6FB64
:10759000002877D0012F76D10A210398F0F7D0FD8B
:1075A0000546F9F707FB002802D16948445D01E070
:1075B0006848445DE007C00F002807D06348C079E1
:1075C00000090001C01D6149C87105E05F48C0792C
:1075D000000900015D49C87102202040002807D041
:1075E0005A48807900090001C01D5849887105E09A
:1075F00056488079000900015449887104202040D0
:10760000002807D05148407900090001C01D4F49AA
:10761000487105E04D484079000900014B49487127
:1076200008202040002807D04848007AF0218843ED
:1076300070304649087205E04448007AF0218843DA
:107640004249087210202040002807D03F48007AA5
:1076500000090001C01D3D49087205E03B48007A61
:1076600000090001394908722020204000280BD071
:107670003648C079F021884370303449C87109E038
:10768000AEE242E1F4E0A4E03048C079F021884362
:107690002E49C87140202040002807D02B4840794F
:1076A000F021884370302949487105E02748407926
:1076B000F0218843254948710A210398F0F740FDDD
:1076C0000D462348445DE007C00F002807D01F483F
:1076D000C07800090001C01D1C49C87005E01B48A6
:1076E000C078000900011949C87002202040002814
:1076F00007D016488078F02188437030134988708D
:1077000005E012488078F0218843104988700420F1
:107710002040002807D00D484078F0218843703081
:107720000A49487005E009484078F0218843074934
:1077300048700820204000280ED0044840780009F6
:107740000001C01D014948700CE000008C2600209B
:107750008C1102009F110200FE48407800090001D0
:10776000FC49487010202040002807D0F9480079D3
:1077700000090001C01DF749087105E0F5480079CE
:1077800000090001F349087120202040002807D09B
:10779000F048C078F02188437030EE49C87005E0A9
:1077A000EC48C078F0218843EA49C8704020204066
:1077B000002807D0E748807800090001C01DE5498E
:1077C0008870B8E2E348807800090001E1498870D8
:1077D000B1E2E0484079F02188437030DD494871DA
:1077E0000846807800090001C01D88700846C079ED
:1077F00000090001C87108468079000900018871FC
:10780000084640790009000148710846007AF021D5
:107810008843D04908720846007A000900010872BE
:107820000846C079F0218843CA49C8710846C07823
:1078300000090001C87008468078F0218843C549D6
:10784000887008464078F0218843C249487008464D
:1078500040780009000148700846007900090001DD
:1078600008710846C078F0218843BA49C87062E2BE
:10787000B8484079F0218843B64948710846807875
:107880000009000188700846C07900090001C8712C
:10789000084680790009000188710846407900098E
:1078A000000148710846007AF0218843A94908720E
:1078B0000846007A0009000108720846C079F021E4
:1078C0008843A449C8710846C07800090001C870FF
:1078D00008468078F02188439E49887008464078A1
:1078E000F02188439B494870084640780009000110
:1078F0004870084600790009000108710846C07800
:10790000F02188439349C87015E2012F73D10A21F1
:107910000398F0F715FC0546F9F74CF9002802D159
:107920008D48445D01E08D48445DE007C00F0028AC
:1079300007D08848C07900090001C01D8549C87179
:1079400005E08448C079000900018249C87102201D
:107950002040002807D07F48807900090001C01D21
:107960007C49887105E07B488079000900017949EC
:10797000887104202040002807D07648407900090B
:107980000001C01D7349487105E072484079000943
:1079900000017049487108202040002807D06D4838
:1079A000007AF021884370306A49087205E069481E
:1079B000007AF0218843674908721020204000288F
:1079C00007D06448007A00090001C01D61490872AF
:1079D00005E06048007A000900015E490872202035
:1079E0002040002808D05B48C079F02188437030DF
:1079F0005849C87106E09DE05648C079F021884397
:107A00005449C87140202040002807D0514840798F
:107A1000F021884370304F49487105E04D48407966
:107A2000F02188434B4948710A210398F0F788FBFD
:107A30000D464948445DE007C00F002807D045487F
:107A4000C07800090001C01D4249C87005E04148E6
:107A5000C078000900013F49C8700220204000287A
:107A600007D03C488078F0218843703039498870CD
:107A700005E038488078F021884336498870042032
:107A80002040002807D033484078F02188437030E8
:107A90003049487005E02F484078F02188432D494F
:107AA000487008202040002807D02A484078000964
:107AB0000001C01D2749487005E0264840780009AC
:107AC00000012449487010202040002807D0214898
:107AD000007900090001C01D1E49087105E01D481C
:107AE0000079000900011B4908712020204000286E
:107AF00007D01848C078F021884370301549C87005
:107B000005E01448C078F02188431249C87040202D
:107B10002040002807D00F48807800090001C01DD0
:107B20000C49887007E10B48807800090001094979
:107B3000887000E107484079F0218843703005499A
:107B400048710846807800090001C01D8870084609
:107B5000C07905E08C2600208C1102009F110200E4
:107B600000090001C8710846807900090001887188
:107B7000084640790009000148710846007AF02162
:107B800088436E4908720846007A000900010872AD
:107B90000846C079F02188436849C8710846C07812
:107BA00000090001C87008468078F02188436349C5
:107BB000887008464078F02188436049487008463C
:107BC000407800090001487008460079000900016A
:107BD00008710846C078F02188435849C870AAE067
:107BE000032E9FD1F9F7CAF8002858D0534840799E
:107BF000F021884370305149487108468078000967
:107C00000001C01D88700846C07900090001C01D30
:107C1000C8710846807900090001C01D88710846B6
:107C2000407900090001C01D48710846007AF02122
:107C300088437030414908720846007A0009000103
:107C400008720846C079F021884370303B49C871FA
:107C50000846C07800090001C01DC8700846807839
:107C6000F021884370303549887008464078F0210B
:107C70008843703031494870084640780009000157
:107C8000C01D4870084600790009000108710846C7
:107C9000C078F021884370302849C8704BE02748ED
:107CA0004079F021884325494871084680780009C9
:107CB000000188700846C07900090001C8710846B3
:107CC00080790009000188710846407900090001A7
:107CD00048710846007AF02188431849087208461E
:107CE000007A0009000108720846C079F021884333
:107CF0001249C8710846C07800090001C8700846DA
:107D00008078F02188430D49887008464078F0213A
:107D100088430A49487008464078000900014870C5
:107D2000084600790009000108710846C078F02172
:107D300088430249C87005B0F0BD00008C260020C1
:107D400070B505460C46012D7ED1B348407D000933
:107D50000001C01DB04948750846007DF0218843E8
:107D60001030AD4908750846007D00090001401C2F
:107D700008750846C07CF02188431030A649C874B5
:107D80000846807CF02188431030A3498874084657
:107D9000807C00090001401C8874F9F75BF8022818
:107DA00003D0F9F757F801286ED19C4800780128D4
:107DB0006AD0F4F7CFFD9A49884265D3F8F7DEFF21
:107DC00000282FD09448007DF021884370309249DC
:107DD00008750846007D00090001C01D08750846A9
:107DE000C07CF021884370308B49C8740846807C81
:107DF000F02188437030884988740846807C0009E7
:107E00000001C01D88740846407DF0218843703011
:107E1000814948750846407CF021884370307E498E
:107E20004874F8E07C48007DF021884310307A499E
:107E300008750846007D00090001401C08750846C9
:107E4000C07CF021884300E0B8E010307249C8746B
:107E50000846807CF021884310306F4988740846BA
:107E6000807C00090001401C88740846407DF02198
:107E700088431030684948750846407CF0218843A3
:107E8000103065494874C6E0F8F742FE002826D154
:107E9000F4F760FD6249884221D3F8F76FFF0028AC
:107EA0000ED05D48407DF021884370305A494875B6
:107EB0000846407CF02188437030574948741CE0E4
:107EC0005548407DF0218843103053494875084695
:107ED000407CF021884310304F4948740DE04E48F3
:107EE000407DF021884370304B4948750846407CFE
:107EF000F0218843703048494874F8F709FE01289A
:107F00002AD146480078012826D0F4F723FD4449B9
:107F1000884221D34048407DF021884370303E495B
:107F200048750846407CF021884370303A494874CF
:107F3000F8F724FF002807D03748007DF021884358
:107F400070303549087566E03348007DF02188437C
:107F50001030314908755EE0230008F07DF9062CE9
:107F6000241C140C042D2C48807C00090001C01D29
:107F70002949887400BF2848807CF02188437030EC
:107F80002549887400BF2448C07CF02188437030A4
:107F90002149C87400BF2048007D00090001C01DB0
:107FA0001D49087500BF1C48007DF02188437030D2
:107FB0001949087500BF00E000BF2CE01648407D5D
:107FC000F0218843144948750846007DF021884314
:107FD000114908750846007D00090001087508462A
:107FE000C07CF02188430C49C8740846807CF0218D
:107FF0008843094988740846807C00090001887418
:108000000846407D0009000148750846407CF02183
:1080100088430149487470BD6C260020050100208A
:10802000B80B000030B50246002901D1002000E065
:108030000720130008F010F90F09141F2B374350C5
:108040005D67727C88929FA9B500574B5B7EF024D8
:10805000A3430401F0252C402343534C6376A1E055
:10806000524B9B79F024A3430401F0252C40234379
:108070004E4CA37196E04D4B2033DB791B091B015D
:108080000407240F2343494C2034E3718AE0464B14
:108090002033DB7C1B091B010407240F2343424CC4
:1080A0002034E3747EE0404B40331B781B091B01F6
:1080B0000407240F23433C4C4034237072E03A4BB6
:1080C0002033DB7FF024A3430401F0252C4023431D
:1080D000354C2034E37765E0334B20335B7BF02471
:1080E000A3430401F0252C4023432F4C2034637319
:1080F00058E02E4B9B791B091B010407240F2343D7
:108100002A4CA3714EE0294B9B7CF024A34304012D
:10811000F0252C402343254CA37443E0234BDB7E06
:108120001B091B010407240F2343204CE37639E08D
:108130001D4B2033DB7F1B091B010407240F234346
:10814000194C2034E3772DE0174B9B7E1B091B0154
:108150000407240F2343144CA37623E0134B20334E
:108160009B79F024A3430401F0252C4023430F4CBA
:108170002034A37116E00D4BDB7D1B091B010407A6
:10818000240F2343094CE3750CE0074B20335B7C41
:108190001B091B010407240F2343034C2034637481
:1081A00000E000BF00BF30BD4C260020202700208B
:1081B000F7B582B00746154600260024FE48007831
:1081C000012804D0F4F7C6FBFC49884279D2FC4868
:1081D000407CF02188437030F94948740846807C1F
:1081E00000090001C01D88740846007D00090001D7
:1081F000C01D08750846007DF02188437030F049A5
:1082000008750846807CF02188437030EC498874FA
:108210000846C07C00090001C01DC8740846C07C27
:10822000F02188437030E649C8740846407C000954
:108230000001C01D48740846407D00090001C01DB2
:1082400048750846407DF02188437030DC49487508
:108250000846007CF02188437030D94908740846EC
:10826000007C00090001C01D08740846C07BF02195
:1082700088437030D249C873BA220A210020FBF724
:108280009BF9BA2213210020FBF796F9BA2211219B
:108290000020FBF791F9BA2212210020FBF78CF99C
:1082A000BA220E210020FBF787F9BA220F21002005
:1082B000FBF782F9BA2210210020FBF77DF9F4E3E5
:1082C000FFE7039836283DD019DC08287ED007DC6C
:1082D000801E030007F0C0FF0635A8FCFBFAF97EFC
:1082E000102874D006DC092872D00D2871D00E2811
:1082F00070D1FDE333286ED03428F9D170E13F28E6
:108300006AD00FDC3738082864D243007B449B884E
:108310005B009F448A009702FF025F005F006503D5
:10832000CB0318004E287BD006DC402879D04128AA
:1083300078D04D28DCD1BBE14F2874D05028D7D15C
:108340004FE100BF00BF9E48407CF02188439C491C
:1083500048740846807C0009000188740846007D46
:1083600000090001C01D08750846007DF021884302
:108370007030934908750846807CF0218843904905
:1083800088740846C07C00090001C01DC8740846F6
:10839000C07CF02188438A49C8740846407C0009A3
:1083A000000148740846407D0009000148750846F0
:1083B000407DF0218843824948750846007CF021C1
:1083C00088437F4908740846007C06E0A1E2FDE38B
:1083D00037E2D2E3FBE394E028E0000900010874EF
:1083E0000846C07BF02188437549C873BA220A2128
:1083F0000020FBF7E1F8BA2213210020FBF7DCF89C
:1084000000220E211046FBF7D7F800220F2110465C
:10841000FBF7D2F8002210211046FBF7CDF877E2E7
:10842000ABE110E2DDE26DE000BF00BF6448407CDC
:10843000F0218843624948740846807C00090001A5
:1084400088740846007D00090001C01D08750846B3
:10845000007DF02188437030594908750846807CBA
:10846000F0218843564988740846C07C0009000101
:10847000C8740846C07CF02188435149C874084636
:10848000407C0009000148740846407D0009000155
:10849000C01D48750846407DF0218843484948750D
:1084A0000846007CF0218843454908740846007C52
:1084B0000009000108740846C07BF0218843404948
:1084C000C873BA220A21002003E055E1EFE086E0FC
:1084D00016E0FBF771F8BA2213210020FBF76CF8C5
:1084E00000220E211046FBF767F800220F211046EC
:1084F000FBF762F8002210211046FBF75DF88EE7CB
:1085000000BF00BF2E48407CF02188432C494874AE
:108510000846807C00090001C01D88740846007D63
:1085200000090001C01D08750846007DF021884340
:108530007030234908750846807CF02188437030EC
:108540001F4988740846C07C00090001C8740846A9
:10855000C07CF02188431A49C8740846407C000951
:10856000000148740846407D00090001487508462E
:10857000407DF0218843124948750846007CF0216F
:1085800088430F4908740846007C000900010874FC
:108590000846C07BF02188430949C873BA220A21E2
:1085A0000020FBF709F8BA2213210020FBF704F89A
:1085B00000220E21104605E005010020B80B000046
:1085C0008C260020FAF7F8FF00220F211046FAF758
:1085D000F3FF002210211046FAF7EEFF1FE700BF5D
:1085E00000BFFE48407CF0218843FC49487408469F
:1085F000807C00090001C01D88740846007D0009C8
:108600000001C01D08750846007DF02188437030C8
:10861000F24908750846807CF0218843EF49887448
:108620000846C07C00090001C8740846C07CF021DF
:108630008843EA49C8740846407C00090001C01D0F
:1086400048740846407D0009000148750846407D91
:10865000F0218843E14948750846007CF0218843B1
:10866000DE4908740846007C0009000108740846C9
:10867000C07BF0218843D949C873BA220A2100205F
:10868000FAF79AFFBA2213210020FAF795FF002289
:108690000E211046FAF790FF00220F211046FAF73C
:1086A0008BFF002210211046FAF786FFF6E300BF89
:1086B000CA48407CF0218843C84948740846807CF9
:1086C0000009000188740846007D00090001087552
:1086D0000846007DF02188437030C049087508467F
:1086E000807CF0218843BD4988740846C07C00091D
:1086F0000001C8740846C07CF02188437030B74937
:10870000C8740846407C0009000148740846407D52
:108710000009000148750846407DF0218843AF49B3
:1087200048750846007CF0218843AC490874084627
:10873000007C0009000108740846C07BF0218843D2
:10874000A649C873BA220A210020FAF735FFBA22D7
:1087500013210020FAF730FF00220E211046FAF70D
:108760002BFF00220F211046FAF726FF00221021CE
:108770001046FAF721FF91E300BF9848407CF021B2
:108780008843964948740846807C00090001887433
:108790000846007D0009000108750846007DF021AB
:1087A000884370308D4908750846807CF0218843E5
:1087B0008A4988740846C07C00090001C8740846CC
:1087C000C07CF02188438549C8740846407C000974
:1087D000000148740846407D0009000148750846BC
:1087E000407DF021884370307C4948750846007C04
:1087F000F0218843794908740846007C000900018B
:1088000008740846C07BF02188437449C873BA22B3
:108810000A210020FAF7D0FEBA2213210020FAF72D
:10882000CBFE00220E211046FAF7C6FE00220F21D1
:108830001046FAF7C1FE002210211046FAF7BCFEDE
:108840002CE300BF00BF6548407CF02188437030B6
:10885000624948740846807C00090001C01D887484
:108860000846007D00090001C01D08750846007D0E
:10887000F02188437030594908750846807CF02102
:108880008843564988740846C07C00090001C874B2
:108890000846C07CF02188435049C8740846407C93
:1088A0000009000148740846407D00090001487530
:1088B0000846407DF0218843484948750846007CB9
:1088C000F0218843454908740846007C00090001EE
:1088D00008740846C07BF02188434049C873BA2217
:1088E0000A210020FAF768FEBA2213210020FAF7C5
:1088F00063FE00220E211046FAF75EFE00220F21D1
:108900001046FAF759FE002210211046FAF754FEDD
:10891000C4E200BF3148407CF02188432F494874AD
:108920000846807C0009000188740846007D000923
:10893000000108750846007DF02188437030274902
:1089400008750846807CF0218843244988740846CD
:10895000C07C00090001C8740846C07CF02188432F
:1089600070301E49C8740846407C000900014874F4
:108970000846407D0009000148750846407DF02109
:108980008843164948750846007CF02188431349FE
:1089900008740846007C0009000108740846C07B82
:1089A000F02188430D49C873BA220A210020FAF742
:1089B00003FEBA2213210020FAF7FEFD00220E2149
:1089C0001046FAF7F9FD00220F211046FAF7F4FDE0
:1089D000002210211046FAF7EFFD5FE28C260020FE
:1089E00000BFFC48407CF0218843FA49487408469F
:1089F000807C0009000188740846007D00090001A0
:108A000008750846007DF02188437030F1490875EB
:108A10000846807CF0218843EE4988740846C07C73
:108A200000090001C8740846C07CF0218843E94968
:108A3000C8740846407C0009000148740846407D1F
:108A40000009000148750846407DF02188437030D8
:108A5000E04948750846007CF0218843DD490874E8
:108A60000846007C0009000108740846C07BF0211C
:108A70008843D849C873BA220A210020FAF79CFD1E
:108A8000BA2213210020FAF797FD00220E2110468A
:108A9000FAF792FD00220F211046FAF78DFD002211
:108AA00010211046FAF788FDF8E1F8E1C948407C4A
:108AB000F02188437030C74948740846807C00091B
:108AC0000001C01D88740846007D00090001C01D1A
:108AD00008750846007DF0218843BE4908750846A0
:108AE000807CF0218843BB4988740846C07C00E044
:108AF000A9E000090001C8740846C07CF021884341
:108B0000B449C8740846407C00090001487408460E
:108B1000407D0009000148750846407DF0218843EA
:108B2000AC4948750846007CF0218843A94908747F
:108B30000846007C0009000108740846C07BF0214B
:108B40008843A449C873BA220A210020FAF734FDE9
:108B5000BA2213210020FAF72FFD00220E21104621
:108B6000FAF72AFD00220F211046FAF725FD002210
:108B700010211046FAF720FD90E19648407CF02144
:108B80008843944948740846807C00090001887431
:108B90000846007D0009000108750846007DF021A7
:108BA00088438C4908750846807CF02188438949B0
:108BB00088740846C07C00090001C8740846C07C5F
:108BC000F02188438349C874084601E09EE003E130
:108BD000407C0009000148740846407D00090001FE
:108BE00048750846407DF02188437A494875084613
:108BF000007CF0218843774908740846007C00090E
:108C0000000108740846C07BF02188437030714928
:108C1000C87300220A211046FAF7CEFC0022132165
:108C20001046FAF7C9FCBA220E210020FAF7C4FC5C
:108C300000220F211046FAF7BFFC00221021104637
:108C4000FAF7BAFC2AE16348407CF0218843614985
:108C500048740846807C0009000188740846007D3D
:108C60000009000108750846007DF0218843594934
:108C700008750846807CF021884356498874084668
:108C8000C07C00090001C8740846C07CF0218843FC
:108C90005049C8740846407C0009000148740846E1
:108CA000407D0009000148750846407DF021884359
:108CB000484948750846007CF021884345490874B6
:108CC0000846007C00090001C01D08740846C07BEE
:108CD000F02188433F49C87300220A211046FAF761
:108CE0006BFC002213211046FAF766FC00220E21CD
:108CF0001046FAF761FCBA220F210020FAF75CFC5B
:108D0000002210211046FAF757FCC7E03148407C9A
:108D1000F02188432F4948740846807C00090001EF
:108D200088740846007D0009000108750846007D2A
:108D3000F0218843274908750846807CF021884344
:108D4000244988740846C07C00090001C87408469C
:108D5000C07CF02188431F49C8740846407C000944
:108D6000000148740846407D000900014875084626
:108D7000407DF0218843174948750846007CF02162
:108D800088437030134908740846007C00090001CC
:108D900008740846C07BF02188430E49C87300223E
:108DA0000A211046FAF708FC002213211046FAF7B0
:108DB00003FC00220E211046FAF7FEFB00220F21D1
:108DC0001046FAF7F9FBBA2210210020FAF7F4FB5B
:108DD00064E000008C260020FB48407CF0218843A2
:108DE000F94948740846807C0009000188740846E7
:108DF000007D0009000108750846007DF0218843C8
:108E0000F14908750846807CF0218843EE49887452
:108E10000846C07C00090001C8740846C07CF021E7
:108E20008843E949C8740846407C00090001487439
:108E30000846407D0009000148750846407DF02144
:108E40008843E14948750846007CF0218843DE49A3
:108E500008740846007C0009000108740846C07BBD
:108E6000F0218843D849C87300220A211046FAF736
:108E7000A3FB002213211046FAF79EFB00220E21CD
:108E80001046FAF799FB00220F211046FAF794FBDF
:108E9000002210211046FAF78FFB00BF00BF002F01
:108EA00003D0CA48007A002804D1F3F753FDC8491B
:108EB000884272D2BA2211210020FAF77DFBBA2231
:108EC00012210020FAF778FBC2480078012804D06C
:108ED000F3F740FDBE49884216D2BF48807BF0219F
:108EE00088437030BC498873084640300078F021D0
:108EF00088437030B849403108700846007800094E
:108F00000001C01D08702DE07D20C000854214D2F4
:108F1000B148807BF0218843AF49887308464030D0
:108F20000078F02188437030AB4940310870084622
:108F3000007800090001087014E0A748807BF02148
:108F400088437030A4498873084640300078F02187
:108F50008843A149403108700846007800090001A3
:108F6000C01D08707D20C000854205D201462846FC
:108F7000EFF7E6F8064604E098492846EFF7E0F8F0
:108F8000064694480078012804D0F3F7E3FC9049A2
:108F9000884203D29248845D02E0A0E29148845D59
:108FA000E007C00F002809D08B484030C078000986
:108FB0000001C01D88494031C87007E08648403034
:108FC000C0780009000184494031C8700220204067
:108FD000002807D08048C07900090001C01D7E49E3
:108FE000C87105E07C48C079000900017A49C87160
:108FF00004202040002807D077488079000900012C
:10900000C01D7549887105E0734880790009000129
:109010007149887108202040002807D06E484079A7
:10902000F021884370306C49487105E06A48407906
:10903000F02188436849487110202040002807D05B
:109040006548407900090001C01D6349487105E089
:1090500061484079000900015F49487120202040A3
:10906000002807D05C480079F021884370305A49C5
:10907000087105E058480079F02188435649087185
:1090800040202040002807D053488079F0218843B1
:1090900070305149887105E04F488079F02188434C
:1090A0004D4988717D20C000854213D26421284635
:1090B000EFF746F8064647480078012804D0F3F752
:1090C00049FC4349884202D24548845D23E0454833
:1090D000845D20E0642128463230EFF731F87D21AD
:1090E000C9000090EFF72CF8019164210198EFF787
:1090F00027F806463C48854208D2364800780128C1
:1091000004D0F3F727FC3249884202D23448845D08
:1091100001E03448845DE007C00F002809D02E48E4
:1091200040308078F021884370302B49403188707E
:1091300007E0294840308078F021884326494031B3
:10914000887002202040002807D02348807A000938
:109150000001C01D2049887205E01F48807A00097F
:1091600000011D49887204202040002807D01A48B9
:10917000407A00090001C01D1749487205E01648F1
:10918000407A000900011449487208202040002854
:1091900007D01148007AF021884370300E490872D8
:1091A00005E00D48007AF02188430B490872102031
:1091B000204000281AD00848007A00090001C01D8C
:1091C0000549087218E000008C2600205C0A002087
:1091D000B80B00000501002000270020A086010038
:1091E0008C1102009F11020010270000FE48007A37
:1091F00000090001FC49087220202040002807D007
:10920000F948C079F02188437030F749C87105E00A
:10921000F548C079F0218843F349C87140202040C7
:10922000002807D0F048407AF02188437030EE499A
:10923000487205E0EC48407AF0218843EA494872D8
:109240007D20C000854219D20A212846EEF778FF1A
:109250000A210190EEF774FF0E460A2D08D2E3486A
:109260000078012804D0F3F775FBE149884202D267
:10927000E048845D12E0E048845D0FE06421284608
:109280003230EEF75DFF0A210090EEF759FF0A2118
:109290000190EEF755FF0E46D6498C5DE007C00FF2
:1092A000002809D0D0484030807800090001C01D56
:1092B000CD494031887007E0CB48403080780009C4
:1092C0000001C9494031887002202040002807D0A1
:1092D000C548807B00090001C01DC349887305E0B3
:1092E000C148807B00090001BF49887304202040E9
:1092F000002807D0BC48407B00090001C01DBA49C6
:10930000487305E0B848407B00090001B64948733E
:1093100008202040002807D0B348007BF021884374
:109320007030B149087305E0AF48007BF0218843F5
:10933000AD49087310202040002807D0AA48C07A01
:1093400000090001C01DA849C87205E0A648C07AFE
:1093500000090001A449C87220202040002807D03D
:10936000A148807AF021884370309F49887205E0D7
:109370009D48807AF02188439B4988724020204094
:10938000002807D09848407BF021884370309649E8
:10939000487305E09448407BF02188439249487324
:1093A0007D20C000854207D20A212846EEF7C8FE7C
:1093B0000E469048845D0BE0642128463230EEF77B
:1093C000BFFE0A210190EEF7BBFE0E4689498C5D77
:1093D000E007C00F002809D0834840304078F021D2
:1093E0008843703080494031487007E07E48403003
:1093F0004078F02188437C49403148700220204069
:10940000002809D078484030407800090001C01D8C
:1094100075494031487007E0734840304078000992
:10942000000171494031487004202040002807D0D5
:109430006D48007CF021884370306B49087405E06A
:109440006948007CF021884367490874082020405F
:10945000002807D06448007C00090001C01D624953
:10946000087405E06048007C000900015E4908744A
:1094700010202040002807D05B48C07BF0218843A3
:1094800070305949C87305E05748C07BF0218843C4
:109490005549C87320202040002807D05248C07B7F
:1094A00000090001C01D5049C87305E04E48C07B4B
:1094B000000900014C49C87340202040002807D013
:1094C0004948407C00090001C01D47494874ECE050
:1094D0004548407C0009000143494874E5E000220A
:1094E0000A211046FAF768F8002213211046FAF70D
:1094F00063F8002211211046FAF75EF800221221CB
:109500001046FAF759F800220E211046FAF754F8DF
:1095100000220F211046FAF74FF8002210211046C2
:10952000FAF74AF830484030C078000900012E4967
:109530004031C8702C48C079000900014039C87119
:109540000846807900090001887108464079F021B9
:10955000884325494871084640790009000148714F
:1095600008460079F02188431F4908710846807930
:10957000F02188431C498871084640308078F021EA
:1095800088431949403188701748807A00090001E2
:10959000403988720846407A00090001487208463E
:1095A000007AF0218843104908720846007A0009C1
:1095B000000108720846C079F02188430A49C87141
:1095C0000846407AF02188430749487208464030EF
:1095D000807800090001403188700348807B0009D1
:1095E00000014039887309E00027002005010020B0
:1095F000B80B00008C1102009F1102000846407B4E
:109600000009000148730846007BF021884328497F
:1096100008730846C07A00090001C8720846807ABB
:10962000F0218843224988720846407BF021884314
:109630001F494873084640304078F02188431C4950
:1096400040314870084640780009000148701848C9
:10965000007CF0218843164908740846007C000904
:10966000000108740846C07BF02188431049C87384
:109670000846C07B00090001C8730846407C000909
:10968000000148740846807BF021884308498873AC
:10969000084640300078F021884305494031087081
:1096A0000846007800090001087005B0F0BD000010
:1096B00000270020F7B582B007460E460121FF20A3
:1096C0000830FBF7A7FF0121FC48FBF7A3FFFC488C
:1096D000007801287ED0F3F73DF9FA49884279D322
:1096E000F7F728FA032843D1F7F71EFA002803D02A
:1096F000F7F71AFA01283BD1002F1CD1F7F73EFBF0
:1097000000280CD0F048407CF0218843EE49487492
:109710000846807C00090001C01D8874EEE0EA481C
:10972000407CF0218843E84948740846807C000961
:1097300000018874E2E0F7F721FB00280CD0E24832
:10974000407CF02188437030DF4948740846807CB3
:10975000000900018874D1E0DB48407CF021884397
:10976000D94948740846807C000900018874C5E026
:10977000F7F7DAF9002803D0F7F7D6F9012865D111
:10978000002F0CD1D048407CF0218843CE4948744A
:109790000846807C00090001C01D88740BE0CA489F
:1097A000407CF02188437030C74948740846807C6B
:1097B000000900018874F7F7B7F9002821D1C248E1
:1097C0002030C078F02188437030BF492031C87004
:1097D000BD4800E064E0807D000900012039887503
:1097E0000846807DF0218843B7498875BA22232135
:1097F0000020F9F7E1FE002222211046F9F7DCFEF5
:109800007CE0F7F791F9012878D1AF482030C07893
:10981000F0218843AC492031C870AB48807D0009F5
:109820000001C01D203988750846807DF0218843DD
:109830007030A5498875002223211046F9F7BCFE37
:10984000BA2222210020F9F7B7FE57E09E48407C5B
:10985000F02188439C4948740846807C0009000137
:10986000887408462030C078F0218843964920311A
:10987000C8709548807D0009000120398875084628
:10988000807DF0218843904988750022232110466D
:10989000F9F792FE002222211046F9F78DFE2DE005
:1098A0008948407CF02188437030874948740846D5
:1098B000807C00090001C01D887408462030C078F3
:1098C000F0218843703080492031C8707E48807D07
:1098D00000090001C01D203988750846807DF021EF
:1098E0008843703078498875BA2223210020F9F71F
:1098F00063FEBA2222210020F9F75EFEF7F714F981
:10990000002808D06E480078012804D0F3F722F828
:109910006C49884276D26D48864209D96A4820301F
:109920004079F0218843703067492031487107E061
:10993000654820304079F0218843634920314871DF
:1099400063493046EEF7FCFB0A210190EEF7F8FB85
:109950000D465E48401C864202D35E48445D01E0ED
:109960005D48445DE007C00F002809D0564820300C
:10997000C07800090001C01D53492031C87007E0BC
:1099800051482030C078000900014F492031C8708B
:1099900002202040002809D04B4820308078F02158
:1099A0008843703048492031887007E046482030AD
:1099B0008078F02188434449203188700420204079
:1099C000002809D0404820304078F021884370308A
:1099D0003D492031487007E03B4820304078F02175
:1099E00088433949203148700820204000280AD097
:1099F00035482030407900090001C01D324920312E
:109A0000487108E0A1E230482030407900090001A7
:109A10002D492031487110202040002809D02A48C3
:109A200020300079F02188437030274920310871B7
:109A300007E0254820300079F02188432249203171
:109A4000087120202040002809D01F4820300079CC
:109A500000090001C01D1C492031087107E01A48A7
:109A60002030007900090001174920310871402099
:109A70002040002809D014482030807800090001D7
:109A8000C01D11492031887007E00F4820308078D0
:109A9000000900010C49203188707D21C900304641
:109AA000EEF74EFB0A210190EEF74AFB0D460848FF
:109AB000864213D30748445D12E00000050500000C
:109AC00005010020B80B0000002700209F86010040
:109AD000102700008C1102009F110200F948445D1C
:109AE000E007C00F002807D0F748C07FF021884367
:109AF0007030F549C87705E0F348C07FF02188430E
:109B0000F149C87702202040002807D0EE48C07FE6
:109B100000090001C01DEC49C87705E0EA48C07F94
:109B200000090001E849C87704202040002807D038
:109B3000E548807F00090001C01DE349887705E002
:109B4000E148807F00090001DF4988770820204034
:109B5000002809D0DC482030407800090001C01DF1
:109B6000D9492031487007E0D748203040780009B3
:109B70000001D5492031487010202040002809D02C
:109B8000D14820300078F02188437030CE49203110
